:020000040000fa
:0800000024510400000000007f
:020000040000fa
:10a00000245104000000000082e904000100000067
:10a0100082e904000100000082e904000100000060
:10a0200082e904000100000082e904000100000050
:10a0300082e904000100000082e904000100000040
:10a0400082e904000100000082e904000100000030
:10a0500082e904000100000082e904000100000020
:10a06000bae60400010000002ae304000100000039
:10a0700082e904000100000082e904000100000000
:10a0800010ea040001000000dce904000100000007
:10a0900082e904000100000082e9040001000000e0
:10a0a00082e904000100000082e9040001000000d0
:10a0b00082e904000100000082e9040001000000c0
:10a0c00082e904000100000082e9040001000000b0
:10a0d00082e904000100000082e9040001000000a0
:10a0e00082e9040001000000fee704000100000016
:10a0f00082e904000100000082e904000100000080
:10a1000082e904000100000082e90400010000006f
:10a1100082e904000100000082e90400010000005f
:10a1200082e904000100000082e90400010000004f
:10a1300082e904000100000082e90400010000003f
:10a1400082e904000100000082e90400010000002f
:10a1500082e904000100000082e90400010000001f
:10a1600082e904000100000082e90400010000000f
:10a1700082e904000100000082e9040001000000ff
:10a1800082e9040001000000e0ea04000100000090
:10a1900082e904000100000082e9040001000000df
:10a1a00082e904000100000082e9040001000000cf
:10a1b00082e904000100000082e9040001000000bf
:10a1c00082e904000100000082e9040001000000af
:10a1d00082e904000100000082e90400010000009f
:10a1e00082e904000100000082e90400010000008f
:10a1f00082e904000100000082e90400010000007f
:10a2000082e904000100000082e90400010000006e
:10a2100082e904000100000082e90400010000005e
:020000040000fa
:10a248004f092400007f240000018800000000005e
:10a258000c000700e0932f001100200011000700f8
:10a26800000020000000e0000200320000000200b0
:10a2780000000000a8090200020000000040da0007
:10a288000000fe004440a900a00625000000e000f0
:10a298000300320010002000a00188004440a800fc
:10a2a8000000060091018800800078000000eb00a3
:10a2b80015003700e280400032a0b4009101ba00d6
:10a2c800e280400032a0b4009102ba00e28040006f
:10a2d80032a0b4000002eb00472bde00f507b20005
:10a2e800602ce10004003a000059eb008301e9000a
:10a2f800fdff3e00040037006128e1000100320044
:10a308000082eb00040007001101ba000200e0001f
:10a31800e8ff3a00000006003159ba008301e9005d
:10a328000c0032002159ba008301e900080032000c
:10a338000400e00003003a00e280400032a0b400cc
:10a34800f5ff370011d9ba008301e900faff3a0096
:10a358008100e800e180400032a0b400000006005f
:10a36800cefa040000000000fcf904000000000020
:10a37800c2f8040000000000ccf80400000000004f
:10a38800eaf8040000000000fcf8040000000000e7
:10a39800e8d0040000000000fafa04000000000001
:10a3a8000afb04000000000030fb0400000000006d
:10a3b80056fb04000000000086fb040000000000bb
:10a3c800b0fb040000000000c2fb04000000000015
:10a3d800dcfb04000000000062f80400000000003c
:10a3e8007af804000000000092f804000000000061
:10a3f800aaf8040000000000ecfb040000000000c4
:10a40800b4f90400000000006af90400000000002c
:10a4180010fc04000000000034fc040000000000f0
:10a4280048fc0400000000005efc0400000000007e
:10a438006efc0400000000007efc04000000000028
:10a448008efc0400000000009efc040000000000d8
:10a45800c6fc040000000000eefc04000000000040
:10a468001efd04000000000056fd0400000000006e
:10a4780068fd04000000000070fd040000000000fa
:10a4880080fd04000000000090fd040000000000b2
:10a49800bcfd040000000000e8fd0400000000000e
:10a4a800f8fd04000000000008fe040000000000a1
:10a4b80018fe04000000000028fe04000000000050
:10a4c80038fe04000000000054fe040000000000f4
:10a4d8005efe0400000000006efe040000000000a4
:10a4e8008cfe0400000000009cfe04000000000038
:10a4f80032ff040000000000c8ff04000000000054
:10a50800f8ff04000000000028000400010000001b
:10a518004800040001000000580004000100000089
:10a52800a400040001000000f00004000100000085
:10a538002001040001000000500104000100000097
:10a548007001040001000000800104000100000007
:10a558009801040001000000a801040001000000a7
:10a56800c001040001000000d00104000100000047
:10a57800f6010400010000001c02040001000000b4
:10a588006c02040001000000a803040001000000a0
:10a59800ba03040001000000ca030400010000001f
:10a5a800da030400010000000004040001000000b8
:10a5b8002604040001000000060504000100000054
:10a5c800180504000100000028050400010000002f
:10a5d80038050400010000006c05040001000000bb
:10a5e800a205040001000000740604000100000038
:10a5f800b606040001000000f8060400010000008f
:10a608003407040001000000700704000100000086
:10a61800c605040001000000d60504000100000082
:10a62800e6050400010000001a060400010000000d
:10a638005006040001000000920704000100000019
:10a64800b407040001000000a8080400010000008d
:10a658009209040001000000b8090400010000008c
:10a66800de09040001000000f009040001000000f8
:10a67800000a0400010000001c0a04000100000098
:10a688004c0a0400010000009c0a040001000000bc
:10a69800c20a0400010000008a0b04000100000047
:10a6a800540c040001000000b40c04000100000078
:10a6b800ec0c040001000000fc0c04000100000088
:10a6c800120d040001000000220d0400010000002a
:10a6d800820d040001000000ba0d04000100000012
:10a6e8005a0d040001000000320d040001000000b2
:10a6f800440e040001000000500e04000100000098
:10a70800600e040001000000800e0400010000003b
:10a71800ce0e0400010000001c0f04000100000020
:10a728007410040001000000d011040001000000b2
:10a73800f0110400010000001a12040001000000da
:10a748004412040001000000f2130400010000009c
:10a75800ac15040001000000cc1504000100000045
:10a76800f615040001000000201604000100000096
:10a778004c170400010000006a18040001000000e2
:10a78800ac18040001000000bc180400010000001f
:10a79800f21804000100000018190400010000006c
:10a7a8007619040001000000ce1904000100000021
:10a7b800e619040001000000f61904000100000079
:10a7c800061a0400010000001a1a04000100000023
:10a7d8002a1a0400010000006c1a0400010000009d
:10a7e800c01a040001000000d41a0400010000008f
:10a7f800e41a040001000000261b04000100000008
:10a808007a1b0400010000008e1b040001000000f8
:10a81800b41b040001000000c41b04000100000078
:10a82800ea1b040001000000fa1b040001000000fc
:10a838000a1c0400010000001a1c040001000000aa
:10a848002a1c040001000000541c04000100000040
:10a858006c1c0400010000009a1c040001000000a8
:10a86800ca1c040001000000dc1c040001000000f8
:10a87800ec1c040001000000121d0400010000008f
:10a88800381d040001000000461d040001000000fe
:10a89800521d040001000000621d040001000000b8
:10a8a800781d040001000000881d0400010000005c
:10a8b800a81d040001000000c01d040001000000e4
:10a8c800cc1d040001000000e21d0400010000008e
:10a8d800b4540400000000003200f8009101880020
:10a8e8008002780062004000e08048003549ba00e4
:10a8f8003204e0000410a700100032008301e900d0
:10a908000e0032002549ba003204e0000410a70006
:10a918000a0032008301e900080032000408a3009d
:10a92800eeff320015c9ba003204e0000410a70097
:10a93800020032008301e900e8ff3a003200f90022
:10a94800000006008001eb000200370081717800ea
:10a958008301e800828f5100fcff3a0000000600e6
:10a96800881f7800020478001c00070008004000d7
:10a978004f047800000006000000fa00881f7800e5
:10a98800000478003fb99700ea81570080007800fa
:10a99800404b250018000700800078000000e00008
:10a9a800020035000040eb0000f478000100780058
:10a9b8004f0478000080fa0000000600800178004b
:10a9c8000001780031407800005978000004e00068
:10a9d800fcff3a0003007800000006008001eb004d
:10a9e8000200370061f079008301e800828f51008e
:10a9f800fcff3a00000006006200fa00889fbe00d3
:10aa08008a9fbe000004be0002057800830078001b
:10aa180060f92f000f004000b000070088979f00e2
:10aa280099979f000000eb00a09f9f009a4578002f
:10aa38000b80fb000000ea00cf04de0050c2b30028
:10aa480080cf550002003200090478000100370069
:10aa58000904e9000800e0000b0034001f9097008b
:10aa6800080178008a0078008f91970003000100a0
:10aa780090979f000000e000930032002f98970005
:10aa880000004400a09f9f000905450050c2b30084
:10aa980080cf5500040032000b04e000e3ff3a00c9
:10aaa8002f989700890037000000eb00809f9f00d7
:10aab800f0979f00e0979f00d0979f00c0979f0056
:10aac800b0979f00c09f9f000900370040002400f6
:10aad800008050000000400081ff2300e100780062
:10aae8004f98970001007000c09f9f000a05e8007a
:10aaf8001a4478008800fb00400024007c0007000e
:10ab0800800078000000e000f0ff3a00a0c2b30027
:10ab1800804f54000e003a00bf8897000180e9007a
:10ab2800b08f9f0010007800b09f9f000000e000e9
:10ab380005003d000000ea00b09f9f004f98970075
:10ab48000020a000c09f9f000a05e8001000370001
:10ab5800b19f9f0003fd2f00f4ff27000800370076
:10ab68003f989700840f5000040032006a00b90033
:10ab78000000410003004000b09f9f000a05e80064
:10ab88001a01fb0003004100e90f5000f4ff3600f2
:10ab9800e0c2b3009a4f1000040032000080eb00be
:10aba800909f9f008a0478001c0037008a04e80000
:10abb800a0c2b300994f100007003a00bf88970061
:10abc8000180e900b08f9f0010007800909f9f00df
:10abd8008a84e800110037000000eb00909f9f0076
:10abe80003fd2f00f4ff2700080037001f98970087
:10abf800840f5000040032006a00b90000004100d0
:10ac080003004000909f9f008904e8001901fb00a1
:10ac180003004100e90f5000f4ff360019447800a2
:10ac28008800fb00a0032400310007000000e000ba
:10ac380002003a0000447800010037008904e80067
:10ac4800a87f9f0080c6b300804f540004003a00dc
:10ac5800994f14000a003a00664050000600370079
:10ac6800c0c6b300804f540005003a00994f140045
:10ac780003003a0065404000a07f9f008904e80077
:10ac88000905e800c8fb2f000f04440060f92f00f5
:10ac98000f0040008085e80088017800194178009d
:10aca800800078000b0078001a0007000000e00020
:10acb80005003a00880078000b0078009201070030
:10acc8000000e00059ff3d000080eb004f05be008a
:10acd8004f04be000080fa00000006000200fa00df
:10ace800f1bf9f00010878000080fa00000006000c
:10acf800040037000204e00001003a0000000500eb
:10ad08000000e80010417800814f5100f9ff3a0037
:10ad180000000600889fbe008a1f780000047800a3
:10ad280001027800824478000305780070c6b300f9
:10ad3800804f510021003c0000c0e900804f5100c5
:10ad4800de003d0072405000804f51004b01320040
:10ad58000d003c006c405000804f51005e013c00eb
:10ad680000c0e900804f5100d4003d0050c2b3003c
:10ad7800804f5100550132007c404000804f510007
:10ad880055013a00cd00370010c6b300804f51007e
:10ad9800ca00320004003c0069405000804f510056
:10ada8004d013a007200370030c6b300804f5100a1
:10adb800180032000040e8000900370000c7b3005f
:10adc800804f51001e01320008003c0000c0e9001d
:10add800804f5100e400320065003c00654050009f
:10ade80080cf54003c013a000f00370050c7b30031
:10adf800804f51005e00320063404000804f510098
:10ae08005b00320065405000804f510032013a002b
:10ae18001a0137009180e900010a78007800900053
:10ae28009171780032013700a8609000c0c6b30065
:10ae380080cf50000a003a009400780064805000e7
:10ae4800000a78001000be004f89de00cf91de00b6
:10ae58000002be0002037800820378001300370066
:10ae680010c7b30080cf500003003200a0c6b30063
:10ae780080cf500006003a009400780068805000a7
:10ae8800000a78003002be002003be000700370029
:10ae98001480e900000a78001000780000027800a9
:10aea800cfa2de000503780086037800049cbe006c
:10aeb8000694be00a860900080c6b30080cf500002
:10aec8000e00320020c6b30080cf500005003a00c3
:10aed8000400fb00cf80de000101780082017800c9
:10aee8000a00370040c7b30080cf5000030032008b
:10aef8006640400080cf500006003a000400780009
:10af0800cf80de000101780082017800009cbe003d
:10af18000294be003800be002801be00e00f5000b9
:10af2800e08f5800e00f5900e08f590003003d0002
:10af380078009000d1c2b3000a00370008109000d2
:10af48000018a3000300320078009000b1c2b300db
:10af5800040037000008a300530032007800900076
:10af680001c2b300017578000000e8004d00370009
:10af7800a8609000c0c6b30080cf500006003a0019
:10af88009400780064805000000a78001002be0027
:10af98006033b8001300370010c7b30080cf5000eb
:10afa80003003200a0c6b30080cf500006003a006c
:10afb8009400780068805000000a78003002be00d3
:10afc8002003be00070037001480e900000a78005b
:10afd800100078000002780005002000060020001c
:10afe80007002000049cbe000694be00a8609000e4
:10aff80080c6b30080cf50000e00320020c6b300d8
:10b0080080cf500005003a000480fb0001002000ba
:10b0180002002000030020000a00370040c7b300e8
:10b0280080cf5000030032006640400080cf5000bf
:10b0380006003a0004007800010020000200200009
:10b0480003002000009cbe000294be00081090007f
:10b058000038a300140032003800be002801be00ea
:10b06800e00f5000e08f5800e00f5900e08f5900c2
:10b078000d00320080c7b30080cf540003003200b7
:10b0880080c5b30080cf540007003a0078009000d4
:10b0980001c3b300017578008000e80009f5780065
:10b0a8000080e800700498007800900000004500d7
:10b0b80060049800894078006d003700a86090000f
:10b0c800c0c4b30080cf500006003a009400780056
:10b0d80068805000000a78005001be004000be00a1
:10b0e800050037009400780064805000000a78005a
:10b0f8001000be0089080700009cbe000294be0034
:10b10800380090000000e00003003d007800900047
:10b11800d1c2b3000a003700081090000018a3003d
:10b128000300320078009000b1c2b3000400370079
:10b138000008a300050032007800900001c2b300a7
:10b14800017578000000e80070049800780090000d
:10b1580000004500600498008940780008007800e5
:10b168003301070064003700a8609000c0c6b30030
:10b1780080cf5000250032000a003c006440500097
:10b1880080cf50002800320000c0e80080cf500077
:10b19800140032006840500080cf500022003a006e
:10b1a8000a00370040c7b30080cf50001e003200ad
:10b1b8006640400080cf50001b00320069405000bc
:10b1c80080cf500018003a00060037001480e900cc
:10b1d800000a780010007800485c90000848780061
:10b1e800450037001480e900000a78001002780052
:10b1f80068089000cf80de000101780082017800a5
:10b20800009abe000292be003b0037001480e9009d
:10b21800000a78001001780068089000cf80de00ee
:10b228000089be00340037001480e900000a780065
:10b2380010007800680c9000080878002e0037008d
:10b248001180e9008008780010007800cf80de00c7
:10b258000101780082017800009cbe000294be00c3
:10b2680078009000000045006004980081c7b30092
:10b2780008007800170307001f0037001480e90052
:10b28800000a7800100078006004980058099000bf
:10b298000200e00002003d009704070009003700a3
:10b2a8008000eb009b040700800078000000e000ad
:10b2b8000300320068009000008050000100370051
:10b2c80058089000100c98000b0037007800900088
:10b2d800027578000600370078009000800045006d
:10b2e8000904e00001003a0059c2b3008948780017
:10b2f8000000e800700498000000eb004f0578009b
:10b308004f04be00000006000400fa00889fbe003b
:10b318008a9fbe008c1f7800000478000106780020
:10b3280070089000f8009000010050008808900014
:10b33800010050009808900001005000a8089000f3
:10b3480001005000b808900001005000c8089000a3
:10b35800810550000002220090bf9f0000032300d7
:10b36800a0bf9f00081090000028a30018003a0012
:10b378000b00e000160034008b0478000905780003
:10b38800e28f5400020036002a0020000200370035
:10b398000900e0000b00340058009000c80190003c
:10b3a8000a017800ee80570003000100500498005d
:10b3b8000000e00096003200680890000000450098
:10b3c800600c98008a8454004240a900ebff3c00be
:10b3d800780190000200e0000b0034005800900053
:10b3e800c80190008c007800030001005004980008
:10b3f8000000e0008600320068089000f800900025
:10b4080001004000600c9800880c90000900e000e2
:10b418001500340009057800e28f54000200360058
:10b428002a002000020037000900e0000b00340069
:10b4380058009000c80190000a017800ec8057007d
:10b4480003000100500498000000e0007000320082
:10b458006808900000004500600c98008a84540039
:10b468004240a900ebff3c00180990000200e000f0
:10b478000b003400e800900058009000c8019000cc
:10b4880003000100500498000000e0006000320052
:10b49800680890009808900001004000600c98002f
:10b4a800a80c90000900e000150034000905780098
:10b4b800e28f5400020036002a0020000200370004
:10b4c8000900e0000b00340058009000c80190000b
:10b4d8000a017800ec80570003000100500498002e
:10b4e8000000e0004a0032006808900000004500b3
:10b4f800600c98008a8454004240a900ebff3c008d
:10b50800380990000200e0000d003400e8009000c7
:10b51800180890008080400058009000c8019000f2
:10b5280003000100500498000000e00038003200d9
:10b5380068089000b808900001004000600c98006e
:10b54800c80c90000900e0001500340009057800d7
:10b55800e28f5400020036002a0020000200370063
:10b568000900e0000b00340058009000c80190006a
:10b578000a017800ec80570003000100500498008d
:10b588000000e0002200320068089000000045003a
:10b59800600c98008a8454004240a900ebff3c00ec
:10b5a800081090000028a3001b0032000b00e000e8
:10b5b800190034008b04780009057800e28f5400e4
:10b5c800020036002a002000020037000900e000cf
:10b5d8000b00340058009000c80190000a01780060
:10b5e800ee80570003000100500498000000e000be
:10b5f800070032006808900000004500600c9800c1
:10b608008a8454004240a90003003400eaff37004e
:10b618000080eb00010037000000eb004f067800c7
:10b628004f05be004f04be000080fa00000006006f
:10b638008f04b000889fbe008a9fbe008c9fbe000a
:10b648008e1f7800f0b79f0081f79f005001be0061
:10b658004000be00f0979f00819f9f00929f9f002f
:10b66800a39f9f0010c6b3000ff19700804f5100b1
:10b678001600320010c4b300804f5100130032008e
:10b68800ffb19700530890000000e00003003d0060
:10b6980060002000d00998000c0037000000e0008e
:10b6a8000a003a0070c6b3000ff29700804f5200ac
:10b6b8000300320070c4b300804f520003003a0008
:10b6c80010002000ffb29700d00a9800ffb0970042
:10b6d800c0fa2f000f00400098030700800178008f
:10b6e800e20f500015003a0030002000ffb097002c
:10b6f8009008980010c6b3000ff19700804f5100d2
:10b708000a00320064404000804f510007003200b8
:10b718000040e800804f51000400320041f123004e
:10b728000040e800804f510001003a0081f12300f9
:10b73800ffb1970063009000160037000000e0009a
:10b7480018003400300020007fb29700100a9800db
:10b7580010c6b3008ff2970080cf52000a00320063
:10b768006440400080cf5200070032000040e800eb
:10b7780080cf520004003200c1f123000040e800ed
:10b7880080cf520001003a0001f223007fb19700f8
:10b7980062009000315878003158780011487800dc
:10b7a800c601370014c6b3008ff2970084cf520049
:10b7b8000300320010c4b30080cf520013003a00d7
:10b7c8007fb09700600190008200780000c3b3004a
:10b7d80080587800ffb29700e102980080c7b30054
:10b7e8008ff2970084cf52000100320080c5b30069
:10b7f800804878000280e800ffb09700e0009800d9
:10b80800710090000080e800f00098000300e0005c
:10b8180005003a00e3979f0064fb2f000f014200e8
:10b8280003077800a001370045f22300e5b79f0021
:10b8380010c6b3008ff0970080cf5000050032008b
:10b8480010c4b30080cf5000a7003a0052f3230081
:10b85800e2b79f00ffb19700530890001e02200036
:10b868000000e000010035000007e8000e02e800d3
:10b87800d4b79f006022b8006033b8007f9097006b
:10b888008f9897001f999700af999700c2060700f5
:10b89800ffb097003102be002103be000000e000a7
:10b8a80004003d000400be000601be0003f0a20033
:10b8b800020037000400be000601be00f0979f009a
:10b8c800819f9f00929f9f00a39f9f006f91970069
:10b8d80064015100e2979f00c3fa2f008f81410055
:10b8e8006a8041000048eb006b824100c4b79f00aa
:10b8f80031003700c201200003002000e5fa2f00c4
:10b908000f804200390307007f9497008f9c9700af
:10b918001f9d9700af9d97000800be000a01be005a
:10b92800a20607000006be005fb19700670151003c
:10b93800d2b79f004240a9000a003400c70607009a
:10b948000002be000203be000800be000a01be00dd
:10b95800c5060700f0979f00819f9f00929f9f0058
:10b96800a39f9f00cfb1970067804100710020001e
:10b97800050037006f6066004c6add004466de0033
:10b988000c067200c4eede00e00f5600e08f5e0089
:10b99800050034008100e900e18f4000f5ff3a001e
:10b9a800010037000060eb008100e900fdff3b006b
:10b9b80067004000c0b79f00dfb297000500e000b5
:10b9c800090034006022b8006033b8007f90970007
:10b9d8008f9897001f999700af999700a4060700c2
:10b9e8000000e000c3ff3c0060fb2f008f00400018
:10b9f8004fb19700010051000000e9008e0f500080
:10ba080001003d00000778000e00e00003003d0043
:10ba180073fb2f000f8141002c003700800f570067
:10ba280005003d000e80400010409000f3c0b300b8
:10ba3800e74f500001003c008041eb00c4fa2f00a2
:10ba48000f0242000e0042006a0040008e0078009b
:10ba5800010037000000e9008100e900104178008a
:10ba6800834f5100fbff32000107e800efcf510080
:10ba780001003a000248e8000100e0000300350038
:10ba880075fb2f000f814200060037000e07e80003
:10ba98006f90970064004000e0979f0061fb2f00c3
:10baa8000f8140008e0041008e01780003003700ae
:10bab8001100fb006fb29700e44878008301e900a9
:10bac8008100e9000300e000f9ff3d00ffb29700a4
:10bad800550890000000e000f3003d000e00e9006a
:10bae800d00a9800f00037007f9497008f9c970049
:10baf8001f9d9700af9d97006022b8006033b80083
:10bb08000800be000a01be00230607000000e0008e
:10bb180005003d000bf0a200f8979f00899f9f0049
:10bb28009a9f9f00ab9f9f006f90970072592700c4
:10bb38000280b900026a280013002000510607009d
:10bb4800e4005000e1979f0015003b00e3801000df
:10bb5800c0ff2f00008460000800ea00e0979f0003
:10bb68007f9097008f9897001f999700af9997003b
:10bb7800c9ec2300070037000808a30003003200bf
:10bb88003902be002903be004d0607000884d10013
:10bb9800e88444000800e000f7ff3c001b00370081
:10bba8000100e0001d003400c0ff2f00008060008d
:10bbb800e0979f00000478006000b80002002000b1
:10bbc80003ff2300c9ec2300070037000808a3007f
:10bbd800030032003902be002903be003806070000
:10bbe8000884d100e88444000800e000f7ff3c0026
:10bbf8000002be000203be007f9097008f98970056
:10bc08001f999700af999700a2060700f0979f0029
:10bc1800819f9f00929f9f00a39f9f00ffb0970066
:10bc28005109900060c6b3008ff1970080cf510092
:10bc3800040032006100200060c4b30080cf5100ce
:10bc480002003a006f929700ea00420001074100a3
:10bc5800f30f5700010034003e01200000c3b30079
:10bc6800e0779f0075fb2f008f824200b5b79f00d9
:10bc7800330037000800be000a01be00cb050700ec
:10bc88000006be00680757004240a9000e003400b5
:10bc9800f20507000002be000203be000800be0055
:10bca8000a01be00f00507006022b80046782d00a2
:10bcb8007719240002060700f0979f00819f9f00d4
:10bcc800929f9f00a39f9f003fb097006804400089
:10bcd800890020000d003700a40020000500200086
:10bce8000c01be00e0fd2f000f004000ba02070063
:10bcf8007fa897008fb097001fb19700afb197004a
:10bd080004c3b300046441000006be00e00f5600ff
:10bd1800e08f5e00060034008904e900e18f4400ea
:10bd2800edff3a000200370000c3b300006478005a
:10bd38008904e900fcff3b0068044400b8b79f0091
:10bd48000e00e0000b0034007f9497008f9c970052
:10bd58001f9d9700af9d97006022b8006033b80020
:10bd68000800be000a01be00c10507000000e0008f
:10bd7800c0ff3c00c5fa2f008f8242006a80420053
:10bd8800bfb09700008050008001e9006f919700d4
:10bd9800e70041006b81420000c3b3000100370097
:10bda8000201e800924f1000fdff320074fb2f00e3
:10bdb8000f004200808040008280500000804100d7
:10bdc80002025000e1979f00ffb29700d50990004a
:10bdd80060c6b3008ff2970080cf52000300320094
:10bde80060c4b30080cf520002003a008100e8002e
:10bdf8000a00370050c6b3008ff0970080cf50007c
:10be0800050032008000eb0050c4b3008ff29700a9
:10be180080cf520001003a00110020000187410044
:10be28008e0f520001003d00040778000e00e0006c
:10be38001d003500840f570005003d00e2407f00db
:10be480095c3b30040c3b30080cf500001003c004d
:10be580005c3b3000e0041008000e9008e017800a0
:10be6800010037008100e9008301e90011427800f0
:10be7800854f5200fbff32000307e80090c3b30070
:10be880080cf520001003a008448e8000300e00037
:10be980005003d000201e9000e07e8006f909700d9
:10bea8000000e800e0979f006f9297008e017800ed
:10beb8008ff097007fb09700640207004f07780063
:10bec8004f06be004f05be004f04be008f04b100f0
:10bed800000006002f03b000889fbe008a9fbe00a6
:10bee8008c9fbe008e1f78000007780010f8230092
:10bef800c0b79f0080c5b30080cf50000800320053
:10bf080002f72300c2b79f007740400080cf50005f
:10bf180003003a0083002000b3b79f000a003700ef
:10bf280080c7b30080cf500005003200a400200075
:10bf3800b4b79f0080c5b30080cf500002003a001c
:10bf480005012000b5b79f003e04be002e05be00c7
:10bf580040c6b30080cf5000030032006540400067
:10bf680080cf50000b003a00e00f5400e08f5c00d7
:10bf7800e00f5d00e08f5d0006003d006000b80046
:10bf88006011b80008045000898458000a05590057
:10bf98008b855900bfb39700e88f53000300320028
:10bfa800f08f530045003a000200370036002000a9
:10bfb8000100370046002000e00f5400e08f5c00cd
:10bfc800e00f5d00e08f5d0005003a005e0890001c
:10bfd80081012000a1b79f000000e00008003200a6
:10bfe8003fb197000200e90008006000cfb1970058
:10bff8006340780090df9f0074012000a4b79f0081
:10c00800860278008502e900050033008b05d1001f
:10c018000a85d3008984d3000884d300f9ff370048
:10c02800089fbe000a97be00afb397000700e9005b
:10c0380021fc2f008f804000008240003fb1970014
:10c048008202e90012003700afb397008703e900c6
:10c05800a7b79f0000806200cfb0970061527800b8
:10c068003e00be002e01be00860378008703e9006b
:10c07800050033008381d1000281d3008180d30081
:10c088000080d300f9ff3700009fbe000297be0072
:10c098003e00be002e01be00e00f5000e08f5800a9
:10c0a800e00f5900e08f5900d6003400afb3970075
:10c0b8000700e000e4ff3c00d2003700ae609000cb
:10c0c80080c6b30080cf50000b00320006003c0051
:10c0d8000104e000080032006640500080cf5000a4
:10c0e80073003a0004003700c0c6b30080cf500088
:10c0f8006f003a0031003700080178000800e000be
:10c1080005003a005e08900081012000a1b79f0059
:10c118000000e00009003200bfb1970011000900db
:10c128000381d8008000fd004fb29700644078007a
:10c1380090df9f0075012000a5b79f00bfb397004f
:10c14800110009000781d80080017800afb097007e
:10c158000100e90022fc2f000f014100000241000c
:10c168000c003700bfb29700110009008501d80004
:10c1780000017800afb397008703e900a7b79f00d5
:10c188000590b90000805100cfb097006152780047
:10c19800820178000300e000030034002fb197000b
:10c1a8000200e000efff3c0003007800cf80de00d3
:10c1b80001017800820178003a0037000806be00c5
:10c1c800e00f5400e08f5c0005003a005e08900024
:10c1d80083012000a3b79f000000e000090032009f
:10c1e8003fb297006121b9000c00be00f5030700bb
:10c1f800cfb297006540780090df9f00770120005c
:10c20800a7b79f003fb297006121b9000c00be009c
:10c21800dc0307000006be00afb297000500e90086
:10c2280027fc2f008f8343008083430097b79f002c
:10c23800110037003fb197006114b9000801be0032
:10c248000c00be008f0407000005be00afb19700c8
:10c258008301e900a3b79f000801be000603070099
:10c26800000056001fb29700cfb2970065527800c1
:10c2780094b79f000a06be00e00f5600e08f5e00ec
:10c2880003003400afb397000700e000e9ff3c006b
:10c298004feade00cfa2de000c00be0004017800e9
:10c2a80084017800009fbe000297be005500370049
:10c2b800e00f5400e08f5c00e00f5d00e08f5d0050
:10c2c80005003a005e08900081012000a1b79f0098
:10c2d8000000e0000d0032003fb197000202780034
:10c2e800cfa2de0005037800860378000800be00b0
:10c2f8000a01be00c20507004fb2970064407800eb
:10c3080090df9f0075012000a5b79f003fb19700ff
:10c3180002027800cfa2de000503780086037800c9
:10c328000800be000a01be00ae050700009fbe005f
:10c338000297be00afb197000300e90024fc2f006c
:10c348000f0242000006420020003700bfb29700eb
:10c3580005047800cfc4de00090578008a05780056
:10c368000802be000a03be005fa89700efa8970066
:10c378007fa997008fb19700a5050700d0b79f0048
:10c38800e1b79f00f2b79f0083bf9f00afb397004c
:10c398008703e900a7b79f000802be000a03be0092
:10c3a800210607005faa970000005200cfb297004d
:10c3b800655678005fb09700efb097007fb197009f
:10c3c8008fb99700009fbe000297be003e00be00d6
:10c3d8002e01be00d0af9f00e1af9f00f2af9f00db
:10c3e80083b79f00e00f5000e08f5800e00f59001e
:10c3f800e08f590003003400afb097000100e0005f
:10c40800d2ff3c003fb19700e80f510013003a00fb
:10c418000e1090000038a30010003200afb1970052
:10c42800f78f510006003e0024fc2f000f02420047
:10c438008300420000c3b300914f10000700320090
:10c44800afb297008502e900a5b79f0000c3b3000b
:10c4580027fc2f008f83430080f37a00afb1970049
:10c4680078811100120f98006e00900024fc2f00b4
:10c478000f0242008300420058f907001e0990008d
:10c488005e089000800f510006003d000200500039
:10c49800000f98000e1090000040a10000179800af
:10c4a8000f0037000000e0000d003d000e10900066
:10c4b80074006000f00f500009003a007e089000f8
:10c4c800fe009000010050008e089000010050000e
:10c4d800020050004240a90001003400000f9800fb
:10c4e8004f0778004f06be004f05be004f04be0040
:10c4f8002f03b1000000060080007800010037001b
:10c508000000e8001004e000fdff3a0001005000c0
:10c51800000006008001eb00040037008301e800fa
:10c5280090cf1000040032000000e800828f510014
:10c53800faff3a000000eb0000000600889fbe00ea
:10c54800800478006684400000ff2700180060001f
:10c558004401de00f07f2000800f51000e003a00f9
:10c56800800ceb00180478006f0064001c003a008f
:10c57800210090000000e00019003a00110090002e
:10c588000000e00016003a00100020001100e00052
:10c5980014003200120037000200e00005003c00e1
:10c5a80001007800dd010700000178000000e000cc
:10c5b80008003c00f00028001800600001fe23007d
:10c5c800010c700020c02f00800c41000080eb009f
:10c5d80004003700800ceb000000eb00010037007e
:10c5e800200020004f04be0000000600889fbe0007
:10c5f8008a1f78008c9fbe00000478000206be00e7
:10c60800e6044000190178000200d0004505de006c
:10c618008a007800f07f2000800f55000c003a0057
:10c628006f00610067003a00280090000000e000f9
:10c6380064003a00180090000000e00061003a0031
:10c64800100020001800e0005f0032005d00370095
:10c658000a00e00007003a0008007800af01070070
:10c66800800078000000e000020034000a00780032
:10c67800550037006108b9000c0140008d81480061
:10c68800e07f2000800f5100e08f59000d0034003a
:10c698001900e00004003d006000b800020020001e
:10c6a80003ff2f00030037006000b80002002000dd
:10c6b80003ff2700009cbe000294be00100020006b
:10c6c80041003700e00f5100e08f590005003400a9
:10c6d800f000280019006000c410dd00810c700013
:10c6e80036003700190078000100280001036000b7
:10c6f8006f0060000040a000800c780061015100cc
:10c70800e0815900c0fc2f00f1ff2f00800f51007d
:10c71800818f590006003d00860c78000000eb0070
:10c728002004980010049800000c780026003700b8
:10c73800020078000881e800e400440005003700a2
:10c74800120c78001109780099087800800ceb0029
:10c7580070004000f00f4000f9ff34008002ea004a
:10c76800150032008881e800708212009800780075
:10c778008508de00130078000400dd00008c7000de
:10c7880064014400930078008508de0012007800f8
:10c798000400dd0080897000920078008508de00c2
:10c7a800190078000400dd00008970001900780085
:10c7b8000500de00800c7800990c73000080eb0007
:10c7c80001003700200020004f06be004f0578000a
:10c7d8004f04be00000006000400fa00889fbe0057
:10c7e8008a9fbe008c1f78000006780092bf9f00c9
:10c7f800a3bf9f000404be000401be001fb8970039
:10c80800afb897001f0307000005be000001be0077
:10c818000800be00980107001fb99700afb997003c
:10c8280000005100818059002006980031069800c8
:10c838000a8ebe000c0078004f0678004f05be0037
:10c848004f04be000080fa00000006000e00fa0047
:10c85800889fbe008a9fbe008c9fbe00000478009f
:10c868000145780002067800830478008406780081
:10c878000300e00002003c00190020000c0924001d
:10c8880060c6b300804f55000e00320060c4b3008c
:10c89800804f55000b00320070c6b300804f550022
:10c8a8000300320070c4b300804f55009c003a006a
:10c8b800e48f46008000350058089000808f5600ad
:10c8c8007d003d008d05e80060c6b300804f55002f
:10c8d8001000320060c4b300804f55000d003200d4
:10c8e800081090000038a30004003a00580890008f
:10c8f800808f540001003d00590c980058089000a2
:10c908000b005000500c980002003b000000eb00a8
:10c91800500c98000b00e00027003c00180990001c
:10c928006800900001c3b300017079008201e8003b
:10c93800130c9800580890000000e00003003c0029
:10c94800081090000038a30005003200680090002d
:10c95800e1c2b30001f079000280e800100c9800f1
:10c96800d80890000b00ea00808f500001003d00bd
:10c978008105ea000b00ea00200c980001804500c0
:10c98800500c9800890f500001003d008004780089
:10c99800390c980068009000980890000100400049
:10c9a800090178008c0078000cf8070058089000fe
:10c9b800090050001a00370098089000680090009d
:10c9c8008b8f540018003d000100400009017800d9
:10c9d8008c00780001f807001808900000814400d6
:10c9e800120c980009805500200c980058089000f7
:10c9f8000000e00003003c00081090000038a3008d
:10ca080006003200e8009000e0c2b30080707900b0
:10ca1800380890000000e800300c98005808900092
:10ca2800400c9800a6003700010040000b01780078
:10ca38008c007800e9f7070018089000008145008d
:10ca4800120c98008b845400580890000000e000f5
:10ca580003003c00081090000038a30005003200d5
:10ca680068009000e1c2b300017079000200e8009c
:10ca7800100c980058089000890f500001003d00e4
:10ca88008004780068009000980890000100400039
:10ca98008b00460009017800d0f7070018089000bd
:10caa80000804400100c98005808900009005000bd
:10cab800200c98008200370070c6b300804f5500e4
:10cac8000300320070c4b300804f550014003a00d0
:10cad80058089000808f540004003d000810900012
:10cae8000038a30001003a00590c9800580890003b
:10caf8000000e900500c980002003b000000eb0029
:10cb0800500c980070c6b300804f550002003a00e0
:10cb18005ac6b3000b0037005ac4b30009003700e7
:10cb280010c6b300804f550002003a000ac7b30090
:10cb38000400370010c4b300804f550001003a00cc
:10cb48000ac5b30018099000680090003c7079008d
:10cb58008201e800130c98000c0278005808900035
:10cb68000000e00003003c00081090000038a3001b
:10cb780017003200e8009000e0c2b30080f07900ae
:10cb88008280e800110c9800580890000000e0002e
:10cb98000f0034008904e900890f500001003d00ae
:10cba8008004780068009000008040000901780047
:10cbb8008400780089f70700180890000080440076
:10cbc800100c98005808900009005000200c98009c
:10cbd8006800900098089000010040000086e80076
:10cbe8000a587800800078000d00e0000400350045
:10cbf800b0c2b300804878008c0478000400370085
:10cc0800d0c2b300804878008c0478008d06ea0012
:10cc18008005eb000a003700a20020008d00780094
:10cc280070805700890007000fb897009fb89700d9
:10cc38007a81550001f17f008b05e80080067800b5
:10cc48000d00e000f4ff3c00e18f550009003c00b6
:10cc580050c6b300804f55000300320050c4b300e3
:10cc6800804f550003003a0000c3b300005e78000f
:10cc78008c0478000b00e000040032000b00e9008f
:10cc8800fa805700008040000600370000c3b30058
:10cc9800805c7800050037008b05e90002c3b3000b
:10cca800a05c41000b00e000fbff3c006800900026
:10ccb800980890000100400000805400300c980053
:10ccc8000810900074006000f00f50000e003a0049
:10ccd800780090009808900001004000a808900093
:10cce80001004000b808900001004000c80890000a
:10ccf8008100400078089000808f500002003d00bd
:10cd080001005000000c98004f06be004f05be0001
:10cd18004f04be000080fa00000006000001780001
:10cd2800e60140001300780001002800810360003c
:10cd38006f0060008009780012003a00220090001d
:10cd48000000e0000f003a00120090000000e00030
:10cd58000c003a00160020001200e00038003200f3
:10cd680008003700e4004100910978000280e800db
:10cd780090087800120878000009eb00700353004f
:10cd880001003700160020001300e000f5ff320014
:10cd9800e40241000282e8001100370080004000f0
:10cda800150078004f00de0080897000950078003b
:10cdb80081804000140078004f00de00808a7000f7
:10cdc8009400780081804000120078004f00de0057
:10cdd800008a700012007800000940000603e9008c
:10cde80013007800ef0f5000ecff36008282e80055
:10cdf800640241000e0037009200d100150078004f
:10ce08004f00dd00008970009500d1001400780003
:10ce18004f00dd00808a70009400d1001300780074
:10ce28004f00dd00008a70009309d1000603e80076
:10ce380013007800ff0f5000efff3e00ef0960007d
:10ce4800938973000600780000000600020278004b
:10ce5800809fbe00110009008200d8000001780000
:10ce68004f00be0002a2b900848050001100980053
:10ce78000208780000000600020ab900001bb90089
:10ce88000200b80081004200810043000000060053
:10ce9800889fbe008a9fbe00010578000100e0005f
:10cea8000400350008003c000000e00020003200cb
:10ceb8000500370060001000e080180002003b0009
:10cec80001f02c001a0037000004be006011b80001
:10ced8006b0920000982cf00020039000882cf00c8
:10cee8000441b000694252000e00320008003b00c5
:10cef80082817100610164008904d1000884d30033
:10cf08008b05e8000442e800f9ff3a000500370005
:10cf18000804440089844c008b05e9000442e900b8
:10cf2800fbff3a00aa0007000af0a70001f0a000e2
:10cf38004f05be004f04be000000060003f0a2002b
:10cf4800889fbe008a9fbe008c1f7800c60007001d
:10cf5800cd0033006450e1004f0032006420e1004e
:10cf68005200320003826c0007003b000905d00024
:10cf78000306d000820f54000c065d000200390041
:10cf88000200320089017800030678008582550086
:10cf980004003d000003fd008103fd008502ea0056
:10cfa8008b854200840f720002003b006000100075
:10cfb800e08018006011b8000005eb007a28e10055
:10cfc8000a00390006007800c75ddd00f707b200e7
:10cfd800878075002d003700828171000a01780072
:10cfe800610560008180d1000080d3008502e900de
:10cff800f9ff3b00060440008784480002003b001c
:10d0080060041400e0841c000988a30007003200b3
:10d018008a81710082817100610164008904d100f4
:10d028000884d3008b05e800170037000978a300af
:10d0380013003a000b00e000130034008b05e900f0
:10d048000804440089844c000a4474000978a30049
:10d058000d003a000b00e000070034008b05e900e2
:10d068000804440089844c0001003a000b002000a9
:10d078000978a300f7ff32000001eb000200370037
:10d08800828171000a017800510007000cf0a700a6
:10d0980001f0a000850037006420e10002003a009a
:10d0a800838f6c00850033000801be000200be00bb
:10d0b8007e003700889fbe008a9fbe008c1f7800c4
:10d0c800690007007000330003866c006450e100bb
:10d0d800240032006420e100270032006150e100a2
:10d0e800220032006120e100210032008b854200dd
:10d0f800eb07b1000134b800003ab8000804420058
:10d1080089844a00013ab8000030b800888040009d
:10d1180009014a00040033000000400081804800f3
:10d12800020149008b05e900c909dd00830170008f
:10d138000100320013002000c814de004814dd008e
:10d148004709de001200b200c808de00088470003b
:10d158001f00070001f0a1000cf0a70001f0a000db
:10d16800520037006120e100540032000801be007f
:10d178000200be00f7ff37006150e100fcff3a00f3
:10d188004e0037006022b800060220000000d000e0
:10d198008180d2000482d2008582d2000000a000e3
:10d1a8000202520083825a00030031000202420048
:10d1b80083824a000000a1000603e900f3ff3a0059
:10d1c80000000600efff07000400be000000060094
:10d1d80081002000618055000b003d000b002000fd
:10d1e80061fe2f000100e1001d0034008281710002
:10d1f800610164008904d1000884d3000000e800bc
:10d20800faff3a007100200061006400030070001a
:10d21800020060000900320061044400e0844c0010
:10d228000988a500050032008b05e8006808e100c0
:10d2380002003a008904d1000884d300f20f2000cc
:10d248000258e10005003d00c75ddd00f907b200a6
:10d258008980750008007800000006000bf8270098
:10d268008b007800000005000004be0016000700cf
:10d278000003be000405be000200be001200070045
:10d28800844f7500000006000200be006450e100f3
:10d29800050036006420e100020036000968a3009a
:10d2a80001003a000800be000160a0004f067800a7
:10d2b8004f05be004f04be0000000600f0ff2f001f
:10d2c800f1ff2700f9ff3700c70ade00f107b200b7
:10d2d800f50fb20008003200e1cf42000200320030
:10d2e8000170a00024000500810f700001003200c9
:10d2f8000408050044000500810f700002003a0090
:10d30800140005008502e9000000400081c04800c3
:10d31800fcff3b000170a000240005008103780099
:10d32800e9ff07000001be006000b8000478a30010
:10d3380013003a006220e10015003e000d0039009c
:10d348008301d1000281d3008180d3008301d10001
:10d358000281d3008180d3008301d1000281d300f0
:10d368008180d3000538b000c42add00f300b20084
:10d378008381720007f0a70003f0a00000000600f8
:10d38800f3ff2700f2ff2f006110b900fbff370001
:10d3980003ff2700f7ff37008f1fd1005002070057
:10d3a8008f87e9000000e000000006001400fa0082
:10d3b800889fbe008a9fbe008c9fbe000004be00ee
:10d3c8000205be00680047000a90be000890be0033
:10d3d8006c0207000070a7000bf0a100304320008a
:10d3e8009e02900080825200b0fe2f000028e100cb
:10d3f80011003d00b0fc2f000028e10015003400aa
:10d408001e0990008e0890007e0090000501b00073
:10d418000201d1008180d3000080d3008502e8009a
:10d42800fbff3a000b00e00091023b006000100097
:10d43800e08018008e023700f0ff2f00f1ff270070
:10d448000b00e0008a023b000100280000002000d9
:10d45800870237006000b800850237004f89de0078
:10d46800820178008702370007f0a200bc0237006b
:10d47800809feb001a0207008f87e9000000e00098
:10d4880000000600839f68000100e00002003d00e4
:10d4980060001000e08018000300e00002003d007a
:10d4a80060011100e081190036ff07004f00e0001d
:10d4b80002003b0060001000e08018000000060039
:10d4c8002800fa00889fbe008a9fbe008c9fbe007d
:10d4d80003866b00520207000028a30064003a008c
:10d4e8000128a30067003a000008a30062003a0080
:10d4f8000108a30065003a001e009000be089000d5
:10d5080081064000ed3fb100f4805700ee01900025
:10d51800111ab8008e099000311bb8009e099000be
:10d52800311cb800511db800f485570046000700ab
:10d53800fe0190003a0007008b85e8003e000700d6
:10d548008e09900040000700ee01900034000700ab
:10d558008b85e800380007008e099000400007001e
:10d568009e0990001b18b800890440000a854800ed
:10d57800fe019000340007008b85e80038000700a2
:10d58800ee019000300007008e0990001b18b800cb
:10d59800890440000a8548000a98a30008003a0058
:10d5a8000402420085824a0006034b0087834b0031
:10d5b80008044c0089844c000a054d008d06e900da
:10d5c80084827200850273004c3add008502720085
:10d5d8000100320015002000443ade001400b200b9
:10d5e8004538de00cb45dd000b007000c540de008d
:10d5f800cb4ddd008b8070004549de00cb55dd004a
:10d608000b017100c551de000d037800d10207003f
:10d6180003f0a1000cf0a70003f0a00014023700eb
:10d628001b18b8008502400006834800e0834b00c1
:10d6380060044c00070037001b18b80006034000c0
:10d6480087834800faff37001b18b800870340009b
:10d6580008844800e0844c0060054d000000060086
:10d668001b18b8000804400089844800faff3700f6
:10d678000108a300fb013a005800be005801be0093
:10d68800e3ff37000008a300f6013a000904780018
:10d69800f9ff37002800fa00889fbe008a9fbe0065
:10d6a8008c9fbe0003866b00dd0107006400e1006b
:10d6b800440032006408e1004a0032006100e100e1
:10d6c800460032006108e10049003200ec064700dc
:10d6d8006000b8003d02be003d03be00f48657005e
:10d6e8006011b8003d04be003d05be007d0320006a
:10d6f8000b0037000000a0008d06e900130032007f
:10d708000402420085824a0006034b0087834b00cf
:10d7180000004000818048000201490083814900df
:10d728000802520089825a000a035b008b835b005f
:10d73800f0ff3b000802420089824a000a034b00be
:10d748008b834b008d06e900edff3a00848272005e
:10d7580086827200f707b2008782720001003200e9
:10d76800150020001e0490003e0b90000603540094
:10d77800e63fb0000368a300070032000000a700de
:10d788000500a0008301d1000281d3008180d3006d
:10d798000080d3000603e8008301d1000281d30092
:10d7a8008180d3000080d3000002eb000482d20005
:10d7b8006802070003f0a1000cf0a70003f0a00026
:10d7c800ab013700640247006408e100a50132009c
:10d7d8003400be003401be00f6ff37006108e100e6
:10d7e800a00132006011b8006000b800f1ff3700f6
:10d7f80003ff270002002000fbff3700881f780086
:10d80800000478005001be004000be000400400043
:10d81800858048000601490087814900009cbe00b8
:10d828000294be000400e1000588e1000690e100d2
:10d838000798e10002003100680044001008e80081
:10d848004f04780000000600f4874700889fbe0058
:10d858008a9fbe008c9fbe008e1f78000205be0006
:10d868000004be00d4b79f00e5b79f00f6b79f003d
:10d8780087bf9f000000eb00c0b79f00b0b79f00b4
:10d88800a0b79f0090b79f0080b79f000d042000ad
:10d89800bfb097004fb09700000140000000e000c3
:10d8a8000f003d004f08de0000007100c0b79f0068
:10d8b8009e00070001003d0012002000a1000700a3
:10d8c80001003d0012002000a6000700b10007007b
:10d8d800b60007000f004000c8ff0700220037000d
:10d8e8004f08de0000067100ccb79f008f000700cc
:10d8f80001003d00120020009200070001003d00d9
:10d908001200200097000700a20007000fb297003e
:10d918009fb297002fb39700bfb39700a9000700e5
:10d928000000520081805a0002015b0083815b0085
:10d9380080b79f0091b79f00a2b79f00b3b79f0021
:10d948000007eb009f0007000020e10001a8e100ac
:10d9580002b0e10003b8e100010031001e00200020
:10d968000e005600c0b79f004fb297000400e000b9
:10d978000700350010002000010020006011b800e9
:10d9880008047000898470000a0571008b85710095
:10d998008d06e900beff3a000400e00003003d00e8
:10d9a800820007000f00400094ff07004fa897006f
:10d9b8000000e00004003a000fb497009fb49700fd
:10d9c8002fb59700bfb59700940007004f07780060
:10d9d8004f06be004f05be004f04be004f01b10008
:10d9e80000000600881f780018002000881f7800b3
:10d9f80095ff07008f87e9004f04780000000600b4
:10da0800801feb0090ff07008f87e90000000600e9
:10da1800889fbe008a9fbe008c1f78006e0007009a
:10da280007003d0073000700e00f5b00e08f5b001c
:10da380007003d00320007000006eb000400370035
:10da48003400070002003d002a0007001c002000e7
:10da580072000700e3ff07000203be000002be00d9
:10da68000c00e00001003200220007000400be00a4
:10da78000601be004f0678004f05be004f04be00e9
:10da880000000600889fbe008a9fbe008c1f780099
:10da98005100070005003d0056000700e00f5b003d
:10daa800e08f5b0006003d00040037001900070006
:10dab80003003d006000b8006011b80010000700c6
:10dac80056000700ceff07000203be000002be009a
:10dad8000c00e00001003200060007000400be0050
:10dae8000601be004f0678004f05be004f04be0079
:10daf800000006006000b8006011b80000003700a0
:10db08000402500085825800060359008783590093
:10db1800000006000006eb00e00f5200e08f5a00fc
:10db2800e00f5b00e08f5b00000006000180400012
:10db380090b79f000001eb008fb097000100e00054
:10db4800000006000200700090b79f0001804000ae
:10db580080b79f000001eb00ffa897000100e000dc
:10db6800000006000200700080b79f00018040009e
:10db78006faa9700cf20de0001007000f0af9f0071
:10db880004024200250007004f18de000002720060
:10db980000000600e4af9f000804440089844c009c
:10dba8000a054d008b854d00000006003fb2970026
:10dbb800cfb297005fb39700efb3970000fe2f0036
:10dbc800000006003fb09700cfb097005fb1970004
:10dbd800efb19700000006000205be000004be0079
:10dbe800e00f5000e08f5800e00f5900e08f590017
:10dbf800000006006000b8006011b800080450007a
:10dc0800898458000a0559008b8559001c0020009a
:10dc1800e00f5200e08f5a00000006000800be0026
:10dc28000a01be0000000600889fbe008a9fbe0051
:10dc38008c1f78000205be000004be000006eb0041
:10dc4800e00f5000e08f5800e00f5900e08f5900b6
:10dc580007003d006000b8006011b80008045000db
:10dc6800898458000a0559008b8559001c0020003a
:10dc7800e00f5200e08f5a00e00f5b00e08f5b007e
:10dc880002003d000f0007000c00a2000800be00c3
:10dc98000a01be005b0107000203be000002be00cd
:10dca8000c00e00001003200060007000400be007e
:10dcb8000601be004f0678004f05be004f04be00a7
:10dcc800000006006000b8006011b80004025000af
:10dcd8008582580006035900878359000000060012
:10dce800889fbe008a9fbe008c9fbe000404be00b1
:10dcf8000605be00809fbe00829fbe00630107002c
:10dd0800040678000800be000a01be005f01070093
:10dd1800840678004f03be004f02be008d4f760088
:10dd28007fb0970013003300f0ff2f008b8f6b003c
:10dd380006003b000d0666000c00a7000a0037002d
:10dd480007f0a600100020000a003700880f5200d4
:10dd5800898f5a008a0f5b008b8f5b0003003900a4
:10dd68001000200001003e000000200007f0a7007e
:10dd78000000ea004f06be004f05be004f04be007b
:10dd880000000600800078005002be005003be006c
:10dd98004439de00f700b200f37f20000301610080
:10dda800090032000218e10016003a0085017200ed
:10ddb80083017300838173000008200015003a0076
:10ddc80040002000130037008501720083017300b2
:10ddd8008381730005003a0004a8be0006a8be00af
:10dde800100020000b0037000201e9000402420085
:10ddf80085824a0006034b0087834b000748a3002f
:10de0800f9ff32000740a00004a8be0006a8be0023
:10de18002000200080009800920098000000060072
:10de2800680447000294be000094be00fc0447004a
:10de38008694be008494be0009007800d1ff0700d4
:10de480008007800cfff070099007800814f700024
:10de58000b003b000800be001e0107004f00b10088
:10de680003003700f3ff2700f2ff2f006110b9000d
:10de78004f06be004f05be004f04be000080fa00ea
:10de880000000600889fbe00830478000300e000bd
:10de98002c00350003003c00008270000402710071
:10dea8002600320036432000c50020008383cf00bf
:10deb8000a0039000541b1008283cf00070039000c
:10dec8000541b1008183cf00040039000541b1004c
:10ded8008083cf00010039000541b10085c353009c
:10dee8006022b800120032000a003b0084827200ef
:10def800610260008301d1000281d3008180d300d8
:10df08000080d3000603e8008743e800f7ff3a00e3
:10df180007003700000040008180480002014900e6
:10df2800838149000603e9008743e900f9ff3a00c5
:10df38008800070009f0a70003f0a0004f04be0006
:10df48000000060060001000e08018006001190061
:10df5800e0811900d3ff3b00033e2c00f7ff370098
:10df68002800fa00889fbe008a9fbe008c9fbe00d2
:10df780007067800878669000c003b0003047800d8
:10df88008704780008f0a10009f0a100840f500070
:10df9800858f5800860f5900890f5c0003003300f5
:10dfa8000cf0a20001003a000cf0a1009cff070051
:10dfb8006400e1005f003200780147006408e10076
:10dfc800610032006c014700748557003200be00c2
:10dfd8001201be003a04be001a05be001e039000de
:10dfe800be0a90008503530006003d000004fd00b2
:10dff8008104fd000205fd008305fd008703ea009a
:10e00800050378000df8a300040032006004140032
:10e01800e0841c0060051d00e0851d006022b8003a
:10e028007d0320000d38e1008006eb000b0039006d
:10e038004433dd00f300b200830173003900370078
:10e04800848272000d027800e10664008b85d1009d
:10e058000a85d3008984d3000884d3008703e900a4
:10e06800f7ff3b0008004000898048000a0149008a
:10e078008b81490004003b0060001000e08018001c
:10e0880060011900e08119000358a300090032005b
:10e098008d82720084827200610260008301d10067
:10e0a8000281d3008180d3000080d3000603e800fa
:10e0b8001b0037000348a30017003a000600e000e1
:10e0c800170034000603e9000d00a3000000480013
:10e0d8008180480002014900838149000348a30068
:10e0e8000f003a000600e000090034000603e900ca
:10e0f80000004000818048000201490083814900f6
:10e1080001003a000003eb000348a300f5ff3200ca
:10e118006022b800020037008482720061826600c3
:10e128000c00070003f0a1000cf0a70003f0a0000a
:10e138004fff3700640147006408e10002003a001d
:10e148000df8a30047ff3a003200be001201be00de
:10e1580047ff37001800200057002000080453002c
:10e168000d003d000600200097fc2f000740e1004d
:10e178001e00340084827200610260008301d100b5
:10e188000281d3008180d3000080d3000804e80016
:10e19800f8ff3a004700200061046000050474009d
:10e1a800040464000d00320061004000e080480073
:10e1b80060014900e081490003b8a500070032006a
:10e1c8000603e8006538e10004003a008301d10045
:10e1d8000281d3008180d3000080d300f87f200023
:10e1e8000830e10003003500080378006000b8003b
:10e1f8006011b8004433dd00f300b20083017300fe
:10e2080000000600889fbe008a9fbe008c9fbe004b
:10e218000404b8000506b8008904460060854e006d
:10e228000606b8000a054600e0854e000706b80055
:10e238008b054600040eb800890446000a854e0086
:10e24800e0854d00050eb8000a0546008b854e0096
:10e25800060eb8008b0546000416b8000a054600ed
:10e268008b854e000516b8008b054600041eb800c5
:10e278008b0546000800be000a01be004f06be001e
:10e288004f05be004f04be000000060005ff270032
:10e2980005826100070032000428e1000100320015
:10e2a800240005000600070001003a0044000500ac
:10e2b8000408050002000700f9ff3a0014000500f1
:10e2c8006f82610081027000850271008502720010
:10e2d80000000600e48240001078a3000700320026
:10e2e800640240001178a3003400be001401be008f
:10e2f800040032000330a700000006003500be000d
:0ce308001501be000330a000000006005c
:020000040000fa
:020000040005f5
:0457f400051e00008e
:020000040000fa
:020000040005f5
:0457f8004d0300005d
:020000040000fa
:020000040005f5
:0457fc00fa3f000070
:020000040000fa
:1000080082e9010082e9010082e9010082e9010038
:1000180082e9010082e9010082e9010082e9010028
:1000280082e9010082e9010082e9010082e9010018
:1000380082e9010082e9010082e90100bae60100d3
:100048002ae3010082e9010082e9010010ea0100c7
:10005800dce9010082e9010082e9010082e901008e
:1000680082e9010082e9010082e9010082e90100d8
:1000780082e9010082e9010082e9010082e90100c8
:1000880082e9010082e9010082e9010082e90100b8
:10009800fee7010082e9010082e9010082e901002e
:1000a80082e9010082e9010082e9010082e9010098
:1000b80082e9010082e9010082e9010082e9010088
:1000c80082e9010082e9010082e9010082e9010078
:1000d80082e9010082e9010082e9010082e9010068
:1000e80082e9010082e9010082e9010082e9010058
:1000f80082e9010082e9010082e9010082e9010048
:1001080082e9010082e9010082e9010082e9010037
:1001180082e9010082e9010082e9010082e9010027
:1001280082e90100e0ea010082e9010082e90100b8
:1001380082e9010082e9010082e9010082e9010007
:1001480082e9010082e9010082e9010082e90100f7
:1001580082e9010082e9010082e9010082e90100e7
:1001680082e9010082e9010082e9010082e90100d7
:1001780082e9010082e9010082e9010082e90100c7
:1001880082e9010082e9010082e9010082e90100b7
:1001980082e9010082e9010082e9010082e90100a7
:1001a80082e9010082e9010082e9010082e9010097
:1001b80082e9010082e9010082e9010082e9010087
:1001c80082e9010082e9010082e9010082e9010077
:1001d80082e9010082e9010082e9010082e9010067
:1001e80082e9010082e9010082e9010082e9010057
:0801f80082e9010082e9010027
:020000040000fa
:1002080082e9010082e9010082e9010082e9010036
:1002180082e9010082e9010082e9010082e9010026
:1002280082e9010082e9010082e9010082e9010016
:1002380082e9010082e9010082e90100bae60100d1
:100248002ae3010082e9010082e9010010ea0100c5
:10025800dce9010082e9010082e9010082e901008c
:1002680082e9010082e9010082e9010082e90100d6
:1002780082e9010082e9010082e9010082e90100c6
:1002880082e9010082e9010082e9010082e90100b6
:10029800fee7010082e9010082e9010082e901002c
:1002a80082e9010082e9010082e9010082e9010096
:1002b80082e9010082e9010082e9010082e9010086
:1002c80082e9010082e9010082e9010082e9010076
:1002d80082e9010082e9010082e9010082e9010066
:1002e80082e9010082e9010082e9010082e9010056
:1002f80082e9010082e9010082e9010082e9010046
:1003080082e9010082e9010082e9010082e9010035
:1003180082e9010082e9010082e9010082e9010025
:1003280082e90100e0ea010082e9010082e90100b6
:1003380082e9010082e9010082e9010082e9010005
:1003480082e9010082e9010082e9010082e90100f5
:1003580082e9010082e9010082e9010082e90100e5
:1003680082e9010082e9010082e9010082e90100d5
:1003780082e9010082e9010082e9010082e90100c5
:1003880082e9010082e9010082e9010082e90100b5
:1003980082e9010082e9010082e9010082e90100a5
:1003a80082e9010082e9010082e9010082e9010095
:1003b80082e9010082e9010082e9010082e9010085
:1003c80082e9010082e9010082e9010082e9010075
:1003d80082e9010082e9010082e9010082e9010065
:1003e80082e9010082e9010082e9010082e9010055
:0803f80082e9010082e9010025
:020000040000fa
:104800000100000000000000006100000120000025
:10481000c0000000005a00000000000055550000d4
:1048200055550000555500005555000055550000e0
:1048300055550000555500005555000055550000d0
:1048400055550000555500005555000055550000c0
:1048500055550000555500005555000055550000b0
:1048600055550000555500005555000055550000a0
:104870005555000055550000555500005555000090
:104880005555000055550000555500005555000080
:104890005555000055550000555500005555000070
:1048a0005555000055550000555500005555000060
:1048b0005555000055550000555500005555000050
:1048c0005555000055550000555500005555000040
:1048d0005555000055550000555500005555000030
:1048e0005555000055550000555500005555000020
:1048f0005555000055550000555500005555000010
:1049000055550000555500005555000055550000ff
:1049100055550000555500005555000055550000ef
:1049200055550000555500005555000055550000df
:1049300055550000555500005555000055550000cf
:1049400055550000555500005555000055550000bf
:1049500055550000555500005555000055550000af
:10496000555500005555000055550000555500009f
:10497000555500005555000055550000555500008f
:10498000555500005555000055550000555500007f
:10499000555500005555000055550000555500006f
:1049a000555500005555000055550000555500005f
:1049b000555500005555000055550000555500004f
:1049c000555500005555000055550000555500003f
:1049d000555500005555000055550000555500002f
:1049e000555500005555000055550000555500001f
:1049f000555500005555000055550000555500000f
:104a000055550000555500005555000055550000fe
:104a10005555000055550000555500000000000098
:104a20000000000000000000000000000000000086
:104a30000000000000000000000000000000000076
:104a40000000000000000000000000000000000066
:104a50000000000000000000000000000000000056
:104a60000000000000000000000000000000000046
:104a70000000000000000000000000000000000036
:104a80000000000000000000000000000000000026
:104a900000000000000000000000000020200000d6
:104aa000505200004f5400004543000020360000e3
:104ab000313000003020000046490000524500001f
:104ac000202000000020000020200000434f0000b4
:104ad0004e540000524f00004c2000005041000096
:104ae0004e4500004c200000202000002000000067
:104af00020200000504100004e4500004c200000e6
:104b00005445000058540000204c0000494e00005d
:104b1000452000003320000000200000205000004d
:104b2000414e0000454c0000205400004558000054
:104b3000542000004c4900004e4500002034000085
:104b40002000000044450000564900004345000095
:104b5000205400004558000054200000414400004b
:104b6000442000003120000020200000004400000c
:104b70004556000049430000452000005445000010
:104b8000585400002041000044440000203200003e
:104b9000202000002000000044450000564900008d
:104ba00043450000205400004558000054200000f8
:104bb0004144000044200000332000002020000079
:104bc0000044000045560000494300004520000015
:104bd00054450000585400002041000044440000a7
:104be0002034000020200000200000004445000088
:104bf000564900004345000020540000455800007d
:104c000054200000414400004420000035200000f2
:104c100020200000004400004556000049430000e9
:104c20004520000054450000585400002041000079
:104c30004444000020360000202000002000000036
:104c40004445000056490000434500002054000040
:104c5000455800005420000041440000442000005a
:104c600037200000202000000044000045560000ce
:104c700049430000452000005445000058540000fe
:104c800020410000444400002038000020200000a3
:104c90002000000044450000564900004345000044
:104ca00020540000455800005420000041440000fa
:104cb00044200000392000002020000000440000b3
:104cc00045560000494300004520000054450000bf
:104cd00058540000204100004444000020310000ee
:104ce000302000002000000044450000564900002c
:104cf00043450000205400004558000054200000a7
:104d00004144000044200000313100002020000018
:104d100000440000455600004943000045200000c3
:104d20005445000058540000204100004444000055
:104d30002031000032200000200000004445000027
:104d4000564900004345000020540000455800002b
:104d50005420000041440000442000003133000092
:104d60002020000000440000455600004943000098
:104d70004520000054450000585400002041000028
:104d800044440000203100003420000020000000d6
:104d900044450000564900004345000020540000ef
:104da0004558000054200000414400004420000009
:104db000313500002020000000440000455600006e
:104dc00049430000452000005445000058540000ad
:104dd0002041000044440000203100003620000043
:104de00020000000444500005649000043450000f3
:104df00020540000455800005420000041440000a9
:104e00004420000031370000202000000044000052
:104e1000455600004943000045200000544500006d
:104e2000585400002041000044440000203100009c
:104e300038200000200000004445000056490000d2
:104e40004345000020540000455800005420000055
:104e500041440000442000003139000020200000bf
:104e60000044000045560000494300004520000072
:104e70005445000058540000204100004444000004
:104e800020320000302000002000000044450000d7
:104e900056490000434500002054000045580000da
:104ea0005420000041440000442000003231000042
:104eb0002020000000440000455600004943000047
:104ec00045200000544500005854000020410000d7
:104ed0004444000020320000322000002000000086
:104ee000444500005649000043450000205400009e
:104ef00045580000542000004144000044200000b8
:104f0000323300002020000000440000455600001d
:104f1000494300004520000054450000585400005b
:104f200020410000444400002032000034200000f2
:104f300020000000444500005649000043450000a1
:104f40002054000045580000542000004144000057
:104f50004420000032350000202000000044000002
:104f6000455600004943000045200000544500001c
:104f7000585400002041000044440000203200004a
:104f80003620000020000000444500005649000083
:104f90004345000020540000455800005420000004
:104fa000414400004420000032370000202000006f
:104fb0000044000045560000494300004520000021
:104fc00054450000585400002041000044440000b3
:104fd000203200003820000020000000444500007e
:104fe0005649000043450000205400004558000089
:104ff00054200000414400004420000032390000e9
:1050000020200000004400004556000049430000f5
:105010004520000054450000585400002041000085
:105020004444000020330000302000002000000035
:10503000444500005649000043450000205400004c
:105040004558000054200000414400004420000066
:1050500033310000202000000044000045560000cd
:10506000494300004520000054450000585400000a
:1050700020410000444400002033000032200000a2
:105080002000000044450000564900004345000050
:105090002054000045580000542000004144000006
:1050a00044200000333300002020000000440000b2
:1050b00045560000494300004520000054450000cb
:1050c00058540000204100004444000020330000f8
:1050d0003420000020000000444500005649000034
:1050e00043450000205400004558000054200000b3
:1050f000414400004420000033350000202000001f
:1051000000440000455600004943000045200000cf
:105110005445000058540000204100004444000061
:10512000203300003620000020000000444500002d
:105130005649000043450000205400004558000037
:105140005420000041440000442000003337000098
:1051500020200000004400004556000049430000a4
:105160004520000054450000585400002041000034
:1051700044440000203300003820000020000000dc
:1051800044450000564900004345000020540000fb
:105190004558000054200000414400004420000015
:1051a0003339000020200000004400004556000074
:1051b00049430000452000005445000058540000b9
:1051c0002041000044440000203400003020000052
:1051d00020000000444500005649000043450000ff
:1051e00020540000455800005420000041440000b5
:1051f0004420000034310000202000000044000062
:105200004556000049430000452000005445000079
:1052100058540000204100004444000020340000a5
:1052200032200000200000004445000056490000e4
:105230004345000020540000455800005420000061
:1052400041440000442000003433000020200000ce
:10525000004400004556000049430000452000007e
:105260005445000058540000204100004444000010
:1052700020340000342000002000000044450000dd
:1052800056490000434500002054000045580000e6
:105290005420000041440000442000003435000048
:1052a0002020000000440000455600004943000053
:1052b00045200000544500005854000020410000e3
:1052c000444400002034000036200000200000008c
:1052d00044450000564900004345000020540000aa
:1052e00045580000542000004144000044200000c4
:1052f0003437000020200000004400004556000024
:105300004943000045200000544500005854000067
:1053100020410000444400002034000038200000f8
:1053200020000000444500005649000043450000ad
:105330002054000045580000542000004144000063
:105340004420000034390000202000000044000008
:105350004556000049430000452000005445000028
:105360005854000020410000444400002035000053
:105370003020000020000000444500005649000095
:105380004345000020540000455800005420000010
:10539000414400004420000035310000202000007e
:1053a000004400004556000049430000452000002d
:1053b00054450000585400002041000044440000bf
:1053c000203500003220000020000000444500008d
:1053d0005649000043450000205400004558000095
:1053e00054200000414400004420000035330000f8
:1053f0002020000000440000455600004943000002
:105400004520000054450000585400002041000091
:10541000444400002035000034200000200000003b
:105420004445000056490000434500002054000058
:105430004558000054200000414400004420000072
:1054400035350000202000000044000045560000d3
:105450004943000045200000544500005854000016
:1054600020410000444400002035000036200000a8
:10547000200000004445000056490000434500005c
:105480002054000045580000542000004144000012
:1054900044200000353700002020000000440000b8
:1054a00045560000494300004520000054450000d7
:1054b0005854000020410000444400002035000002
:1054c000382000002000000044450000564900003c
:1054d00043450000205400004558000054200000bf
:1054e0004144000044200000353900002020000025
:1054f00000440000455600004943000045200000dc
:10550000544500005854000020410000444400006d
:10551000203600003020000020000000444500003c
:105520005649000043450000205400004558000043
:1055300054200000414400004420000036310000a7
:1055400020200000004400004556000049430000b0
:105550004520000054450000585400002041000040
:1055600044440000203600003220000020000000eb
:105570004445000056490000434500002054000007
:105580004558000054200000414400004420000021
:105590003633000020200000004400004556000083
:1055a00049430000452000005445000058540000c5
:1055b0002041000044440000203600003420000058
:1055c000200000004445000056490000434500000b
:1055d00020540000455800005420000041440000c1
:1055e0004420000036350000202000000044000068
:1055f0004556000049430000452000005445000086
:1056000058540000204100004444000020360000af
:1056100036200000200000004445000056490000ec
:10562000434500002054000045580000542000006d
:1056300041440000442000003637000020200000d4
:10564000004400004556000049430000452000008a
:10565000544500005854000020410000444400001c
:1056600020360000382000002000000044450000e3
:1056700056490000434500002054000045580000f2
:10568000542000004144000044200000363900004e
:10569000202000000044000045560000494300005f
:1056a00045200000544500005854000020410000ef
:1056b000444400002037000030200000200000009b
:1056c00044450000564900004345000020540000b6
:1056d00045580000542000004144000044200000d0
:1056e0003731000020200000004400004556000033
:1056f0004943000045200000544500005854000074
:105700002041000044440000203700003220000007
:1057100020000000444500005649000043450000b9
:10572000205400004558000054200000414400006f
:105730004420000037330000202000000044000017
:105740004556000049430000452000005445000034
:10575000585400002041000044440000203700005d
:10576000342000002000000044450000564900009d
:10577000434500002054000045580000542000001c
:105780004144000044200000373500002020000084
:105790000044000045560000494300004520000039
:1057a00054450000585400002041000044440000cb
:1057b0002037000036200000200000004445000093
:1057c00056490000434500002054000045580000a1
:1057d00054200000414400004420000037370000fe
:1057e000202000000044000045560000494300000e
:1057f000452000005445000058540000204100009e
:105800004444000020370000382000002000000041
:105810004445000056490000434500002054000064
:10582000455800005420000041440000442000007e
:1058300037390000202000000044000045560000d9
:105840004943000045200000544500005854000022
:1058500020410000444400002038000030200000b7
:105860002000000044450000564900004345000068
:10587000205400004558000054200000414400001e
:1058800044200000383100002020000000440000c7
:1058900045560000494300004520000054450000e3
:1058a000585400002041000044440000203800000b
:1058b000322000002000000044450000564900004e
:1058c00043450000205400004558000054200000cb
:1058d0004144000044200000383300002020000034
:1058e00000440000455600004943000045200000e8
:1058f000544500005854000020410000444400007a
:105900002038000034200000200000004445000042
:10591000564900004345000020540000455800004f
:1059200054200000414400004420000038350000ad
:1059300020200000004400004556000049430000bc
:10594000452000005445000058540000204100004c
:1059500044440000203800003620000020000000f1
:105960004445000056490000434500002054000013
:10597000455800005420000041440000442000002d
:105980003837000020200000004400004556000089
:1059900049430000452000005445000058540000d1
:1059a000204100004444000020380000382000005e
:1059b0002000000044450000564900004345000017
:1059c00020540000455800005420000041440000cd
:1059d000442000003839000020200000004400006e
:1059e0004556000049430000452000005445000092
:1059f00058540000204100004444000020390000b9
:105a000030200000200000004445000056490000fe
:105a10004345000020540000455800005420000079
:105a200041440000442000003931000020200000e3
:105a30000044000045560000494300004520000096
:105a40005445000058540000204100004444000028
:105a500020390000322000002000000044450000f2
:105a600056490000434500002054000045580000fe
:105a7000542000004144000044200000393300005d
:105a8000202000000044000045560000494300006b
:105a900045200000544500005854000020410000fb
:105aa00044440000203900003420000020000000a1
:105ab00044450000564900004345000020540000c2
:105ac00045580000542000004144000044200000dc
:105ad0003935000020200000004400004556000039
:105ae0004943000045200000544500005854000080
:105af000204100004444000020390000362000000e
:105b000020000000444500005649000043450000c5
:105b1000205400004558000054200000414400007b
:105b2000442000003937000020200000004400001d
:105b30004556000049430000452000005445000040
:105b40005854000020410000444400002039000067
:105b500038200000200000004445000056490000a5
:105b60004345000020540000455800005420000028
:105b7000414400004420000039390000202000008a
:105b80000044000045560000494300004520000045
:105b900054450000585400002041000044440000d7
:105ba000203100003030000020000000444500009b
:105bb00056490000434500002054000045580000ad
:105bc0005420000041440000442000003130000017
:105bd0003120000000440000455600004943000009
:105be00045200000544500005854000020410000aa
:105bf000444400002031000030320000200000004a
:105c00004445000056490000434500002054000070
:105c1000455800005420000041440000442000008a
:105c200031300000332000000044000045560000e1
:105c3000494300004520000054450000585400002e
:105c400020410000444400002031000030340000b6
:105c50002000000044450000564900004345000074
:105c6000205400004558000054200000414400002a
:105c700044200000313000003520000000440000c6
:105c800045560000494300004520000054450000ef
:105c9000585400002041000044440000203100001e
:105ca0003036000020000000444500005649000046
:105cb00043450000205400004558000054200000d7
:105cc0004144000044200000313000003720000033
:105cd00000440000455600004943000045200000f4
:105ce0005445000058540000204100004444000086
:105cf0002031000030380000200000004445000042
:105d0000564900004345000020540000455800005b
:105d100054200000414400004420000031300000c5
:105d200039200000004400004556000049430000af
:105d30004520000054450000585400002041000058
:105d400044440000203100003130000020000000f9
:105d5000444500005649000043450000205400001f
:105d60004558000054200000414400004420000039
:105d70003131000031200000004400004556000091
:105d800049430000452000005445000058540000dd
:105d90002041000044440000203100003132000066
:105da0002000000044450000564900004345000023
:105db00020540000455800005420000041440000d9
:105dc0004420000031310000332000000044000076
:105dd000455600004943000045200000544500009e
:105de00058540000204100004444000020310000cd
:105df00031340000200000004445000056490000f6
:105e00004345000020540000455800005420000085
:105e100041440000442000003131000035200000e2
:105e200000440000455600004943000045200000a2
:105e30005445000058540000204100004444000034
:105e400020310000313600002000000044450000f1
:105e5000564900004345000020540000455800000a
:105e60005420000041440000442000003131000073
:105e70003720000000440000455600004943000060
:105e80004520000054450000585400002041000007
:105e900044440000203100003138000020000000a0
:105ea00044450000564900004345000020540000ce
:105eb00045580000542000004144000044200000e8
:105ec0003131000039200000004400004556000038
:105ed000494300004520000054450000585400008c
:105ee0002041000044440000203100003230000016
:105ef00020000000444500005649000043450000d2
:105f00002054000045580000542000004144000087
:105f10004420000031320000312000000044000025
:105f2000455600004943000045200000544500004c
:105f3000585400002041000044440000203100007b
:105f400032320000200000004445000056490000a5
:105f50004345000020540000455800005420000034
:105f60004144000044200000313200003320000092
:105f70000044000045560000494300004520000051
:105f800054450000585400002041000044440000e3
:105f900020310000323400002000000044450000a1
:105fa00056490000434500002054000045580000b9
:105fb0005420000041440000442000003132000021
:105fc0003520000000440000455600004943000011
:105fd00045200000544500005854000020410000b6
:105fe0004444000020310000323600002000000050
:105ff000444500005649000043450000205400007d
:106000004558000054200000414400004420000096
:1060100031320000372000000044000045560000e7
:10602000494300004520000054450000585400003a
:1060300020410000444400002031000032380000bc
:106040002000000044450000564900004345000080
:106050002054000045580000542000004144000036
:1060600044200000313200003920000000440000cc
:1060700045560000494300004520000054450000fb
:10608000585400002041000044440000203100002a
:106090003330000020000000444500005649000055
:1060a00043450000205400004558000054200000e3
:1060b0004144000044200000313300003120000042
:1060c0000044000045560000494300004520000000
:1060d0005445000058540000204100004444000092
:1060e0002031000033320000200000004445000051
:1060f0005649000043450000205400004558000068
:1061000054200000414400004420000031330000ce
:1061100033200000004400004556000049430000c1
:106120004520000054450000585400002041000064
:1061300044440000203100003334000020000000ff
:10614000444500005649000043450000205400002b
:106150004558000054200000414400004420000045
:106160003133000035200000004400004556000097
:1061700049430000452000005445000058540000e9
:10618000204100004444000020310000333600006c
:10619000200000004445000056490000434500002f
:1061a00020540000455800005420000041440000e5
:1061b000442000003133000037200000004400007c
:1061c00045560000494300004520000054450000aa
:1061d00058540000204100004444000020310000d9
:1061e00033380000200000004445000056490000fc
:1061f0004345000020540000455800005420000092
:1062000041440000442000003133000039200000e8
:1062100000440000455600004943000045200000ae
:106220005445000058540000204100004444000040
:106230002031000034300000200000004445000000
:106240005649000043450000205400004558000016
:10625000542000004144000044200000313400007c
:106260003120000000440000455600004943000072
:106270004520000054450000585400002041000013
:1062800044440000203100003432000020000000af
:1062900044450000564900004345000020540000da
:1062a00045580000542000004144000044200000f4
:1062b0003134000033200000004400004556000047
:1062c0004943000045200000544500005854000098
:1062d000204100004444000020310000343400001c
:1062e00020000000444500005649000043450000de
:1062f0002054000045580000542000004144000094
:10630000442000003134000035200000004400002b
:106310004556000049430000452000005445000058
:106320005854000020410000444400002031000087
:1063300034360000200000004445000056490000ab
:106340004345000020540000455800005420000040
:106350004144000044200000313400003720000098
:10636000004400004556000049430000452000005d
:1063700054450000585400002041000044440000ef
:1063800020310000343800002000000044450000a7
:1063900056490000434500002054000045580000c5
:1063a000542000004144000044200000313400002b
:1063b0003920000000440000455600004943000019
:1063c00045200000544500005854000020410000c2
:1063d000444400002031000035300000200000005f
:1063e0004445000056490000434500002054000089
:1063f00045580000542000004144000044200000a3
:1064000031350000312000000044000045560000f6
:106410004943000045200000544500005854000046
:1064200020410000444400002031000035320000cb
:10643000200000004445000056490000434500008c
:106440002054000045580000542000004144000042
:1064500044200000313500003320000000440000db
:106460004556000049430000452000005445000007
:106470005854000020410000444400002031000036
:10648000353400002000000044450000564900005b
:1064900043450000205400004558000054200000ef
:1064a0004144000044200000313500003520000048
:1064b000004400004556000049430000452000000c
:1064c000544500005854000020410000444400009e
:1064d0002031000035360000200000004445000057
:1064e0005649000043450000205400004558000074
:1064f00054200000414400004420000031350000d9
:1065000037200000004400004556000049430000c9
:106510004520000054450000585400002041000070
:106520004444000020310000353800002000000005
:106530004445000056490000434500002054000037
:106540004558000054200000414400004420000051
:10655000313500003920000000440000455600009d
:1065600049430000452000005445000058540000f5
:10657000204100004444000020310000363000007b
:10658000200000004445000056490000434500003b
:1065900020540000455800005420000041440000f1
:1065a000442000003136000031200000004400008b
:1065b00045560000494300004520000054450000b6
:1065c00058540000204100004444000020310000e5
:1065d000363200002000000044450000564900000b
:1065e000434500002054000045580000542000009e
:1065f00041440000442000003136000033200000f8
:1066000000440000455600004943000045200000ba
:10661000544500005854000020410000444400004c
:106620002031000036340000200000004445000006
:106630005649000043450000205400004558000022
:106640005420000041440000442000003136000086
:10665000352000000044000045560000494300007a
:10666000452000005445000058540000204100001f
:1066700044440000203100003636000020000000b5
:1066800044450000564900004345000020540000e6
:106690004558000054200000414400004420000000
:1066a000313600003720000000440000455600004d
:1066b00049430000452000005445000058540000a4
:1066c0002041000044440000203100003638000022
:1066d00020000000444500005649000043450000ea
:1066e00020540000455800005420000041440000a0
:1066f0004420000031360000392000000044000032
:106700004556000049430000452000005445000064
:106710005854000020410000444400002031000093
:1067200037300000200000004445000056490000ba
:10673000434500002054000045580000542000004c
:1067400041440000442000003137000031200000a7
:106750000044000045560000494300004520000069
:1067600054450000585400002041000044440000fb
:1067700020310000373200002000000044450000b6
:1067800056490000434500002054000045580000d1
:106790005420000041440000442000003137000034
:1067a000332000000044000045560000494300002b
:1067b00045200000544500005854000020410000ce
:1067c0004444000020310000373400002000000065
:1067d0004445000056490000434500002054000095
:1067e00045580000542000004144000044200000af
:1067f00031370000352000000044000045560000fd
:106800004943000045200000544500005854000052
:1068100020410000444400002031000037360000d1
:106820002000000044450000564900004345000098
:10683000205400004558000054200000414400004e
:1068400044200000313700003720000000440000e1
:106850004556000049430000452000005445000013
:106860005854000020410000444400002031000042
:106870003738000020000000444500005649000061
:1068800043450000205400004558000054200000fb
:10689000414400004420000031370000392000004e
:1068a0000044000045560000494300004520000018
:1068b00054450000585400002041000044440000aa
:1068c0002031000038300000200000004445000066
:1068d0005649000043450000205400004558000080
:1068e00054200000414400004420000031380000e2
:1068f00031200000004400004556000049430000dc
:10690000452000005445000058540000204100007c
:106910004444000020310000383200002000000014
:106920004445000056490000434500002054000043
:10693000455800005420000041440000442000005d
:1069400031380000332000000044000045560000ac
:106950004943000045200000544500005854000001
:106960002041000044440000203100003834000081
:106970002000000044450000564900004345000047
:1069800020540000455800005420000041440000fd
:106990004420000031380000352000000044000091
:1069a00045560000494300004520000054450000c2
:1069b00058540000204100004444000020310000f1
:1069c0003836000020000000444500005649000011
:1069d00043450000205400004558000054200000aa
:1069e00041440000442000003138000037200000fe
:1069f00000440000455600004943000045200000c7
:106a00005445000058540000204100004444000058
:106a1000203100003838000020000000444500000c
:106a2000564900004345000020540000455800002e
:106a30005420000041440000442000003138000090
:106a40003920000000440000455600004943000082
:106a5000452000005445000058540000204100002b
:106a600044440000203100003930000020000000c4
:106a700044450000564900004345000020540000f2
:106a8000455800005420000041440000442000000c
:106a9000313900003120000000440000455600005c
:106aa00049430000452000005445000058540000b0
:106ab0002041000044440000203100003932000031
:106ac00020000000544500005854000020460000fb
:106ad0004f520000205a00004f4e00004520000099
:106ae0003120000020200000202000000054000081
:106af0004558000054200000464f0000522000007e
:106b00005a4f00004e4500002032000020200000b7
:106b100020200000200000005445000058540000d0
:106b2000204600004f520000205a00004f4e000047
:106b3000452000003320000020200000202000001d
:106b4000005400004558000054200000464f00004b
:106b5000522000005a4f00004e4500002034000033
:106b600020200000202000002000000054450000ec
:106b700058540000204600004f520000205a0000e8
:106b80004f4e00004520000035200000202000006e
:106b90002020000000540000455800005420000050
:106ba000464f0000522000005a4f00004e450000a2
:106bb00020360000202000002020000020000000df
:106bc0005445000058540000204600004f52000079
:106bd000205a00004f4e00004520000037200000e2
:106be0002020000020200000005400004558000034
:106bf00054200000464f0000522000005a4f000071
:106c00004e45000020380000202000002020000019
:106c100020000000544500005854000020460000a9
:106c20004f520000205a00004f4e00004520000047
:106c30003920000020200000202000000054000027
:106c40004558000054200000464f0000522000002c
:106c50005a4f00004e450000203100003020000057
:106c6000202000002000000054450000585400007f
:106c7000204600004f520000205a00004f4e0000f6
:106c800045200000313100002020000020200000bd
:106c9000005400004558000054200000464f0000fa
:106ca000522000005a4f00004e45000020310000e5
:106cb0003220000020200000200000005445000089
:106cc00058540000204600004f520000205a000097
:106cd0004f4e00004520000031330000202000000e
:106ce00020200000005400004558000054200000ff
:106cf000464f0000522000005a4f00004e45000051
:106d0000203100003420000020200000200000007e
:106d10005445000058540000204600004f52000027
:106d2000205a00004f4e0000452000003135000081
:106d300020200000202000000054000045580000e2
:106d400054200000464f0000522000005a4f00001f
:106d50004e450000203100003620000020200000b9
:106d60002000000054450000585400002046000058
:106d70004f520000205a00004f4e000045200000f6
:106d800031370000202000002020000000540000c7
:106d90004558000054200000464f000052200000db
:106da0005a4f00004e4500002031000038200000fe
:106db000202000002000000054450000585400002e
:106dc000204600004f520000205a00004f4e0000a5
:106dd0004520000031390000202000002020000064
:106de000005400004558000054200000464f0000a9
:106df000522000005a4f00004e4500002032000093
:106e00003020000020200000200000005445000039
:106e100058540000204600004f520000205a000045
:106e20004f4e0000452000003231000020200000bd
:106e300020200000005400004558000054200000ad
:106e4000464f0000522000005a4f00004e450000ff
:106e5000203200003220000020200000200000002e
:106e60005445000058540000204600004f520000d6
:106e7000205a00004f4e0000452000003233000031
:106e80002020000020200000005400004558000091
:106e900054200000464f0000522000005a4f0000ce
:106ea0004e45000020320000342000002020000069
:106eb0002000000054450000585400002046000007
:106ec0004f520000205a00004f4e000045200000a5
:106ed0003235000020200000202000000054000077
:106ee0004558000054200000464f0000522000008a
:106ef0005a4f00004e4500002032000036200000ae
:106f000020200000200000005445000058540000dc
:106f1000204600004f520000205a00004f4e000053
:106f20004520000032370000202000002020000013
:106f3000005400004558000054200000464f000057
:106f4000522000005a4f00004e4500002032000041
:106f500038200000202000002000000054450000e0
:106f600058540000204600004f520000205a0000f4
:106f70004f4e000045200000323900002020000064
:106f8000202000000054000045580000542000005c
:106f9000464f0000522000005a4f00004e450000ae
:106fa00020330000302000002020000020000000de
:106fb0005445000058540000204600004f52000085
:106fc000205a00004f4e00004520000033310000e1
:106fd0002020000020200000005400004558000040
:106fe00054200000464f0000522000005a4f00007d
:106ff0004e45000020330000322000002020000019
:107000002000000000000000000000000000000060
:10701000000000000000000000000000010100006e
:10702000020300000401000004010000020300004c
:10703000040100000401000002030000040100003c
:1070400002010000020300000401000003ff000031
:10705000ffff0000ffff0000ffff0000ffff000038
:10706000ffff0000ffff0000ffff0000ffff000028
:10707000ffff0000ffff0000ffff0000ffff000018
:10708000ffff0000ffff0000ffff0000ffff000008
:10709000ffff0000ffff0000ffff0000ffff0000f8
:1070a000ffff0000ffff0000ffff0000ff140000d3
:1070b0000c0000000c0000000202000000000000b4
:1070c00018000000000000000200000000000000a6
:1070d000010000000120000000000000000000008e
:1070e00000000000000000000000000000000000a0
:1070f0000000000000000000000000000000000090
:10710000000000000000000000000000000000007f
:10711000000000000000000000000000000000006f
:020000040000fa
:1030000000000000000000000000000001010000be
:1030100001110000f00100000000000000000000ad
:10302000000000000000000000000000010100009e
:1030300001110000f001000000000000000000008d
:10304000000000000000000000000000010100007e
:1030500001110000f001000000000000000000006d
:10306000000000000000000000000000010100005e
:1030700001110000f001000000000000000000004d
:10308000000000000000000000000000010100003e
:1030900001110000f001000000000000000000002d
:1030a000000000000000000000000000010100001e
:1030b00001110000f001000000000000000000000d
:1030c00000000000000000000000000001010000fe
:1030d00001110000f00100000000000000000000ed
:1030e00000000000000000000000000001010000de
:1030f00001110000f00100000000000000000000cd
:1031000000000000000000000000000001010000bd
:1031100001110000f00100000000000000000000ac
:10312000000000000000000000000000010100009d
:1031300001110000f001000000000000000000008c
:10314000000000000000000000000000010100007d
:1031500001110000f001000000000000000000006c
:10316000000000000000000000000000010100005d
:1031700001110000f001000000000000000000004c
:10318000000000000000000000000000010100003d
:1031900001110000f001000000000000000000002c
:1031a000000000000000000000000000010100001d
:1031b00001110000f001000000000000000000000c
:1031c00000000000000000000000000001010000fd
:1031d00001110000f00100000000000000000000ec
:1031e00000000000000000000000000001010000dd
:1031f00001110000f00100000000000000000000cc
:1032000000000000000000000000000001010000bc
:1032100001110000f00100000000000000000000ab
:10322000000000000000000000000000010100009c
:1032300001110000f001000000000000000000008b
:10324000000000000000000000000000010100007c
:1032500001110000f001000000000000000000006b
:10326000000000000000000000000000010100005c
:1032700001110000f001000000000000000000004b
:10328000000000000000000000000000010100003c
:1032900001110000f001000000000000000000002b
:1032a000000000000000000000000000010100001c
:1032b00001110000f001000000000000000000000b
:1032c00000000000000000000000000001010000fc
:1032d00001110000f00100000000000000000000eb
:1032e00000000000000000000000000001010000dc
:1032f00001110000f00100000000000000000000cb
:1033000000000000000000000000000001010000bb
:1033100001110000f00100000000000000000000aa
:10332000000000000000000000000000010100009b
:1033300001110000f001000000000000000000008a
:10334000000000000000000000000000010100007b
:1033500001110000f001000000000000000000006a
:10336000000000000000000000000000010100005b
:1033700001110000f001000000000000000000004a
:10338000000000000000000000000000010100003b
:1033900001110000f001000000000000000000002a
:1033a000000000000000000000000000010100001b
:1033b00001110000f001000000000000000000000a
:1033c00000000000000000000000000001010000fb
:1033d00001110000f00100000000000000000000ea
:1033e00000000000000000000000000001010000db
:1033f00001110000f00100000000000000000000ca
:1034000000000000000000000000000001010000ba
:1034100001110000f00100000000000000000000a9
:10342000000000000000000000000000010100009a
:1034300001110000f0010000000000000000000089
:10344000000000000000000000000000010100007a
:1034500001110000f0010000000000000000000069
:10346000000000000000000000000000010100005a
:1034700001110000f0010000000000000000000049
:10348000000000000000000000000000010100003a
:1034900001110000f0010000000000000000000029
:1034a000000000000000000000000000010100001a
:1034b00001110000f0010000000000000000000009
:1034c00000000000000000000000000001010000fa
:1034d00001110000f00100000000000000000000e9
:1034e00000000000000000000000000001010000da
:1034f00001110000f00100000000000000000000c9
:1035000000000000000000000000000001010000b9
:1035100001110000f00100000000000000000000a8
:103520000000000000000000000000000101000099
:1035300001110000f0010000000000000000000088
:103540000000000000000000000000000101000079
:1035500001110000f0010000000000000000000068
:103560000000000000000000000000000101000059
:1035700001110000f0010000000000000000000048
:103580000000000000000000000000000101000039
:1035900001110000f0010000000000000000000028
:1035a0000000000000000000000000000101000019
:1035b00001110000f0010000000000000000000008
:1035c00000000000000000000000000001010000f9
:1035d00001110000f00100000000000000000000e8
:1035e00000000000000000000000000001010000d9
:1035f00001110000f00100000000000000000000c8
:1036000000000000000000000000000001010000b8
:1036100001110000f00100000000000000000000a7
:103620000000000000000000000000000101000098
:1036300001110000f0010000000000000000000087
:103640000000000000000000000000000101000078
:1036500001110000f0010000000000000000000067
:103660000000000000000000000000000101000058
:1036700001110000f0010000000000000000000047
:103680000000000000000000000000000101000038
:1036900001110000f0010000000000000000000027
:1036a0000000000000000000000000000101000018
:1036b00001110000f0010000000000000000000007
:1036c00000000000000000000000000001010000f8
:1036d00001110000f00100000000000000000000e7
:1036e00000000000000000000000000001010000d8
:1036f00001110000f00100000000000000000000c7
:1037000000000000000000000000000001010000b7
:1037100001110000f00100000000000000000000a6
:103720000000000000000000000000000101000097
:1037300001110000f0010000000000000000000086
:103740000000000000000000000000000101000077
:1037500001110000f0010000000000000000000066
:103760000000000000000000000000000101000057
:1037700001110000f0010000000000000000000046
:103780000000000000000000000000000101000037
:1037900001110000f0010000000000000000000026
:1037a0000000000000000000000000000101000017
:1037b00001110000f0010000000000000000000006
:1037c00000000000000000000000000001010000f7
:1037d00001110000f00100000000000000000000e6
:1037e00000000000000000000000000001010000d7
:1037f00001110000f00100000000000000000000c6
:1038000000000000000000000000000001010000b6
:1038100001110000f00100000000000000000000a5
:103820000000000000000000000000000101000096
:1038300001110000f0010000000000000000000085
:103840000000000000000000000000000101000076
:1038500001110000f0010000000000000000000065
:103860000000000000000000000000000101000056
:1038700001110000f0010000000000000000000045
:103880000000000000000000000000000101000036
:1038900001110000f0010000000000000000000025
:1038a0000000000000000000000000000101000016
:1038b00001110000f0010000000000000000000005
:1038c00000000000000000000000000001010000f6
:1038d00001110000f00100000000000000000000e5
:1038e00000000000000000000000000001010000d6
:1038f00001110000f00100000000000000000000c5
:1039000000000000000000000000000001010000b5
:1039100001110000f00100000000000000000000a4
:103920000000000000000000000000000101000095
:1039300001110000f0010000000000000000000084
:103940000000000000000000000000000101000075
:1039500001110000f0010000000000000000000064
:103960000000000000000000000000000101000055
:1039700001110000f0010000000000000000000044
:103980000000000000000000000000000101000035
:1039900001110000f0010000000000000000000024
:1039a0000000000000000000000000000101000015
:1039b00001110000f0010000000000000000000004
:1039c00000000000000000000000000001010000f5
:1039d00001110000f00100000000000000000000e4
:1039e00000000000000000000000000001010000d5
:1039f00001110000f00100000000000000000000c4
:103a000000000000000000000000000001010000b4
:103a100001110000f00100000000000000000000a3
:103a20000000000000000000000000000101000094
:103a300001110000f0010000000000000000000083
:103a40000000000000000000000000000101000074
:103a500001110000f0010000000000000000000063
:103a60000000000000000000000000000101000054
:103a700001110000f0010000000000000000000043
:103a80000000000000000000000000000101000034
:103a900001110000f0010000000000000000000023
:103aa0000000000000000000000000000101000014
:103ab00001110000f0010000000000000000000003
:103ac00000000000000000000000000001010000f4
:103ad00001110000f00100000000000000000000e3
:103ae00000000000000000000000000001010000d4
:103af00001110000f00100000000000000000000c3
:103b000000000000000000000000000001010000b3
:103b100001110000f00100000000000000000000a2
:103b20000000000000000000000000000101000093
:103b300001110000f0010000000000000000000082
:103b40000000000000000000000000000101000073
:103b500001110000f0010000000000000000000062
:103b60000000000000000000000000000101000053
:103b700001110000f0010000000000000000000042
:103b80000000000000000000000000000101000033
:103b900001110000f0010000000000000000000022
:103ba0000000000000000000000000000101000013
:103bb00001110000f0010000000000000000000002
:103bc00000000000000000000000000001010000f3
:103bd00001110000f00100000000000000000000e2
:103be00000000000000000000000000001010000d3
:103bf00001110000f00100000000000000000000c2
:103c000000000000000000000000000001010000b2
:103c100001110000f00100000000000000000000a1
:103c20000000000000000000000000000101000092
:103c300001110000f0010000000000000000000081
:103c40000000000000000000000000000101000072
:103c500001110000f0010000000000000000000061
:103c60000000000000000000000000000101000052
:103c700001110000f0010000000000000000000041
:103c80000000000000000000000000000101000032
:103c900001110000f0010000000000000000000021
:103ca0000000000000000000000000000101000012
:103cb00001110000f0010000000000000000000001
:103cc00000000000000000000000000001010000f2
:103cd00001110000f00100000000000000000000e1
:103ce00000000000000000000000000001010000d2
:103cf00001110000f00100000000000000000000c1
:103d000000000000000000000000000001010000b1
:103d100001110000f00100000000000000000000a0
:103d20000000000000000000000000000101000091
:103d300001110000f0010000000000000000000080
:103d40000000000000000000000000000101000071
:103d500001110000f0010000000000000000000060
:103d60000000000000000000000000000101000051
:103d700001110000f0010000000000000000000040
:103d80000000000000000000000000000101000031
:103d900001110000f0010000000000000000000020
:103da0000000000000000000000000000101000011
:103db00001110000f0010000000000000000000000
:103dc00000000000000000000000000001010000f1
:103dd00001110000f00100000000000000000000e0
:103de00000000000000000000000000001010000d1
:103df00001110000f00100000000000000000000c0
:103e000000000000000000000000000001010000b0
:103e100001110000f001000000000000000000009f
:103e20000000000000000000000000000101000090
:103e300001110000f001000000000000000000007f
:103e40000000000000000000000000000101000070
:103e500001110000f001000000000000000000005f
:103e60000000000000000000000000000101000050
:103e700001110000f001000000000000000000003f
:103e80000000000000000000000000000101000030
:103e900001110000f001000000000000000000001f
:103ea0000000000000000000000000000101000010
:103eb00001110000f00100000000000000000000ff
:103ec00000000000000000000000000001010000f0
:103ed00001110000f00100000000000000000000df
:103ee00000000000000000000000000001010000d0
:103ef00001110000f00100000000000000000000bf
:103f000000000000000000000000000001010000af
:103f100001110000f001000000000000000000009e
:103f2000000000000000000000000000010100008f
:103f300001110000f001000000000000000000007e
:103f4000000000000000000000000000010100006f
:103f500001110000f001000000000000000000005e
:103f6000000000000000000000000000010100004f
:103f700001110000f001000000000000000000003e
:103f8000000000000000000000000000010100002f
:103f900001110000f001000000000000000000001e
:103fa000000000000000000000000000010100000f
:103fb00001110000f00100000000000000000000fe
:103fc00000000000000000000000000001010000ef
:103fd00001110000f00100000000000000000000de
:103fe00000000000000000000000000001010000cf
:103ff00001110000f00100000000000000000000be
:1040000000000000000000000000000001010000ae
:1040100001110000f001000000000000000000009d
:10402000000000000000000000000000010100008e
:1040300001110000f001000000000000000000007d
:10404000000000000000000000000000010100006e
:1040500001110000f001000000000000000000005d
:10406000000000000000000000000000010100004e
:1040700001110000f001000000000000000000003d
:10408000000000000000000000000000010100002e
:1040900001110000f001000000000000000000001d
:1040a000000000000000000000000000010100000e
:1040b00001110000f00100000000000000000000fd
:1040c00000000000000000000000000001010000ee
:1040d00001110000f00100000000000000000000dd
:1040e00000000000000000000000000001010000ce
:1040f00001110000f00100000000000000000000bd
:1041000000000000000000000000000001010000ad
:1041100001110000f001000000000000000000009c
:10412000000000000000000000000000010100008d
:1041300001110000f001000000000000000000007c
:10414000000000000000000000000000010100006d
:1041500001110000f001000000000000000000005c
:10416000000000000000000000000000010100004d
:1041700001110000f001000000000000000000003c
:10418000000000000000000000000000010100002d
:1041900001110000f001000000000000000000001c
:1041a000000000000000000000000000010100000d
:1041b00001110000f00100000000000000000000fc
:1041c00000000000000000000000000001010000ed
:1041d00001110000f00100000000000000000000dc
:1041e00000000000000000000000000001010000cd
:1041f00001110000f00100000000000000000000bc
:1042000000000000000000000000000001010000ac
:1042100001110000f001000000000000000000009b
:10422000000000000000000000000000010100008c
:1042300001110000f001000000000000000000007b
:10424000000000000000000000000000010100006c
:1042500001110000f001000000000000000000005b
:10426000000000000000000000000000010100004c
:1042700001110000f001000000000000000000003b
:10428000000000000000000000000000010100002c
:1042900001110000f001000000000000000000001b
:1042a000000000000000000000000000010100000c
:1042b00001110000f00100000000000000000000fb
:1042c00000000000000000000000000001010000ec
:1042d00001110000f00100000000000000000000db
:1042e00000000000000000000000000001010000cc
:1042f00001110000f00100000000000000000000bb
:1043000000000000000000000000000001010000ab
:1043100001110000f001000000000000000000009a
:10432000000000000000000000000000010100008b
:1043300001110000f001000000000000000000007a
:10434000000000000000000000000000010100006b
:1043500001110000f001000000000000000000005a
:10436000000000000000000000000000010100004b
:1043700001110000f001000000000000000000003a
:10438000000000000000000000000000010100002b
:1043900001110000f001000000000000000000001a
:1043a000000000000000000000000000010100000b
:1043b00001110000f00100000000000000000000fa
:1043c00000000000000000000000000001010000eb
:1043d00001110000f00100000000000000000000da
:1043e00000000000000000000000000001010000cb
:1043f00001110000f00100000000000000000000ba
:1044000000000000000000000000000001010000aa
:1044100001110000f0010000000000000000000099
:10442000000000000000000000000000010100008a
:1044300001110000f0010000000000000000000079
:10444000000000000000000000000000010100006a
:1044500001110000f0010000000000000000000059
:10446000000000000000000000000000010100004a
:1044700001110000f0010000000000000000000039
:10448000000000000000000000000000010100002a
:1044900001110000f0010000000000000000000019
:1044a000000000000000000000000000010100000a
:1044b00001110000f00100000000000000000000f9
:1044c00000000000000000000000000001010000ea
:1044d00001110000f00100000000000000000000d9
:1044e00000000000000000000000000001010000ca
:1044f00001110000f00100000000000000000000b9
:1045000000000000000000000000000001010000a9
:1045100001110000f0010000000000000000000098
:104520000000000000000000000000000101000089
:1045300001110000f0010000000000000000000078
:104540000000000000000000000000000101000069
:1045500001110000f0010000000000000000000058
:104560000000000000000000000000000101000049
:1045700001110000f0010000000000000000000038
:104580000000000000000000000000000101000029
:1045900001110000f0010000000000000000000018
:1045a0000000000000000000000000000101000009
:1045b00001110000f00100000000000000000000f8
:1045c00000000000000000000000000001010000e9
:1045d00001110000f00100000000000000000000d8
:1045e00000000000000000000000000001010000c9
:1045f00001110000f00100000000000000000000b8
:1046000000000000000000000000000001010000a8
:1046100001110000f0010000000000000000000097
:104620000000000000000000000000000101000088
:1046300001110000f0010000000000000000000077
:104640000000000000000000000000000101000068
:1046500001110000f0010000000000000000000057
:104660000000000000000000000000000101000048
:1046700001110000f0010000000000000000000037
:104680000000000000000000000000000101000028
:1046900001110000f0010000000000000000000017
:1046a0000000000000000000000000000101000008
:1046b00001110000f00100000000000000000000f7
:1046c00000000000000000000000000001010000e8
:1046d00001110000f00100000000000000000000d7
:1046e00000000000000000000000000001010000c8
:1046f00001110000f00100000000000000000000b7
:1047000000000000000000000000000001010000a7
:1047100001110000f0010000000000000000000096
:104720000000000000000000000000000101000087
:1047300001110000f0010000000000000000000076
:104740000000000000000000000000000101000067
:1047500001110000f0010000000000000000000056
:104760000000000000000000000000000101000047
:1047700001110000f0010000000000000000000036
:104780000000000000000000000000000101000027
:1047900001110000f0010000000000000000000016
:1047a0000000000000000000000000000101000007
:1047b00001110000f00100000000000000000000f6
:1047c00000000000000000000000000001010000e7
:1047d00001110000f00100000000000000000000d6
:1047e00000000000000000000000000001010000c7
:1047f00001110000f00100000000000000000000b6
:020000040000fa
:10a2340036310000303000002020000020200000d3
:04a2440020200000d6
:020000040000fa
:08a22400313200003741000057
:020000040000fa
:08a22c0030300000303000006a
:020000040000fa
:04a22000000000003a
:020000040000fa
:020000040001f9
:10000000205300004f5500004e44000020410000e6
:100010004c410000524d00005320000041430000bd
:100020005449000056450000002000002020000038
:1000300020500000414e0000454c0000204d0000c3
:1000400055540000454400002020000020200000fe
:10005000200000002020000020200000504100006f
:100060004e4500004c200000524500005345000062
:10007000542000002020000020200000002000006c
:1000800020200000504100004e4500004c200000a0
:10009000534900004c4500004e4300004544000019
:1000a000202000002000000020200000204400004c
:1000b0004556000049430000452000004e4f000017
:1000c000524d0000414c0000202000002020000084
:1000d0000020000020440000455600004943000075
:1000e00045200000494e0000204100004c41000026
:1000f000524d0000202000002000000020200000c1
:1001000020200000444500005649000043450000ff
:1001100020460000415500004c5400002020000003
:100120002020000000440000455600004943000024
:100130004520000046410000494c000045440000b5
:1001400020530000455400005550000020000000de
:1001500020200000444500005649000043450000af
:100160002050000052450000414c00004152000068
:100170004d20000020200000002000002020000072
:10018000205a00004f4e000045200000494e00005c
:10019000205400004553000054200000202000009f
:1001a00020000000202000005a4f00004e450000b3
:1001b0002044000049530000414200004c4500002b
:1001c0004d4500004e54000020200000002000009b
:1001d00020200000202000005a4f00004e45000063
:1001e00020460000415500004c5400002020000033
:1001f000202000002000000020200000202000001f
:10020000414c0000415200004d20000046410000da
:10021000554c000054200000202000002020000049
:1002200000200000204100004c410000524d000021
:10023000532000004449000053410000424c00009c
:100240004544000020200000200000002020000085
:100250004649000052450000204c0000494e000075
:100260004b20000046410000554c00005420000087
:1002700020200000002000004649000052450000f8
:10028000204c0000494e00004b2000004449000073
:1002900053410000424c0000454400002000000093
:1002a0002046000049520000452000004c49000053
:1002b0004e4b0000204f000050450000524100000e
:1002c00054450000442000000020000020200000d1
:1002d00042410000545400004552000059200000e3
:1002e00046410000554c0000542000002020000032
:1002f0002000000020200000202000004d410000d0
:10030000494e00005320000046410000494c0000c7
:1003100045440000202000002020000000200000b4
:100320002020000020520000455000004541000000
:100330005420000046410000554c000054200000ad
:100340002020000020000000202000004155000077
:100350005820000053550000505000004c59000038
:1003600020460000415500004c54000020200000b1
:100370000020000020200000204300004c4100002d
:100380005353000020430000484100004e47000046
:100390004520000020200000200000002020000058
:1003a00020200000524500004d4f00005445000041
:1003b000204100004c410000524d00002020000070
:1003c000202000000020000055530000455200008e
:1003d000204300004f44000045200000454e00002f
:1003e0005445000052450000442000002000000059
:1003f00020200000454e000047200000434f000031
:1004000044450000204500004e54000045520000c5
:100410004544000020200000004100004456000038
:10042000204500004e470000204300004f440000dc
:1004300045200000454e0000544500005245000094
:100440004400000020200000202000002043000085
:100450004c4f0000434b0000205300004554000067
:1004600020200000202000002020000000200000ac
:100470002020000020500000414e0000454c0000ac
:100480002052000045530000544100005254000027
:10049000202000002000000020200000202000007c
:1004a000204c00004f4f000050200000464100004b
:1004b000554c0000542000002020000020200000a7
:1004c0000020000020420000555a00005a4500005c
:1004d000522000004449000053410000424c0000fb
:1004e00045440000202000002000000020200000e3
:1004f0002020000050430000204300004f4e000029
:100500004e450000435400004544000020200000f8
:100510002020000000200000534900005445000046
:10052000204400004154000041200000434f0000df
:1005300052520000555000005420000020000000de
:10054000204c00004f4f00005020000044450000a8
:10055000564900004345000053200000414400007c
:10056000444500004420000000200000204c000012
:100570004f4f000050200000414c0000415200004d
:100580004d20000046410000554c00005420000062
:100590002000000020200000505200004f470000c3
:1005a000524100004d200000525500004e20000036
:1005b00045520000524f0000522000000020000071
:1005c00020200000204c00004f4f00005020000071
:1005d0004c4f000047470000454400002020000029
:1005e00020200000200000002020000053490000cf
:1005f0005445000020440000415400004120000008
:1006000043480000414e00004745000044200000e0
:100610000020000020200000205300004552000070
:1006200056490000434500002044000055450000a5
:1006300020200000202000002000000020200000da
:10064000204e00004947000048540000205300009d
:10065000454e0000532000004f4e000020200000b7
:10066000202000000020000045560000414300000b
:1006700020500000414e0000454c00002041000089
:1006800043540000495600004520000020000000af
:100690004d4100004e200000464900005245000038
:1006a000204c0000494e00004b2000004641000055
:1006b000554c000054200000002000004f50000066
:1006c00020470000524f0000555000002044000019
:1006d00049530000414200004c4500004420000006
:1006e00020000000434f00004e540000204f000047
:1006f00050470000525000005320000044490000c1
:1007000053410000424c000045440000002000001e
:1007100020200000534900005445000046490000d5
:100720004c45000020450000525200004f5200008e
:100730002020000020000000202000004445000090
:100740005649000043450000204400004953000082
:10075000414200004c4500004420000020200000e1
:100760000020000020200000464200005020000031
:10077000434f00004d4d0000532000004641000053
:10078000554c0000542000002000000020200000f4
:10079000414c0000415200004d5300002052000027
:1007a000455300004f5500004e44000045440000f2
:1007b000202000000044000045560000494300008e
:1007c00045200000494e00005649000053490000f2
:1007d000424c00004520000053570000200000005c
:1007e0004f500000475200004f55000050200000bd
:1007f0003331000020440000495300004142000012
:100800004c45000044200000004f0000504700000d
:10081000524f0000555000002033000032200000ed
:100820004449000053410000424c00004544000090
:10083000200000004e4f00004e4500002020000028
:1008400020200000200000004f4600004649000024
:100850004345000020200000200000004245000029
:10086000445200004f4f00004d20000020000000c7
:10087000454e0000484100004e4300004544000042
:10088000200000004e4f0000204f00005054000098
:1008900020200000200000005052000049530000ba
:1008a0004f4e00002020000020000000202000000b
:1008b0002020000020200000202000002020000038
:1008c0002020000020200000202000002020000028
:1008d00020200000002000002020000053590000cc
:1008e00053540000454d0000204e00004f520000c0
:1008f0004d4100004c20000020200000200000009e
:10090000202000005359000053540000454d0000c2
:100910002052000045530000455400005449000097
:100920004e47000020200000002000005359000026
:1009300053540000454d0000204900004e4900007e
:1009400054490000414c000049530000494e00004a
:1009500047000000202000002053000059530000f1
:10096000544500004d200000535400004154000045
:10097000555300002020000020200000004500000a
:100980004e54000045520000204600004f52000027
:10099000204d00004f52000045200000444100005f
:1009a00054410000200000002020000020550000dd
:1009b0004e4300004f4d00004953000053490000d2
:1009c0004f4e000045440000202000002020000081
:1009d00000200000204500004e5400004552000059
:1009e000205500005345000052200000434f0000f6
:1009f000444500002020000020000000205000009e
:100a00005245000053530000205300004f55000092
:100a10004e440000204100004c410000524d0000b7
:100a20005320000000200000494e00005645000001
:100a30005354000049470000415400004520000085
:100a4000414c0000415200004d20000020000000f9
:100a5000505200004553000053200000534900004d
:100a60004c4500004e43000045200000414c000072
:100a7000415200004d530000002000005052000081
:100a8000455300005320000052450000534500002c
:100a900054200000504100004e4500004c20000052
:100aa0002000000020500000524500005353000079
:100ab000204d000055540000452000004255000024
:100ac0005a5a000045520000202000000055000046
:100ad00053450000522000004c45000056450000e0
:100ae0004c200000414300004345000053530000e8
:100af000454400002000000020200000434f00007b
:100b00004e540000524f00004c530000204500009e
:100b10004e410000424c00004544000020200000ef
:100b20000020000020200000202000004d41000097
:100b3000494e0000204d0000454e000055200000a9
:100b400020200000202000002000000020200000c5
:100b500020200000564900004557000020460000b4
:100b6000415500004c54000053200000202000009c
:100b700020200000002000005649000045570000da
:100b80002044000049530000414200004c45000051
:100b90004d4500004e54000053200000200000008e
:100ba000204e00004f20000045560000454e00003a
:100bb00054530000205400004f200000564900000c
:100bc0004557000020200000004300004c45000075
:100bd00041520000205300005953000054450000ca
:100be0004d20000046410000554c000054530000c9
:100bf0002000000020200000544500005354000055
:100c0000204900004e4400004943000041540000c8
:100c1000494f00004e53000020200000002a000031
:100c20002a2a00004c430000442a00004c490000de
:100c30004e450000312a0000544500005354000086
:100c40002a2a00002a0000002a2a00002a4c00005c
:100c5000434400002a4c0000494e00004532000089
:100c60002a54000045530000542a00002a2a00009c
:100c7000002a00002a2a00004c430000442a0000f9
:100c80004c4900004e450000332a00005445000046
:100c9000535400002a2a00002a0000002a2a0000db
:100ca0002a4c0000434400002a4c0000494e00003a
:100cb000453400002a54000045530000542a000027
:100cc0002a2a0000002000002045000058430000b0
:100cd000484100004e470000452000004445000008
:100ce000564900004345000053200000200000004a
:100cf0002020000052450000504c000041430000fd
:100d000045200000455800004953000054490000a8
:100d10004e4700002020000000200000204400007a
:100d2000455600004943000045530000205700008d
:100d300049540000482000004e45000057200000a4
:100d40002000000020200000204400004556000044
:100d50004943000045530000204f0000462000009a
:100d60005448000045200000202000000020000022
:100d70002020000020200000534100004d450000cd
:100d800020540000595000004520000020200000a1
:100d90002020000020000000204f00004c440000f4
:100da00020000000204e00004557000020000000f9
:100db000504100004e4500004c2000005749000003
:100dc0004c4c0000205200004553000045540000e8
:100dd000204100004e44000000200000205500008b
:100de00050440000415400004520000053490000d9
:100df0005445000020440000415400004120000000
:100e00002000000020200000202000005a4f000099
:100e10004e450000204f000050540000494f000094
:100e20004e5300002020000020200000005a000047
:100e30004f4e0000450000004e4f0000524d000094
:100e4000414c00000054000045530000544900008c
:100e50004e470000202000000044000045560000de
:100e60004943000045530000204900004e20000087
:100e70005448000049530000205a00004f4e000023
:100e8000450000002020000020200000415200000a
:100e900045200000494e0000204100004c41000068
:100ea000524d000020200000202000000020000003
:100eb00020500000414e0000454c0000205700002b
:100ec000494c00004c2000005245000053450000f2
:100ed00054200000200000002020000044490000b1
:100ee00053410000424c0000452000004f500000dc
:100ef000544900004f4e0000532000002020000005
:100f00000046000049520000452000004c49000006
:100f10004e4b000000420000555a00005a450000a8
:100f200052000000454e0000414200004c450000c8
:100f300044200000004400004953000041420000ea
:100f40004c45000044000000202000004544000003
:100f50004954000020440000455600004943000069
:100f60004520000054450000585400002020000097
:100f700000200000202000004544000049540000eb
:100f8000205a00004f4e000045200000544500004c
:100f900058540000202000002000000020530000d2
:100fa000455400002044000041540000452000004a
:100fb000414e000044200000544900004d4500000f
:100fc00020200000002000002056000049450000bd
:100fd00057200000414c0000415200004d2000000d
:100fe000434f0000554e0000542000002000000038
:100ff000202000004c4f0000472000004c4f000014
:101000004f500000204400004556000049430000b6
:10101000455300002020000000520000455300000e
:1010200045540000544900004e470000004c0000a9
:101030004f470000474900004e470000004d0000a8
:1010400041500000504900004e470000004300009e
:101050004f4d0000504c000045540000450000007a
:101060005355000043430000455300005300000067
:1010700046410000494c000045440000004c00007f
:101080004f4f000050000000434c00004f53000041
:101090004544000000490000534f00004c00000090
:1010a000505200004f470000524100004d20000008
:1010b000414400004452000045530000532000000a
:1010c000444100005441000000410000444400003d
:1010d0005245000053530000005300004e550000dd
:1010e0004d000000494e0000505500005420000003
:1010f000475200004f55000050200000004f0000f4
:101100005554000050550000542000004752000084
:101110004f550000500000004c41000054430000b7
:10112000484900004e470000202000002020000019
:10113000004e00004f4e0000204c000041540000c3
:1011400043480000494e00004700000044410000b1
:1011500059200000534500004e530000202000009d
:10116000200000004e4900004748000054200000c5
:10117000534500004e53000020000000564f000071
:101180004c5500004d4500002020000020200000ac
:1011900020200000200000004c4f000057200000dd
:1011a000004d0000454400002000000048490000b8
:1011b00047480000004900004e560000414c000026
:1011c00049440000004300004c410000535300001c
:1011d000202000002020000020200000004100000e
:1011e000555400004f4d0000415400004943000099
:1011f000004d0000414e0000554100004c20000011
:101200002020000000530000494c0000454e000023
:10121000434500002020000000520000455300001c
:101220004554000020200000202000000053000052
:101230004e440000204100004c4d000053200000af
:1012400000410000434300004550000054200000ce
:1012500020200000004900005245000053450000d6
:10126000542000002020000000200000202000006a
:10127000204400004556000049430000452000007e
:10128000525600004156000020200000202000009f
:10129000200000004445000056490000434500007e
:1012a000532000005345000054200000544f00001c
:1012b000205200005641000056200000004300006c
:1012c000414e00004e4f00005420000044450000f5
:1012d0005445000043540000204100002046000017
:1012e000495200004500000020200000202000009e
:1012f000204300004f4e0000544900004e550000ae
:10130000452000003f200000202000002020000099
:1013100000530000544100005254000020410000de
:1013200044440000524500005353000000450000b3
:101330004e4400002041000044440000524500009b
:101340005353000020200000002000002020000057
:1013500020200000564900004557000020460000ac
:1013600049520000452000002020000020200000fd
:10137000200000002020000020200000564900002e
:101380004557000020470000454e00004552000030
:10139000414c000020200000202000000020000020
:1013a000202000002020000045560000454e00008f
:1013b000542000004c4f0000472000002020000077
:1013c00020200000200000002020000056490000de
:1013d000455700002046000049520000452000000b
:1013e00045560000454e00005453000020200000e8
:1013f0000056000049450000572000004745000006
:101400004e450000524100004c20000045560000af
:10141000454e000054530000200000002020000032
:1014200020200000204300004c45000041520000f5
:101430002046000049520000452000002020000006
:10144000202000000020000020200000434c00006d
:101450004541000052200000474500004e45000075
:10146000524100004c20000020200000200000001d
:10147000204100004c4c0000204600004952000072
:10148000452000004c4f0000472000004441000070
:101490005441000020200000004100004c4c00009e
:1014a00020470000454e000045520000414c00001e
:1014b000204c00004f470000204400004154000031
:1014c00041000000574900004c4c00002042000041
:1014d0004520000050450000524d0000414e0000e4
:1014e000454e0000544c0000592000000020000030
:1014f000202000002020000020440000454c000077
:101500004554000045440000202000002020000039
:1015100020200000200000002020000020440000c7
:1015200049530000504c00004159000020200000a9
:101530004c4f00004f5000002020000020200000f1
:10154000002000002020000020440000455600003c
:101550004943000045200000444100005441000080
:10156000202000002020000020000000545900002e
:10157000504500002000000028530000485400009f
:1015800029000000284d000045440000290000000b
:10159000284c00004e470000290000005430000095
:1015a00020200000543100002020000054320000b0
:1015b0002020000054330000202000005448000088
:1015c00020200000004d000049530000534500005a
:1015d0004420000053430000414e0000530000002f
:1015e000434f000020460000415500004c540000cd
:1015f0002020000020200000005200005641000082
:10160000560000004c4500004420000053540000e8
:101610004154000045200000004f00004e20000013
:10162000004f000046460000004400004554000002
:10163000204f00004e0000005250000054200000d7
:101640004f4e000000440000455400002f5200009f
:1016500050540000204f00004e0000005052000087
:10166000454100004c410000524d00000041000087
:101670004c410000524d000000460000414900006e
:101680004c45000044200000534500005455000024
:10169000500000004d5500004c540000490000006f
:1016a000434f000020430000454c00004c20000048
:1016b0004f4b000020200000004500004550000076
:1016c000524f00004d200000505200004f470000d4
:1016d000202000000050000041530000534500004e
:1016e000440000002044000049530000504c00001a
:1016f000415900002044000049410000474e0000cd
:101700004f53000054490000432000000020000017
:1017100020200000202000002020000020440000a5
:101720004154000041200000202000002020000043
:1017300020200000200000002020000020200000c9
:10174000204c00004f4f000050200000444100009a
:101750005441000020200000202000002020000034
:10176000004c0000502000004f4c000020560000ac
:10177000414c0000004c0000502000004443000099
:1017800020560000414c00000020000020410000d5
:1017900055580000494c00004c49000041520000df
:1017a0005920000044410000544100002020000066
:1017b0002000000041550000582000003234000095
:1017c000562000000046000049520000454c000031
:1017d000494e00004b0000002020000020200000a7
:1017e000202000005053000055200000444100001c
:1017f0005441000020200000202000002020000094
:10180000004300004852000047200000564f0000ef
:101810004c540000530000004241000054540000aa
:10182000205600004f4c00005453000000420000be
:101830004154000054200000494d00005020000099
:101840002000000020200000204400004953000038
:10185000504c00004159000020500000414e000053
:10186000454c000020200000202000000020000047
:1018700020200000202000002044000045540000eb
:10188000414900004c5300002020000020200000af
:1018900020200000200000005357000020560000c8
:1018a0004552000020000000535000002056000068
:1018b0004552000020000000534600002052000066
:1018c000455600000020000020200000434f00008b
:1018d0004e4e00004543000054200000544f0000cd
:1018e00020500000432000002020000020000000c5
:1018f0002020000020200000205500005349000057
:101900004e470000205500005342000020200000f8
:1019100020200000202000000020000020200000e7
:101920002020000020570000415200004e490000d6
:101930004e47000020200000202000002020000052
:10194000200000005359000053540000454d000092
:1019500020430000414e00004e4f00005420000084
:10196000444500005445000043540000002000009e
:10197000464900005245000053200000494e000037
:101980002054000048490000532000004d4f000043
:1019900044450000200000002020000020520000ec
:1019a00045530000544100005254000020530000f1
:1019b00059530000544500004d2000002020000035
:1019c00000200000434c0000454100005220000070
:1019d000414c0000415200004d200000434f0000e8
:1019e000554e00005420000020000000204100005f
:1019f0004c410000524d0000204300004f550000b4
:101a00004e5400004552000020570000494c000091
:101a10004c200000002000002020000020200000ba
:101a200042450000204300004c45000041520000a8
:101a3000454400002020000020200000200000007d
:101a40002020000052450000535400004f52000077
:101a5000452000004445000046410000554c000070
:101a6000545300002020000000200000202000002f
:101a700020200000202000002059000045530000d5
:101a80002020000020200000202000002020000056
:101a90002000000020200000202000002020000066
:101aa000202000004e4f00002020000020200000d9
:101ab0002020000020200000202000000020000046
:101ac000202000002020000045580000495400005c
:101ad000204d0000454e0000552000002020000051
:101ae000202000002000000046410000554c00006e
:101af0005400000046490000524500000044000028
:101b000049530000414200004c4500004d45000093
:101b10004e540000004400004953000000540000ef
:101b200045530000540000004f46000000460000ee
:101b30004952000053540000004c00004154000082
:101b40004553000054000000494e000000450000cd
:101b5000564500004e540000005300005441000060
:101b6000544500002020000020000000494e0000e5
:101b700049540000004100004c410000524d00005b
:101b80005300000053450000454e00002053000064
:101b9000434100004e53000020200000004600009a
:101ba000415500004c54000053000000444900001f
:101bb00053410000424c0000454d0000454e0000de
:101bc00054530000005a00004f4e000045530000df
:101bd0000020000020200000494e0000434f00007c
:101be000525200004543000054200000434f0000c3
:101bf00044450000202000002000000020200000bc
:101c000020430000414c00004c200000494e0000e1
:101c100053540000414c00004c450000522000008d
:101c20002020000000530000430000004f4300004c
:101c3000004f00004b000000475200004f550000cd
:101c4000500000002020000020200000414c000037
:101c5000415200004d530000204100004354000059
:101c60004956000045200000202000000020000010
:101c70005341000056450000204100004c4c00003c
:101c800020430000484100004e470000455300003b
:101c9000203f000020000000200000002020000065
:101ca0004449000053410000424c00004520000020
:101cb0004120000044450000564900004345000013
:101cc0002020000000540000454300004820000090
:101cd000414c00004d20000000490000205300004e
:101ce0005749000054430000482000000044000011
:101cf00049530000204300004e54000020470000dc
:101d00000044000049530000204f000050470000ed
:101d1000333100000044000049530000204f000010
:101d20005047000033320000000000000080000037
:101d3000158000002a8000003f80000054800000d1
:101d4000698000007e80000093800000a880000071
:101d5000bd800000d2800000e7800000fc80000011
:101d600011810000268100003b81000050810000ad
:101d7000658100007a8100008f810000a48100004d
:101d8000b9810000ce810000e3810000f8810000ed
:101d90000d82000022820000378200004c82000089
:101da00061820000768200008b820000a082000029
:101db000b5820000ca820000df820000f4820000c9
:101dc000098300001e830000338300004883000065
:101dd0005d83000072830000878300009c83000005
:101de000b1830000c6830000db830000f0830000a5
:101df000058400001a840000248400002e84000062
:101e000038840000428400004c84000056840000a6
:101e10006b8400008084000095840000aa84000088
:101e2000bf840000d4840000e9840000fe84000028
:101e300013850000288500003d85000052850000c4
:101e4000678500007c85000091850000a685000064
:101e5000bb850000d0850000e5850000fa85000004
:101e60000f86000024860000398600004e860000a0
:101e700063860000788600008d860000a286000040
:101e8000b7860000cc860000d2860000d88600000d
:101e9000ed86000002870000178700001c87000005
:101ea000238700002d87000042870000578700002d
:101eb0006c870000818700008b87000092870000fc
:101ec0009b870000a4870000b9870000ce87000030
:101ed000e3870000f88700000d88000017880000e5
:101ee0001f88000027880000308800003888000024
:101ef0003f880000448800004b88000050880000a4
:101f0000658800006d880000728800007f880000ee
:101f10008c88000099880000a6880000b288000024
:101f2000be880000cc880000d1880000d688000060
:101f3000db880000e3880000ef880000f9880000db
:101f4000038900000d890000178900002189000025
:101f50002b890000358900004a8900005f89000054
:101f6000748900008989000097890000a589000014
:101f7000ba890000cf890000e4890000f9890000d7
:101f80000e8a0000238a0000388a00004d8a000073
:101f9000628a0000778a00008c8a0000a18a000013
:101fa000b68a0000bc8a0000c28a0000c88a00000d
:101fb000ce8a0000e38a0000f08a0000fd8a00005b
:101fc000028b00000d8b0000118b0000158b0000b0
:101fd0001c8b0000238b00002e8b0000378b000031
:101fe0003d8b00004a8b0000508b00005d8b000091
:101ff0006b8b0000728b0000878b00009c8b0000b5
:10200000b18b0000bb8b0000c58b0000da8b000099
:10201000e38b0000ec8b0000018c00000c8c0000b6
:10202000178c0000228c0000378c00004c8c0000c4
:10203000548c00005c8c0000638c0000788c0000e5
:102040008d8c0000a28c0000b78c0000cc8c0000ae
:10205000e18c0000f68c00000b8d0000208d00004c
:10206000358d00004a8d00005f8d0000748d0000ea
:102070007a8d00007f8d00008b8d00008f8d000019
:10208000948d0000978d00009d8d0000a48d0000b0
:10209000a78d0000ad8d0000b68d0000bb8d000047
:1020a000c28d0000cf8d0000d68d0000e38d0000b2
:1020b000e98d0000fe8d0000138e0000168e0000da
:1020c000198e00001c8e0000228e0000378e00004a
:1020d0004c8e00004e8e0000638e00006d8e00005e
:1020e000778e0000818e00008b8e00002020000083
:1020f000204f00004e54000052550000494d000092
:10210000494e000047200000414100004e200000e1
:102110002020000000200000204800004552000060
:1021200053540000454c0000205a00004f45000069
:102130004d4500005220000020200000200000003b
:102140002020000048450000525300005445000084
:102150004c200000434500004e5400005241000056
:102160004c4500002020000000200000202000003e
:102170004f4e000054520000554900004d490000e8
:102180004e47000020550000495400002020000068
:102190002000000020440000454500004c4e000097
:1021a000454d000045520000204e00004f520000f7
:1021b0004d410000414c00002020000000200000a4
:1021c00044450000454c00004e4500004d450000d0
:1021d00052200000494e0000204100004c41000008
:1021e000524d00002000000044450000454c000016
:1021f0004e4500004d45000052200000494e0000b1
:1022000020530000544f0000524900004e47000088
:1022100000440000454500004c4e0000204e0000e8
:102220004945000054200000494e00004745000089
:1022300053540000454c0000440000004445000099
:10224000454c00004e4500004d4500005220000066
:10225000564f00004f520000414c00004152000018
:102260004d200000002000005a4f00004e450000a5
:10227000205500004954000047450000534300002a
:10228000484100004b4500004c4400002000000085
:102290002020000020200000535400004f52000076
:1022a000494e0000472000005a4f00004e450000f4
:1022b000202000002020000000530000544f0000a8
:1022c000524900004e4700002042000045570000e0
:1022d0002053000054550000524900004e470000b2
:1022e00020000000204f00004e5400005255000016
:1022f000494d0000494e00004720000055490000ac
:1023000054530000434800002e20000000530000fa
:10231000544f0000524900004e4700002042000088
:1023200045570000204400004f4f0000524d000070
:10233000454c000044000000444f00004f52000094
:102340004d4500004c440000494e0000472000006d
:102350005549000054470000455300004348000021
:102360000020000020420000524100004e440000c6
:10237000204400004f4f000052470000454d000030
:10238000454c0000442000002000000020200000f8
:1023900020200000535400004f520000494e00001e
:1023a000472000004143000043550000202000006a
:1023b00020200000002000002047000045450000cc
:1023c0004e2000004e4500005453000050410000d4
:1023d0004e4e0000494e0000472000002000000043
:1023e000535400004f520000494e000047200000a7
:1023f0004e450000564500004e500000414e000082
:10240000454500004c20000000530000544f0000e0
:10241000524900004e47000020450000585400007b
:102420002e200000564f000045440000494e000099
:102430004700000047450000425200002e200000e7
:10244000434f000044450000204900004e47000073
:10245000455600004f450000524400000053000064
:1024600045520000562e0000204300004f4400005b
:1024700045200000494e000047450000564f00002f
:102480004552000044000000484f0000474500004e
:1024900052200000434f0000444500002049000046
:1024a0004e470000455600004f45000052440000d2
:1024b0000020000020200000544900004a44000091
:1024c000204900004e530000544500004c4c0000d1
:1024d000454e0000202000002000000020200000c9
:1024e00052450000535400004152000054200000a7
:1024f000434500004e540000524100004c4500008e
:10250000202000000020000020200000204c0000bf
:102510005553000020530000544f00005249000062
:102520004e47000020200000202000002000000076
:102530005a4f0000454d0000455200002055000054
:102540004954000047450000534300004841000043
:102550004b4500004c4400000020000020200000fb
:102560005043000020410000414e0000474500005c
:10257000534c00004f540000454e00002020000046
:102580002000000020200000205300004f460000e3
:10259000545700004152000045200000464f000003
:1025a00055540000202000002020000000200000e2
:1025b00044450000454c00004e2e00002054000011
:1025c0004f45000047450000564f000045470000ba
:1025d0004420000020000000535400004f5200002f
:1025e000494e0000472000004f4e000054520000aa
:1025f0002e520000494e0000474c00005553000089
:1026000000200000505200004f43000045530000de
:10261000534f000052200000535400004f5200005e
:10262000494e00004720000020000000202000004c
:10263000204c000055530000204900004e47000088
:10264000454c0000455a0000454e00002020000087
:102650002020000000200000474500004745000002
:10266000564500004e53000020410000414e00003e
:102670004745000050410000535400002000000076
:10268000202000004f4e000044450000524800004a
:102690004f550000442000004e4f00004449000008
:1026a0004720000020200000002000002020000023
:1026b0004e410000434800005453000054410000c4
:1026c0004e44000020410000414e00002020000048
:1026d000200000004f4e0000545200002e20000049
:1026e0005649000041200000504100004e450000c6
:1026f000454c000020410000414e00000020000039
:10270000535400004f520000494e00004720000083
:10271000444f00004f5200004d2e000020480000a2
:102720004d20000020000000202000004f55000038
:10273000545000005554000020470000524f000044
:102740005550000020550000495400002020000092
:1027500000200000202000005354000055520000cb
:10276000494e0000474500004e200000554900003a
:102770005420000020200000200000002044000021
:10278000454500004c4e00002e5500004954000005
:102790004745000053430000484100004b450000fe
:1027a0004c440000004f0000504700005020000043
:1027b0003331000020550000495400004745000017
:1027c00053430000484100004b2e00002000000051
:1027d0004f5000004750000020330000322000001e
:1027e000554900005447000045530000434800008d
:1027f000414b00002e20000000200000202000009f
:102800005359000053540000454500004d2000007e
:102810004e4f0000524d0000414100004c2000008e
:1028200020000000205300005953000054450000d0
:10283000454d0000204900004e20000048450000a2
:1028400052530000544500004c200000005300008b
:102850005953000054450000454d00002049000038
:102860004e49000054490000414c0000495300000b
:10287000494e0000470000002020000020530000c7
:102880005953000054450000454d000020530000fe
:102890005441000054550000532000002020000047
:1028a000004500004e540000455200002056000034
:1028b0004f4f0000522000004d45000045520000df
:1028c0002044000041540000410000004e49000037
:1028d000455400002047000045500000524f0000c2
:1028e00047520000414d00004d4500004552000098
:1028f00044200000005600004f4500005220000018
:102900004745000042520000554900004b2e000090
:10291000434f000044450000204900004e000000e5
:1029200044520000554b0000204f00004e54000060
:1029300052550000494d0000494e0000472000005c
:10294000414100004e200000002000004f4e0000da
:1029500044450000525a00004f4500004b20000043
:102960004d4500004c440000494e00004720000047
:102970002000000044520000554b0000204f000092
:102980004e54000052550000494d0000494e0000d1
:10299000472000005549000054200000004400007a
:1029a000525500004b2000004845000052530000e3
:1029b000544500004c200000434500004e540000e8
:1029c000522e00002000000020440000525500005c
:1029d0004b2000004f500000205a00004f450000df
:1029e0004d450000522000005549000054200000d1
:1029f000005400004f450000474100004e470000d2
:102a00002047000045420000522e0000204e0000ea
:102a100049560000454100005500000042450000b5
:102a200044490000454e0000494e00004720000088
:102a3000494e000020570000455200004b4900005d
:102a40004e47000000200000202000002020000051
:102a5000484f00004f460000444d0000454e000026
:102a60005520000020200000202000002000000051
:102a700020200000205400004f4f00004e20000096
:102a8000535400004f520000494e000047450000db
:102a90004e20000020200000005400004f4f000096
:102aa0004e200000554900005453000043480000e8
:102ab000414b0000454c0000494e000047450000d6
:102ac0004e00000020200000204700004545000087
:102ad0004e2000004d4500004c440000494e0000cf
:102ae000474500004e200000202000000048000064
:102af0004552000053540000454c00002053000094
:102b00005953000054450000454d0000464f000059
:102b1000555400002000000020200000202000006c
:102b2000202000004c4500004420000054450000d7
:102b3000535400002020000020200000202000002e
:102b4000002a00002a4c0000434400002a520000e2
:102b500045470000454c00002a3100002a5400007f
:102b600045530000542a00002a0000002a2a0000d1
:102b70004c430000442a0000524500004745000035
:102b80004c2a0000322a0000544500005354000033
:102b90002a2a0000002a00002a4c000043440000ba
:102ba0002a52000045470000454c00002a3300002f
:102bb0002a54000045530000542a00002a00000057
:102bc0002a2a00004c430000442a0000524500001d
:102bd000474500004c2a0000342a000054450000fc
:102be000535400002a2a000000440000454500001c
:102bf0004c4e0000454d000045520000205600009c
:102c000045520000564100004e470000454e00006e
:102c100020000000205600004552000056410000f0
:102c20004e47000020420000455300005441000080
:102c3000414e00004445000020200000002000001c
:102c400044450000454c00004e4500004d45000045
:102c500052530000204d0000455400002045000064
:102c6000454e0000200000004e4900004555000080
:102c70005745000020440000454500004c4e000030
:102c8000454d00004552000020560000414e000016
:102c9000002000002020000048450000545a000099
:102ca000454c0000464400004520000054590000f7
:102cb000504500002020000020000000204f0000b0
:102cc00055440000200000004e490000455500001a
:102cd0005700000020200000424d0000432000006b
:102ce0005a4100004c2000005245000053450000ae
:102cf00054540000454e0000202000000045000014
:102d00004e200000534f0000465400005741000081
:102d1000524500002055000050440000415400007e
:102d2000454e000020000000202000002020000070
:102d30005a4f00004e450000204f00005054000044
:102d40004945000053200000202000002020000002
:102d5000004e00004f5200004d410000414c000069
:102d600000540000455300005420000020200000c3
:102d7000202000000020000044450000454c0000d9
:102d80004e4500004d450000525300002049000010
:102d90004e200000444500005a450000200000007d
:102da0005a4f00004e4500002053000054410000df
:102db000414e0000204900004e200000414c000020
:102dc000415200004d200000002000005549000045
:102dd0005453000043480000414b0000454c0000a4
:102de000204f0000505400004945000053200000cf
:102df00020000000444f00004f5200004d450000ed
:102e00004c440000494e0000470000005a4f0000ab
:102e1000454d00004552000000410000414e0000b9
:102e20000055000049540000202000002020000030
:102e300020000000474500004546000020540000e7
:102e4000454b00005354000020440000454500005d
:102e50004c4e0000454d000045520000002000008f
:102e60002020000047450000454600002054000097
:102e7000454b000053540000205a00004f4e000004
:102e8000452000002000000020200000544f0000da
:102e90004f4e0000204100004c410000524d000008
:102ea000544500004c4c000045520000202000001a
:102eb0000041000044520000455300002020000063
:102ec0000049000052450000534500005420000016
:102ed0002020000020000000202000002020000012
:102ee000544f00004f4e00002042000052410000ad
:102ef0004e44000020200000202000002020000080
:102f00000020000020200000544f00004f4e000021
:102f100020530000544f0000524900004e4700006b
:102f2000532000002020000020000000202000008e
:102f30004d4500004c440000494e0000474500004c
:102f40004e200000494e0000204c00004f4700007a
:102f500020200000002000004c4f0000472000000f
:102f600042520000414e0000444d0000454c00001c
:102f7000444900004e470000454e0000200000007c
:102f800020200000204c00004f470000205300008c
:102f9000544f0000524900004e470000454e0000cb
:102fa0002020000020200000002000002020000041
:102fb000202000005749000053200000425200002a
:102fc000414e00004420000020200000202000008e
:102fd00020000000202000002020000057490000b1
:102fe00053200000535400004f520000494e00008f
:102ff000475300002020000020200000004a00006d
:1030000041200000004e0000454500000020000067
:103010002020000020560000455200004c410000d6
:1030200041540000204d0000454e00005520000096
:103030002020000020000000535400004f520000e8
:10304000494e00004700000042520000414e00007f
:10305000440000005549000054530000434800005c
:10306000414b0000454c0000494e00004700000065
:103070005549000054000000564100004e00000079
:10308000454500005253000054450000004c00002c
:10309000414100005453000054450000004d000021
:1030a000454c0000444900004e470000005300001a
:1030b000544100005455000053200000200000003f
:1030c0004f4e000054520000554900004d49000089
:1030d0004e47000000530000454500004e20000010
:1030e00053430000414e00005300000053540000c1
:1030f0004f520000494e0000474500004e000000be
:10310000554900005453000043480000414b000063
:10311000454c0000494e0000474500004e000000ad
:1031200020200000494e0000434f00005252000092
:103130004543000054450000204300004f44000078
:10314000452000002020000000420000454c000007
:103150002055000057200000494e00005354000045
:10316000414c00004c410000544500005552000005
:1031700020000000574900004a5a0000494700005b
:10318000494e0000474500004e2000004f5000000f
:10319000534c0000414100004e3f0000004200003f
:1031a000524100004e4400004d4500004c440000d8
:1031b000494e0000474500004e000000202000005e
:1031c000554900005453000043480000414b0000a3
:1031d000454c0000454e00002044000045450000dd
:1031e0004c2e000000000000769000008b90000044
:1031f000a0900000b5900000ca900000df90000091
:10320000f4900000099100001e910000bd800000b4
:1032100033910000489100005d9100007291000020
:10322000879100009c910000b1910000c6910000c0
:10323000db910000f091000005920000b9810000d0
:10324000ce8100001a9200002f92000044920000ec
:10325000599200006e920000839200009892000044
:10326000ad920000c2920000d7920000ec920000e4
:1032700001930000169300002b9300004093000080
:10328000559300006a9300007f9300009493000020
:10329000a993000087830000be930000b183000063
:1032a000c6830000db830000d3930000e893000096
:1032b0001a840000248400002e840000388400005a
:1032c000428400004c84000056840000fd930000fe
:1032d00012940000279400003c94000051940000d8
:1032e000669400007b94000090940000a594000078
:1032f000ba940000cf940000e4940000f994000018
:103300000e95000023950000389500004d950000b3
:1033100062950000779500008c950000a195000053
:10332000b6950000cb950000e0950000f5950000f3
:103330000a9600001f96000034960000499600008f
:103340005e960000649600006a9600007f9600007a
:103350009496000017870000a9960000b19600001f
:10336000bb960000d09600006a960000e59600002b
:10337000fa960000069700000d97000011970000d4
:103380001a9700002f970000599200004497000000
:10339000f88700000d880000178800001f880000d3
:1033a0002788000030880000388800003f8800002f
:1033b000448800004b8800005088000059970000a6
:1033c0006d880000728800007f8800008c880000f3
:1033d00099880000a6880000b2880000be8800001e
:1033e000cc880000d1880000d6880000db8800006f
:1033f000e3880000ef880000f988000003890000de
:103400000d890000178900002189000061970000e4
:10341000358900004a8900005f8900007489000036
:1034200089890000978900006c970000819700004f
:1034300096970000ab970000c0970000d59700005a
:10344000ea970000388a00004d8a0000628a000076
:10345000778a00008c8a0000a18a0000b68a0000ea
:10346000bc8a0000c28a0000c88a0000ce8a000020
:10347000e38a0000f08a0000fd8a0000028b000051
:10348000ff97000003980000158b00001c8b0000c4
:10349000238b00002e8b0000378b00003d8b00003b
:1034a0004a8b0000508b00005d8b00006b8b00008e
:1034b000728b0000878b00009c8b0000b18b00009a
:1034c000bb8b0000c58b0000da8b0000e38b000093
:1034d000ec8b0000018c00000c8c0000178c0000ad
:1034e000228c0000378c00004c8c0000548c0000b3
:1034f0005c8c0000638c0000788c00008d8c0000d8
:10350000a28c0000b78c0000cc8c0000e18c000085
:10351000f68c00000b8d0000208d0000358d000022
:103520004a8d0000079800001c98000024980000b5
:103530002a980000389800008f8d00003c98000009
:103540004098000047980000a48d00004f980000ac
:1035500057980000b68d0000609800006b9800003e
:103560007698000080980000e38d0000909800009d
:10357000a5980000138e0000168e0000198e000022
:103580001c8e000076900000ba980000cf980000d2
:10359000de980000638e00006d8e0000778e0000c4
:1035a000818e00008b8e0000205300005a490000dd
:1035b000524500004e4100004b200000414b0000ee
:1035c00054490000564100004c56000041200000c4
:1035d00000200000204b00004f5a0000504f000018
:1035e0004e540000204e0000454d0000495400009c
:1035f0004153000020200000200000002020000097
:103600004b4f00005a5000004f4e00005420000065
:10361000544f0000524f00004c560000452000005f
:103620002020000000200000204b00004f5a000026
:10363000504f00004e540000204e0000454d000049
:1036400049540000564100002020000020000000e6
:1036500020200000204e00004f5200004d4100008d
:103660004c200000455300005a4b00004f5a000008
:10367000202000002020000000200000522e00002a
:103680002d420000414e0000204c00004556000035
:103690004f200000455300005a4b00002e20000030
:1036a00020000000202000002020000048490000e9
:1036b0004241000053200000455300005a4b0000d7
:1036c0004f5a0000202000002020000000200000b1
:1036d0002045000047590000532e000048490000d3
:1036e000424100005320000042450000414c0000d0
:1036f0004c20000020000000202000004553000066
:103700005a4b00002e200000454c00004f52000094
:1037100049410000535a00005420000020200000be
:103720000020000054450000535a0000542e0000b1
:10373000424500004e4c0000455600002e5a000045
:103740004f4e00004120000020000000202000001b
:103750005a4f00004e410000204b0000494b000032
:1037600041500000435300004f4c00005641000000
:103770002020000000200000202000002020000069
:103780005a4f00004e41000020480000494200000e
:103790004120000020200000202000002000000028
:1037a0002020000020200000535a00004952000051
:1037b000454e000041200000484900004241000001
:1037c0002020000020200000002000002020000019
:1037d000535a0000495200002e2000004b490000bf
:1037e0004b41000050430000532e000020200000f9
:1037f00020000000205300005a5500004d2e00000c
:10380000545500005a2000004b4900004d2e000086
:103810004849000042410000202000000020000034
:10382000535a0000554d00002e540000555a000018
:10383000204b0000494d00002e4b0000494b00007a
:103840002e20000020000000205300005a550000e8
:103850004d2e0000545500005a2000004b49000036
:103860004d2e0000204100004b540000202000009d
:10387000002000002020000020200000414b00001c
:103880004b5500002e200000484900004241000036
:103890002020000020200000200000002020000048
:1038a00020480000414c00004f5a000041540000e5
:1038b000492000004849000042410000202000004b
:1038c000202000000020000020540000415600008d
:1038d0004b4900004a4500004c5a00004f200000b0
:1038e0004849000042410000202000002000000064
:1038f00020200000205400004150000045470000f7
:10390000595300004547000020480000494200008c
:1039100041200000202000000020000020200000a6
:103920004f5300005a540000414c00005920000041
:10393000564100004c54000041530000202000007c
:10394000200000002020000054410000564f0000dd
:103950004c4900002052000049410000535a000029
:1039600054410000532000002020000000200000ef
:10397000464500004c480000415300005a4e0000ec
:103980002e4b00004f44000020420000455600002e
:103990002e20000020000000202000004d450000e7
:1039a000524e00004f4b0000492000004b4f0000da
:1039b0004420000042450000562e00002020000058
:1039c0000020000020200000544500004c4500006d
:1039d000502e00004b4f00004420000042450000e4
:1039e000562e0000202000002000000020200000b3
:1039f000204f0000524100002042000045410000dd
:103a00004c4c0000495400004153000020200000ad
:103a10002020000000200000504100004e45000022
:103a20004c200000554a000052410000494e000061
:103a300044490000544100005320000020000000d1
:103a400020200000202000002048000055520000e7
:103a50004f4b000020480000494200004120000078
:103a6000202000002020000000200000205a00003c
:103a7000554d00004d450000522000004b4900000c
:103a80004b41000050430000532e00002020000056
:103a9000200000002050000043200000435300009d
:103aa000415400004c4100004b4f00005a540000ac
:103ab000415400005641000020200000002000007a
:103ac0002048000049420000415300002049000006
:103ad0004e4600002e2000004144000041540000ea
:103ae000202000002000000020450000535a000064
:103af0004b4f00005a200000484f00005a5a000067
:103b000041410000444100005341000020200000da
:103b100000200000482e000054410000504c0000de
:103b20002e200000535a0000495200002e48000089
:103b30004942000041200000200000002020000039
:103b400020200000505200004f4700002e46000089
:103b50002e200000484900004241000020200000c3
:103b600020200000002000002048000055520000e6
:103b70004f4b000020420000454f00004c56000013
:103b800041530000564100002020000020000000aa
:103b900020200000494e0000464f0000524d00001a
:103ba00041430000494f000020560000414c0000f6
:103bb000542e00002020000000200000535a000076
:103bc00045520000564900005a20000050450000b0
:103bd000524900004f440000555300002e200000c1
:103be00020000000204500004a5300005a2e00002b
:103bf0004d4f000044200000424500004b410000b2
:103c000050430000532e0000202000000020000040
:103c10002020000045560000414b000055410000a7
:103c2000434900004f200000414b0000542e00008b
:103c30002020000020000000205300005a55000002
:103c40004d2e0000545500005a2000004b49000042
:103c50004d20000048490000422e000020200000b6
:103c600000200000202000004b4900004d200000f3
:103c7000435300004f50000020480000494200001c
:103c8000412e0000202000002000000020460000ff
:103c90004f4c0000592e00004b4900004d2e0000f3
:103ca000435300004f50000048490000422e0000de
:103cb0002020000000200000204f00004c440000a5
:103cc000414c000020460000494c00004520000007
:103cd00048490000422e0000202000002000000083
:103ce00020200000455300005a4b0000204b0000ec
:103cf000494b000041500000435300004f4c00006e
:103d00005641000020200000004e0000494e0000f7
:103d1000435300002e200000202000000049000036
:103d2000524f0000444100002020000020200000ed
:103d300000480000414c00004f5300005a4f000063
:103d400042410000004d0000454700004552000080
:103d50004f53000049540000004e00004f20000067
:103d60004f500000434900004f2000000042000077
:103d70004f520000544f00004e2000002020000051
:103d800000200000204e00004f5200004d41000076
:103d90004c200000524500004e440000535a0000e1
:103da00045520000202000002000000020520000aa
:103db000454e0000445300005a45000052200000c8
:103dc000554a000052410000494e0000442e0000b8
:103dd0002020000000200000524500004e4400005a
:103de000535a000045520000204900004e44000094
:103df0004954000041530000412000002000000011
:103e000020520000454e0000445300005a45000077
:103e100052200000414c00004c410000504f000077
:103e2000544100002020000000200000204100003c
:103e300044410000544f00004b2000004245000068
:103e400056490000544500004c4500002020000069
:103e50002000000020200000202000002020000082
:103e600048490000414e0000595a00004f20000010
:103e70002020000020200000202000000020000062
:103e80002020000020460000454c0000482e000085
:103e90004b4f000044200000424500005620000027
:103ea0002020000020000000205300005a4900009c
:103eb000524500004e4100004b20000042450000ea
:103ec0004b41000050430000532e00002020000012
:103ed000002000002052000049410000535a000019
:103ee0005441000053200000464500004c440000af
:103ef000455200002e20000020000000202000007d
:103f000043530000454e000044450000532000008c
:103f100052490000415300005a5400004153000030
:103f20002020000000200000204b00005020000056
:103f30004a4500004c5a0000455300002054000040
:103f40004f5200004c4500005320000020000000ac
:103f5000202000005a5500004d4d00004552000041
:103f6000204e0000454d0000495400004153000020
:103f7000412000002020000000200000204600001a
:103f8000454c000048410000535a00004e200000fc
:103f9000484f00005a5a0000414600002e20000001
:103fa0002000000020200000204500004e470000b7
:103fb0002e200000564500005a450000524c0000db
:103fc00045530000202000002020000000200000b9
:103fd000202000002020000020200000464f00008c
:103fe0004d4500004e55000020200000202000001c
:103ff00020200000200000002020000020480000b9
:1040000049420000414b0000204d000045470000a0
:10401000544500004b2e000020200000202000000e
:1040200000200000202000004b4900004b41000010
:1040300050430000532e0000204d00004547000073
:10404000542e00002020000020000000204e000020
:10405000204d000045470000544500004b2e000055
:1040600020450000534500004d4500004e5900001a
:104070002020000000200000522e0000535a0000b3
:104080004552000048490000424100004b2e00000c
:10409000544f0000524c00002e2000002000000071
:1040a000202000002020000054450000535a00004a
:1040b000542000004a4500004c4500004b20000001
:1040c0002020000020200000002a00002a4c0000d0
:1040d000434400002a5600004f4e0000414c0000af
:1040e000312a000054450000535a0000542a0000b1
:1040f0002a0000002a2a00004c430000442a000045
:10410000564f00004e4100004c3200002a5400007f
:10411000455300005a5400002a2a0000002a0000db
:104120002a4c0000434400002a5600004f4e000075
:10413000414c0000332a000054450000535a00004f
:10414000542a00002a0000002a2a00004c430000e4
:10415000442a0000564f00004e4100004c3400003d
:104160002a540000455300005a5400002a2a000037
:104170000020000020450000535a00004b4f000073
:104180005a4f00004b2000004353000045520000ee
:10419000454a0000452000002000000020200000cb
:1041a000202000004d450000474c00002e2000005c
:1041b000454c000054410000562e00002020000015
:1041c00020200000002000002020000045530000b7
:1041d0005a4b00004f5a00004f4b00002041000096
:1041e0005a200000554a0000202000002000000056
:1041f0002020000020200000204100005a20000064
:10420000455300005a4b00004f5a00002020000088
:1042100020200000202000000020000020200000be
:10422000204100005a4f00004e4f00005320000074
:104230005449000050550000532000002020000089
:104240002000000052450000474900002000000007
:10425000205500004a20000020000000202000001f
:10426000412000004b500000205500004a52000041
:10427000414900004e4400002e200000455300003c
:104280002020000000200000204900004e460000d1
:104290002e20000046520000495300005349000000
:1042a000544500005345000020200000200000007d
:1042b00020200000202000005a4f00004e41000046
:1042c00020500000524f000047520000414d0000b6
:1042d0002020000020200000005a00004f4e000067
:1042e0004100000054450000535a000054450000ae
:1042f0004c45000053000000205a00004f4e0000c3
:1043000041420000414e000020540000414c00009a
:104310002e200000455300005a4b000020200000d2
:104320000020000052490000415300005a54000090
:104330002e420000414e000020560000414e000079
:104340004e4100004b200000200000002020000013
:104350004b5000002e5500004a5200004149000019
:104360004e44000049540000415300004120000029
:104370002020000000200000202000004b49000009
:104380004b410000502e0000204f00005043000021
:10439000494f00004b2000002020000020000000ba
:1043a0004f5300005a2e0000545500005a200000c0
:1043b0004b4900004d0000005a5500004d4d0000d3
:1043c00045520000004500004e4700002e5a0000f4
:1043d0004554000054200000200000004b4900001c
:1043e0004b41000050430000534f00004c5400006c
:1043f0000020000020200000455300005a4b000020
:104400002e5300005a4f0000562e0000204a000094
:104410004156000020200000200000002020000065
:10442000205a00004f4e0000412e0000535a000059
:104430004f5600002e2000004a4100005620000088
:104440002020000000200000204400004154000013
:10445000554d000020490000444f0000204200005c
:10446000454100004c4c00002e20000020000000c0
:104470002052000049410000535a00002e53000012
:104480005a4100004d4c00002e4d000045470000f1
:10449000542e0000202000000020000020480000d2
:1044a000555200004f4b000020420000454f0000d5
:1044b0004c560000415300004153000020200000f2
:1044c00020000000554a000052410000494e000003
:1044d0004449000054410000530000004e410000d8
:1044e000504c00004f5a00004153000000450000ae
:1044f000535a000020540000455200004b000000b9
:10450000544500004c4a0000455300000053000091
:10451000494b00004552000000480000494200009d
:104520004153000000480000555200004f4b00006e
:10453000005a00004152000054000000495a000097
:104540004f4c000000200000202000002050000000
:10455000524f000047520000414d00002043000030
:10456000494d000020200000202000002000000015
:10457000434900004d000000424500004d2e000060
:10458000435300004f500000202000002020000076
:10459000004b0000494d00002e430000534f000027
:1045a0005020000020200000200000004e59000094
:1045b00055470000544100005a4100004e4400009d
:1045c0004f200000004e0000454d0000204e00002e
:1045d0005955000047540000202000002000000032
:1045e0004e410000502e0000455200005a200000ad
:1045f0002020000020000000454a0000535a00001f
:104600002e49000020450000525a00002000000002
:10461000484100004e4700002020000020200000fc
:10462000202000002020000020000000414c00005d
:104630002e20000020200000200000004b4f000032
:104640005a45000050450000530000004d41000055
:104650004741000053200000200000004f5300009d
:104660005a540000414c0000592000002020000056
:104670002000000041550000544f00004d41000053
:104680005441000020200000004b0000455a00006b
:104690004920000020200000202000002000000011
:1046a00043530000454e00004445000053200000e5
:1046b00020200000005400004f5200004c45000034
:1046c000532000002020000020000000484100008e
:1046d0004e47000052490000415300005a54000068
:1046e000004100004c4b0000414c00004d410000d7
:1046f0005a5600004100000049200000544f0000bd
:10470000524c000045530000202000000020000013
:104710002020000020540000415600004f4c0000b3
:1047200049200000564900005a2e000020200000b9
:10473000202000002000000020450000535a000007
:104740004b2e000020560000495a00002e20000089
:1047500042450000414c00004c2e0000202000008b
:10476000002000002020000020540000555a0000c6
:10477000204e0000454d000020450000525a000028
:104780002020000020200000200000002020000049
:1047900020200000204600004f4c0000595400002b
:1047a000415400004a4100003f200000202000004a
:1047b00020200000004b0000455a0000444f00003c
:1047c00020430000494d0000202000002020000070
:1047d000005a0000415200004f20000043490000f1
:1047e0004d200000202000002020000000200000bc
:1047f00020540000555a0000204a0000454c00009b
:104800005a2e0000204d000045470000544500008e
:104810004b2000002000000020200000414c000040
:10482000544100004c4100004e4f00005320000056
:104830004e4500005a450000542000002020000092
:104840000020000020450000534500004d450000b9
:104850004e590000204e0000415000004c4f000017
:104860005a410000532000002000000020200000da
:10487000545500005a450000534500004d2e0000dd
:10488000204d000045470000544500004b2e00001d
:104890002020000000200000204100004c540000b7
:1048a0002e450000534500004d2e00004d450000f0
:1048b00047540000454b00002e200000200000005f
:1048c0002020000020200000545500005a20000045
:1048d000544f0000524c000045530000452000009a
:1048e00020200000202000000020000020410000c7
:1048f0004c540000414c0000414e00004f5300005a
:10490000205400004f5200004c450000532000008e
:1049100020000000204d0000494e000044450000ea
:104920004e200000545500005a4500005345000039
:104930004d4500004e5900002020000000200000de
:104940004d2e0000414c0000542e0000204e00006f
:10495000415000004c4f0000204100004441000045
:1049600054200000200000002020000056450000d8
:10497000474c0000454700004553000053450000e8
:1049800020560000414c0000494b00002020000050
:104990000020000020200000202000002054000003
:1049a0004f5200004f4c00005645000020200000f0
:1049b0002020000020200000200000002020000017
:1049c00020480000555200004f4b0000204b0000d3
:1049d000494a0000454c00005a45000053200000a1
:1049e00020200000002000002020000020200000e7
:1049f000455300005a4b00004f5a00002041000070
:104a0000444100005420000020200000200000004d
:104a1000544900005055000053200000005200008f
:104a20004f56000049440000004b00004f5a000060
:104a300020200000004800004f530000535a00009f
:104a4000004800005a200000564900005a53000058
:104a5000472e00002020000020000000414c0000f4
:104a6000542e000020480000494200004120000070
:104a70002020000000540000415600002e200000bd
:104a8000564900005a550000414c00002e0000001d
:104a90004c45000044200000414c00004c2e00001a
:104aa0002020000000420000454b00004150000063
:104ab000435300004f4c0000004b0000494b0000e6
:104ac00041500000435300004f4c000000450000df
:104ad0004c4f0000524900004100000052490000c4
:104ae000535a0000540000004849000042410000b1
:104af0005320000042450000414c00004c000000e3
:104b0000434f000020430000454c00004c200000b3
:104b1000524500004e440000004500004550000092
:104b2000524f00004d200000505200004f4700003f
:104b30002e200000004500004c4600004f470000ba
:104b400000200000202000004b4900004a450000e2
:104b50004c5a00004f20000044490000414700002b
:104b60002e20000020200000200000002020000057
:104b700020200000202000002020000041440000f0
:104b800041540000202000002020000020200000d0
:104b90002020000000200000202000002020000035
:104ba00048550000524f00004b20000041440000d7
:104bb00041540000202000002020000020000000c0
:104bc000202000004b4900004547000045530000ed
:104bd0005a490000544f00002041000044410000a9
:104be0005420000020200000003200003456000055
:104bf000204500005254000020000000202000004a
:104c000020200000205400004150000020450000fa
:104c100052540000454b00002020000020200000de
:104c20002020000000460000455300005a200000ec
:104c3000564100004c5400002e000000414b000083
:104c40004b55000020560000414c0000542e00003f
:104c5000004100004b4b000055200000494d000072
:104c6000502e00002000000020200000204b0000fb
:104c7000494a0000454c00005a4f000020500000f7
:104c8000414e0000454c0000202000002020000084
:104c900000200000202000002020000052450000dd
:104ca000535a00004c450000544500004b200000c2
:104cb0002020000020200000200000002020000014
:104cc00043530000415400004c2e000020410000de
:104cd00020500000432d0000484500005a200000ed
:104ce000202000000020000020200000555300007c
:104cf0004220000048410000535a00004e4100008d
:104d00004c41000054410000202000002000000021
:104d100020200000204600004947000059450000bf
:104d20004c4d0000455a0000544500005445000019
:104d3000532000002020000000200000205200002e
:104d4000454e0000442e00004e4500004d2000005e
:104d50004b450000502e0000455200005a20000034
:104d6000200000002020000020540000555a0000c0
:104d70004a2e000020450000204d00004f44000056
:104d8000424100004e2000002020000000200000d2
:104d900020520000454e0000445300005a450000d8
:104da00052200000554a000052410000494e0000c8
:104db0004420000020000000205200004941000073
:104dc000535a0000542e0000535a0000414d000079
:104dd0004c2e0000544f0000524c000020200000d8
:104de0000020000052490000415300005a540000c6
:104df00041530000205300005a4100004d4c000078
:104e0000414c00004f20000020000000204b00001b
:104e1000494b000041500000435300002e48000061
:104e2000454c000059520000454100004c2e000046
:104e30002020000000200000202000002020000092
:104e40002020000020490000474500004e200000bf
:104e50002020000020200000202000002000000072
:104e60002020000020200000202000002020000042
:104e70004e4500004d2000002020000020200000b2
:104e80002020000020200000002000004b490000ee
:104e90004c45000050450000532000004120000018
:104ea0004d4500004e550000424f00004c200000d0
:104eb000200000004849000042410000005400006a
:104ec000555a0000004b0000494b000041500000c3
:104ed000435300004f4c00004153000000450000c8
:104ee0004c5300004f000000555400004f4c000090
:104ef000534f000000450000534500004d450000a1
:104f00004e590000004100004c4c00004150000090
:104f10004f5400002000000052490000415300009f
:104f20005a540000415300004f4b0000004800005d
:104f300049420000414b0000004b0000494b00007b
:104f400041500000435300004f4c0000415300000b
:104f50004f4b0000005a00004f4e0000414b000034
:104f600000200000202000002045000052560000d4
:104f7000544c0000454e0000204b00004f44000000
:104f80002020000020200000200000002048000019
:104f9000495600004a410000204100002054000012
:104fa000454c000045500000495400004f5400009b
:104fb0002020000000430000534f0000500000007c
:104fc000202000002052000049410000535a0000f8
:104fd0005441000053200000414b000054490000a0
:104fe000562000002020000000200000204d00007e
:104ff000454e00005449000020410000204d0000b3
:105000004f4400002e2d00004f5400003f200000b0
:105010002000000020200000455300005a4b0000f3
:10502000204b0000494b000041500000435300005a
:105030004f4c000041530000202000000000000001
:10504000d49a0000e99a0000fe9a0000139b000029
:10505000289b00003d9b0000529b0000679b0000c6
:105060007c9b0000919b0000a69b0000bb9b000066
:10507000d09b0000e59b0000fa9b00000f9c000005
:10508000249c0000399c00004e9c0000639c0000a2
:10509000789c00008d9c0000a29c0000b79c000042
:1050a000cc9c0000e19c0000f69c00000b9d0000e1
:1050b000209d0000359d00004a9d00005f9d00007e
:1050c000749d0000899d00009e9d0000b39d00001e
:1050d000c89d0000dd9d0000f29d0000079e0000bd
:1050e0001c9e0000319e0000469e00005b9e00005a
:1050f000709e0000b1830000c6830000db830000c7
:10510000f083000005840000859e00008f9e000053
:10511000999e0000a39e0000ad9e0000b79e000077
:1051200056840000c19e0000d69e0000eb9e000049
:10513000009f0000159f00002a9f00003f9f000075
:10514000549f0000699f00007e9f0000939f000015
:10515000a89f0000bd9f0000d29f0000e79f0000b5
:10516000fc9f000011a0000026a000003ba0000052
:1051700050a0000065a000007aa000008fa00000f1
:10518000a4a00000b9a00000cea00000e3a0000091
:10519000f8a000000da1000022a1000028a100003d
:1051a0002ea1000043a1000058a100006da1000045
:1051b0001c87000072a100007ca1000091a10000ea
:1051c000a6a10000bba10000d0a10000dca100004e
:1051d000e3a10000eea10000f9a100000ea2000072
:1051e00023a2000038a200004da2000062a200002d
:1051f0006ea2000077a2000080a2000087a200003b
:105200008da2000093a2000099a200009ea20000bf
:10521000a3a20000b8a200006d880000bca200009c
:10522000c9a20000d6a20000e3a20000f0a2000084
:10523000fca2000008a3000016a300001ea30000ab
:1052400026a30000db8800002ea300003aa3000084
:1052500045a3000050a300005ba3000066a300006c
:1052600071a300007ca3000087a300009ca30000a2
:10527000b1a30000c6a30000dba30000e9a3000067
:10528000f7a300000ca4000021a4000036a4000035
:105290004ba4000060a4000075a400008aa40000d4
:1052a0009fa40000b4a40000c9a40000dea4000074
:1052b000f3a4000008a500000fa5000015a500003c
:1052c0001ba50000ce8a000021a500002ea500002d
:1052d0003ba5000048a5000053a500005da5000007
:1052e000158b00001c8b0000238b000067a50000bd
:1052f0006ea5000074a500004a8b000080a5000088
:105300008da500009ba50000a1a50000b6a500008a
:10531000cba50000b18b0000bb8b0000e0a5000016
:10532000f5a50000e38b0000fea5000013a6000019
:105330001ea6000029a6000034a6000049a6000011
:105340004c8c0000548c00005c8c00005ea60000b9
:1053500073a6000088a600009da60000b2a600006b
:10536000c7a60000dca60000f1a60000c9a400004a
:1053700006a700001ba7000030a7000045a70000fb
:105380005aa700005fa7000063a700008b8d0000f4
:105390008f8d0000948d00006fa7000074a700009f
:1053a000a48d00007ba7000083a70000b68d00003d
:1053b0008ca70000c28d000097a700009da70000e9
:1053c000aba70000b1a70000c6a70000138e000025
:1053d000168e0000198e0000dba70000e0a7000079
:1053e000f5a700004c8e00000aa80000638e0000a4
:1053f0006d8e0000778e0000818e00008b8e000085
:10540000414c0000415200004d4f00005247000047
:10541000414e0000204100004b540000495600005e
:105420004552000054200000002000002020000011
:105430002020000020410000565300005449000085
:105440004c540000202000002020000020200000fc
:10545000200000002020000020200000544900000f
:105460004c420000414b00004553000054490000ed
:105470004c540000202000002020000000200000ec
:1054800020200000535500004d4d00004552000003
:105490002041000056530000544900004c540000c5
:1054a00020200000200000002020000020410000fb
:1054b000445200004553000053450000204e0000b8
:1054c0004f5200004d4100004c2000002020000001
:1054d000002000002041000044520000455300001d
:1054e0005345000020490000204100004c410000cd
:1054f000524d00002020000020000000202000006d
:1055000046450000494c00002050000041200000aa
:105510004144000052450000535300004520000064
:1055200020200000004100004452000045530000cc
:1055300053450000204f000050500000534500002c
:105540005454000020460000454900004c00000073
:105550002041000044520000455300005345000024
:10556000204600004f5200005641000052530000f8
:10557000454c0000202000000020000020200000fa
:10558000205300004f4e000045200000492000003d
:10559000544500005354000020200000202000004b
:1055a0002000000020200000205300004f4e00008b
:1055b0004520000046520000414b00004f420000d1
:1055c0004c45000054200000202000000020000076
:1055d0002020000020460000454900004c2000002b
:1055e00049200000534f00004e45000020200000dd
:1055f00020200000200000002020000020200000cb
:10560000204100004c410000524d000020460000a7
:10561000454900004c200000202000002020000010
:1056200000200000204100004c410000524d0000cd
:1056300020460000524100004b4f0000424c000049
:105640004554000020200000200000002020000021
:105650004f56000045520000464f000052490000de
:105660004e47000053460000454900004c20000012
:1056700020200000004f0000564500005246000068
:105680004f520000494e00004720000046520000e3
:10569000414b00004f4200004c4500005400000008
:1056a0004f56000045520000464f0000524900008e
:1056b0004e470000204100004b54000049560000b6
:1056c000455200005420000000200000202000006f
:1056d000204200004154000054450000524900009f
:1056e00020460000454900004c200000202000001a
:1056f00020000000202000002020000020200000ca
:105700004e4500005454000046450000494c00003e
:1057100020200000202000002020000000200000a9
:10572000205300004c41000056450000504100004d
:105730004e4500004c20000046450000494c00004a
:1057400020200000200000002041000055580000eb
:10575000204600004f520000535900004e490000ff
:105760004e47000053460000454900004c20000011
:1057700000200000202000004b4c0000415300009e
:1057800053450000204500004e44000052450000f3
:1057900054200000202000002000000020200000f5
:1057a00020200000204600004a450000524e000024
:1057b000414c0000415200004d200000202000001c
:1057c000202000000020000042520000554b000045
:1057d00045520000204b00004f44000045200000cf
:1057e00054410000535400004554000020000000c4
:1057f00020200000494e0000535400002e200000dd
:105800004b4f00004445000020540000415300006d
:105810005445000020200000002000004d41000001
:1058200053540000455200004b4f00004445000017
:105830002054000041530000544500005420000053
:105840002000000020200000204b00004c4f0000f2
:105850004b4b000045200000494e00004e53000015
:10586000542e000020200000202000000020000016
:10587000504100004e4500004c20000054490000fb
:105880004c420000414b00004553000054490000c9
:105890004c540000200000002020000020200000c8
:1058a000205300004c4f00005946000045460000c0
:1058b000454900004c20000020200000202000006e
:1058c0000020000020530000554d00004d45000011
:1058d0005220000046520000414b00004f420000a1
:1058e0004c45000054200000200000002020000053
:1058f000202000005043000020540000494c0000cc
:105900004b4f0000424c0000455400002020000096
:1059100020200000002000004f4d000052410000f8
:105920004445000020440000415400004120000094
:10593000534b00004144000045540000200000008b
:10594000534c00004f59000046450000454e0000f2
:1059500048450000542000004c410000475400001e
:1059600020540000494c000000200000205300009b
:105970004c4f000059460000454100004c410000da
:10598000524d000020460000454900004c20000018
:105990002000000020460000454900004c20000087
:1059a00049200000505200004f47000052410000c3
:1059b0004d4d000045540000202000000020000054
:1059c00020200000534c00004f59000046450000c5
:1059d000204c00004f4700004745000054200000c5
:1059e0002020000020000000204f00004d52000049
:1059f00041440000452000004441000054410000a3
:105a0000204500004e440000524500005420000094
:105a100000200000205400004944000020460000ff
:105a20004f5200002053000045520000564900002c
:105a3000434500002020000020000000202000003e
:105a40004e4100005454000020530000544900000f
:105a50004c4c0000494e00004720000050c500009b
:105a600020200000004100004c410000524d000089
:105a7000204600005241000020530000454e000027
:105a8000545200002e4100004b5400002000000042
:105a9000484f000056450000442e0000414c0000d5
:105aa0002e4f000056450000524600002e460000d2
:105ab000454900004c200000002000005554000023
:105ac000474100004e4700004552000020460000bc
:105ad000524100004b4f0000424c00004554000072
:105ae000200000004b4f00004e5400002e550000d7
:105af000544700002e470000522e0000465200007e
:105b0000414b00004f4200004c20000000200000ec
:105b100020460000454900004c2000005041000094
:105b2000204b00004f4e0000462e0000464900006a
:105b30004c20000020000000202000002020000059
:105b400041440000522e000046520000414b00002c
:105b50004f4200004c45000054200000202000006f
:105b600000550000544700002e470000522000005e
:105b70003331000020460000524100004b4f00002e
:105b8000424c000045540000200000005554000025
:105b9000472e000047520000203300003220000052
:105ba00046520000414b00004f4200004c450000af
:105bb00054200000004900004e470000454e000000
:105bc0002020000020200000004b00004f4e00006d
:105bd000544f00005220000020200000005300001d
:105be0004f560000455200004f4d0000202000009d
:105bf000004600004f5200004245000044520000a1
:105c000045540000004900004e470000454e00008a
:105c1000204f00005054000000460000454e000098
:105c200047530000454c00002020000000200000e9
:105c3000202000005359000053540000454d00003f
:105c4000204e00004f5200004d4100004c54000017
:105c50002020000020000000202000002054000030
:105c6000494c0000424100004b45000053540000e5
:105c7000494c00004c45000052200000202000004c
:105c80000020000020200000535900005354000061
:105c9000454d000045540000204900004e490000d9
:105ca000542e00002020000020000000205400009e
:105cb000525900004b4b0000204600004f5200009c
:105cc000204d0000455200002044000041540000d7
:105cd0004120000000200000204900004b4b000044
:105ce00045200000505200004f4700005241000084
:105cf0004d4d0000455200005420000020000000df
:105d000020200000544100005354000020420000b5
:105d1000525500004b450000524b00004f4400001c
:105d200045200000202000000054000052590000cf
:105d30004b4b0000204100004b540000495600002e
:105d400045520000204100004c410000524d00002f
:105d50002000000020200000205500004e440000dc
:105d600045520000534f00004b200000414c000002
:105d7000415200004d2000002020000000200000c3
:105d800020540000525900004b4b000020410000fd
:105d900056530000544900004c4c000020410000c4
:105da0004c20000020000000205400005259000048
:105db0004b4b000020540000494c000042410000c1
:105dc0004b45000053540000494c00004c2000009b
:105dd00000540000525900004b4b000020410000cd
:105de00056530000544900004c4c00002053000062
:105df000554d00004d4500005200000020420000bb
:105e0000455400004a4500004e4900004e4700003e
:105e1000204100004b54000049560000455200004c
:105e2000542000000020000020200000202000005e
:105e3000484f000056450000444d0000454e00000c
:105e40005920000020200000202000002000000039
:105e5000202000002053000045200000414b00009e
:105e60005449000056450000204600004549000006
:105e70004c200000202000000020000020530000e3
:105e80004520000046520000414b00004f420000f8
:105e90004c4900004e470000455200002020000001
:105ea0002000000020200000494e0000474500006f
:105eb0004e200000484500004e440000454c0000c4
:105ec0005345000052200000202000000020000068
:105ed000205300004c4500005454000020530000a3
:105ee00059530000544500004d460000454900004c
:105ef0004c2000002000000020200000544500003d
:105f000053540000204900004e440000494b00005b
:105f1000415300004a4f00004e20000020200000a6
:105f200000200000202000004259000054540000ce
:105f300045200000454e0000484500005445000043
:105f400052200000202000002000000045520000e8
:105f5000535400004154000054200000454b000001
:105f6000534900005354000045520000454e0000c4
:105f700044450000002000002020000041440000b3
:105f80005245000053530000452000004d450000dd
:105f9000442000004e590000202000002000000096
:105fa000202000002020000020410000445200007a
:105fb00045530000534500002041000056200000da
:105fc00020200000202000000020000020200000f1
:105fd00020530000414d00004d45000020540000ba
:105fe00059500000454e00002020000020200000f5
:105ff00020000000204700004d4c00002000000061
:10600000204e0000592000002000000053450000f1
:106010004e540000524100004c2000005449000042
:106020004c420000414b000045530000542e00003c
:106030004f47000000200000204f0000505000009b
:106040004441000054450000524500005220000029
:1060500044410000544100002020000020000000c6
:106060002020000020200000205300004f4e0000a0
:1060700045200000564100004c4700002020000051
:106080002020000020200000005300004f4e0000a0
:1060900045000000544500005354000045520000e4
:1060a0002020000020000000204100004452000099
:1060b0002e20000049200000444500004e4e000004
:1060c00045200000534f00004e4500004e200000c8
:1060d0000020000020200000202000004552000089
:1060e00020490000204100004c410000524d0000ba
:1060f0002020000020200000200000005345000068
:106100004e54000052200000544900004c42000050
:10611000414b000045530000544900004c4c000026
:1061200045520000002000002020000046520000e0
:10613000414b00004f4200004c450000205600003b
:10614000414c0000472000002020000020000000fb
:106150004f56000045520000464f000052490000d3
:106160004e470000004900004e5400002e5300002e
:10617000554d00004d45000052000000414b00000d
:10618000544900005600000046520000414b0000f8
:106190004f4200004c450000540000002020000049
:1061a000454e0000445200004520000041440000dc
:1061b000522e0000544500004b53000054200000b4
:1061c0002020000000200000204500004e44000078
:1061d0005245000020500000414e0000454c000098
:1061e000544500004b5300005420000020000000e4
:1061f00020200000534500005454000020540000ab
:1062000049440000204f00004720000044410000a6
:10621000544f000020200000002000002053000008
:1062200045200000414c0000415200004d2000007c
:10623000544500004c4c0000455200002020000056
:10624000200000004c4f0000474700002053000092
:106250004c4f000059460000454500004e480000e4
:1062600045540000454e0000452000000054000049
:10627000494c0000424100004b45000053540000cf
:10628000004c00004f47000047450000520000004e
:106290004645000052440000494700000046000007
:1062a000454900004c45000054000000534c0000dc
:1062b0004f590000464500000053000054450000bf
:1062c0004e4700005400000020500000524f0000d4
:1062d0004752000020410000445200004553000096
:1062e00053450000204400004154000041200000bc
:1062f0000041000044520000455300005345000097
:10630000004900004e4e0000472e0000475200009a
:10631000555000005045000020000000555400007a
:10632000472e000047520000555000005045000025
:1063300020200000004400004147000020530000de
:10634000454e00005320000020200000004e0000b9
:106350004154000054200000534500004e530000fb
:1063600020200000005600004f4c0000554d00005a
:10637000202000002020000020200000202000001d
:10638000004c0000415600002020000020000000ca
:106390004d45000044490000554d000000480000f4
:1063a0004f59000020200000200000005547000049
:1063b000594c000044490000470000004d4f0000c8
:1063c0004455000053200000202000002020000041
:1063d0002000000041550000544f0000004d000017
:1063e000414e0000554500004c4c000020200000ac
:1063f00000530000544900004c4c000045200000b0
:1064000020200000004100004b5400002e410000fd
:106410004c410000524d000020000000414b0000a4
:106420005345000050540000455200004500000054
:106430004952000045530000455400000020000070
:10644000202000002041000044520000455300007d
:106450005345000020520000564100005620000025
:1064600020200000200000002041000044520000d5
:106470002e2000005341000054540000205400001e
:10648000494c0000205200005641000056200000f8
:10649000004b0000414e0000204900004b4b000023
:1064a0004520000044450000542e0000204200001a
:1064b000524100004e4e000020000000202000004d
:1064c00020200000464f00005254000053450000b9
:1064d00054540000452000003f2000002020000010
:1064e00020200000005300005441000052540000de
:1064f0004144000052450000535300004500000095
:10650000534c000055540000544100004452000018
:1065100045530000534500000020000020200000eb
:1065200020200000205300004520000042520000bf
:10653000414e00004e2000002020000020200000de
:106540002000000020200000202000005345000013
:1065500020470000454e000045520000454c000019
:106560004c2000002020000020200000002000001f
:1065700020200000484500004e440000454c00002b
:1065800053450000534c00004f47000047200000d7
:1065900020200000200000002053000045200000c3
:1065a00042520000414e00004e20000048450000cd
:1065b0004e440000454c00005345000052200000ae
:1065c0000020000020200000205300004520000093
:1065d000484500004e440000454c00005345000073
:1065e0005220000020200000200000002020000099
:1065f0002041000056530000544900004c4c00005c
:1066000020420000524100004e4e000020200000b9
:106610002020000000200000204100005653000010
:10662000544900004c4c000020470000454e00003b
:1066300045520000454c00004c20000020000000a6
:10664000414c00004c450000204200005241000037
:106650004e4e000020480000454e0000444500001a
:106660004c53000045520000002000002041000073
:106670004c4c00004520000020480000454e000022
:10668000444500004c53000045520000202000000b
:106690002000000020560000494c0000204200006d
:1066a0004c49000020500000455200004d410000c0
:1066b0004e4500004e540000202000000020000045
:1066c0002020000020200000205300004c45000046
:1066d00054540000455400002020000020200000f9
:1066e00020200000200000002020000020200000ca
:1066f0002056000049530000205300004c4f00007a
:106700005946000045200000202000002020000005
:106710000020000020200000204100004452000022
:106720004553000053450000204400004154000040
:106730004120000020200000200000004c45000007
:106740004420000053540000415400005553000001
:1067500000500000410000004156000000460000cb
:106760004f52000056410000525300002e0000001e
:1067700053450000545500005020000046450000dd
:10678000494c00004554000000500000524f0000ea
:10679000472e000020450000505200004f4d0000e1
:1067a0002020000000200000205600004953000077
:1067b0002044000049410000474e00004f530000b4
:1067c000544900004b4b0000202000002000000036
:1067d0002020000020200000534c00004f590000f2
:1067e00046450000204400004154000041200000c4
:1067f00020200000202000000020000020200000b9
:1068000020200000204100005558000020440000d6
:106810004154000041200000202000002020000002
:10682000200000004f56000045520000462e000098
:106830002020000000200000202000002053000045
:10684000545200004f4d0000462e0000444100000d
:106850005441000020200000202000002000000003
:106860004c41000044450000535000002e20000021
:106870002020000000420000415400005445000068
:1068800052490000535000002e0000004241000019
:10689000545400002e4d00004f540000532e0000b1
:1068a00000200000202000002020000056490000a9
:1068b00053200000504100004e4500004c200000d5
:1068c00020200000202000002000000020200000e8
:1068d000202000002020000044450000544100001a
:1068e0004c4a0000455200002020000020200000fb
:1068f000202000000020000020200000204b00008d
:106900004f4200004c45000020540000494c00005c
:106910002050000043200000202000002000000044
:106920002020000020200000202000004d45000015
:1069300044200000555300004220000020200000a9
:106940002020000020200000002000002020000067
:106950002020000020410000445600004152000069
:10696000534500004c2000002020000020200000a3
:1069700020000000534500004e540000522e00003d
:106980004b4100004e200000494b00004b450000e9
:1069900020440000455400002e200000004200006a
:1069a000524100004e4e00002049000020440000eb
:1069b000454e00004e450000204d00004f440000b1
:1069c0005553000020000000202000005245000028
:1069d000535400004152000054200000535900005d
:1069e00053540000454d0000455400002020000095
:1069f00000540000494c0000424100004b4500009b
:106a000053540000494c00004c2000005445000045
:106a10004c4c0000455200002000000020200000e7
:106a2000414c0000415200004d2000005445000040
:106a30004c4c00004552000020560000494c00001c
:106a40002020000000200000204200004c490000ef
:106a500020540000494c0000424100004b4500001a
:106a600053540000494c0000542000002000000056
:106a7000474a0000454e00004f50000050520000b1
:106a8000455400005420000053540000414e0000c3
:106a9000444100005244000000200000202000007b
:106aa0002020000020200000202000004a4100009b
:106ab00020200000202000002020000020200000d6
:106ac00020000000202000002020000020200000e6
:106ad000202000004e45000049200000202000003a
:106ae00020200000202000002020000000200000c6
:106af00020200000202000004558000049540000dc
:106b0000204d0000454e00005920000020200000cc
:106b1000202000002000000046450000494c0000f5
:106b200000420000524100004e4e000000460000ae
:106b3000524100004b4f0000424c0000494e000003
:106b4000474500005200000046520000410000008e
:106b5000464f00005253000054450000005300000f
:106b6000495300005445000000490000004800005f
:106b7000454e0000444500004c5300004500000015
:106b8000494e000049540000494100004c490000b2
:106b90005345000052000000414c000041520000eb
:106ba0004d450000520000005649000053540000bb
:106bb00045200000534b0000414e00004e2e0000c7
:106bc000005300004f4e000045520000002000001e
:106bd000202000002020000046450000494c000015
:106be000204b00004f440000452000002020000002
:106bf000202000002000000020200000524900005a
:106c00004e470000204900004e5300005441000050
:106c10004c4c0000415400004f5200002020000066
:106c200000470000525500005050000000200000b6
:106c300020200000414c0000415200004d45000062
:106c400052200000414b000054490000564500000e
:106c500020200000200000004c41000047520000ae
:106c600045200000414c00004c450000204500003c
:106c70004e440000524900004e47000045520000bb
:106c800000200000202000002046000052410000ab
:106c90004b4f0000424c00004520000041440000e2
:106ca000522e00002020000020000000544500006b
:106cb0004b4e00002e4100004c2000002000000040
:106cc00000aa000015aa00002aaa00003faa00009e
:106cd00054aa000069aa00007eaa000093aa00003e
:106ce000a8aa0000bdaa0000d2aa0000e7aa0000de
:106cf000fcaa000011ab000026ab00003bab00007b
:106d000050ab000065ab00007aab00008fab000019
:106d1000a4ab0000b9ab0000ceab0000e3ab0000b9
:106d2000f8ab00000dac000022ac000037ac000056
:106d30004cac000061ac000076ac00008bac0000f5
:106d4000a0ac0000b5ac0000caac0000dfac000095
:106d5000f4ac000009ad00001ead000033ad000032
:106d600048ad00005dad000072ad000087ad0000d1
:106d70009cad0000b1830000c6830000db830000ef
:106d8000b1ad0000c6ad0000dbad0000e5ad000018
:106d9000efad0000f9ad000003ae00000dae000045
:106da0005684000017ae00002cae000041ae00007b
:106db000aa84000056ae00006bae000080ae00005a
:106dc00095ae0000aaae0000bfae0000d4ae000039
:106dd000e9ae0000e3ab0000feae000013af000020
:106de00028af00003daf000052af000067af0000c9
:106df0007caf00000f86000024860000398600006a
:106e00004e86000091af0000a6af0000bbaf0000af
:106e1000d0af0000e5af0000faaf000000b0000006
:106e200006b000001bb0000030b0000045b000000c
:106e30001c8700004ab0000054b0000069b0000098
:106e40007eb0000093b00000a8b00000b3b0000016
:106e5000beb00000c4b00000ceb00000e3b000003f
:106e6000f8b000000db1000022b1000037b1000001
:106e700041b100001f88000048b10000198e0000d9
:106e80004fb1000056b100005db100004b8800001a
:106e900064b1000079b100006d88000081b100008c
:106ea0008eb100008c880000998800009bb1000022
:106eb000a7b10000b3b10000c1b10000c8b100002b
:106ec000cfb10000d6b10000deb10000eab1000091
:106ed000efb10000f9b1000037b1000003b20000cb
:106ee0000eb2000018b200001fb2000034b2000061
:106ef00049b200005eb2000073b2000080b2000030
:106f00008db20000a2b20000b7b20000ccb2000007
:106f1000e1b20000f6b200000bb3000020b30000a5
:106f200035b300004ab300005fb3000074b3000043
:106f300089b30000b68a0000bc8a0000c28a000043
:106f4000c88a0000ce8a0000e38a0000f08a0000b0
:106f5000fd8a00009eb30000a9b30000acb300009e
:106f6000158b00001c8b0000238b0000afb30000ca
:106f7000378b0000b8b300004a8b0000508b000034
:106f8000c5b300006b8b0000d3b30000878b0000fb
:106f9000e8b30000b18b0000bb8b0000fdb3000024
:106fa000da8b000012b400001bb4000030b4000003
:106fb0003bb4000046b4000051b4000066b40000c9
:106fc0004c8c0000548c00005c8c00007bb40000f2
:106fd00090b40000a5b40000bab40000cfb4000023
:106fe000e4b40000f9b400000eb5000023b50000c1
:106ff00038b500004db5000062b5000077b500005f
:107000008cb5000091b5000097b50000a4b5000054
:107010008f8d0000acb30000a8b50000afb5000034
:10702000b5b50000b7b5000057980000c0b5000026
:10703000ccb50000d4b500008cb5000097b50000b9
:10704000e1b50000e7b50000fcb50000138e0000bc
:10705000168e0000198e000011b6000017b6000051
:107060002cb600004c8e000041b6000056b6000061
:107070006d8e0000778e0000818e00008b8e0000e8
:1070800003040000050600000700000001020000e4
:1070900020410000424300004445000046470000f4
:1070a000484900004a4b00004c4d00004e4f000084
:1070b0005051000052530000545500005657000034
:1070c000585900005a3000003132000033340000bb
:1070d000353600003738000039260000402800000f
:1070e000292c00002d2e00002f00000000000000c1
:1070f00000c00000000000000030000000000000a0
:10710000000c000000000000000300000000000070
:10711000c00000000000000030000000000000007f
:107120000c000000000000000300000000c0000090
:10713000000000000030000000000000000c000013
:10714000000000000003000000000000c00000007c
:107150000000000030000000000000000c000000f3
:1071600000000000030000000000000021220000d9
:1071700023240000010200000304000005060000b3
:10718000070800002526000027280000292a000003
:107190002b2c0000090a00000b0c00000d0e000053
:1071a0000f1000002d2e00002f30000011120000e3
:1071b000131400001516000017180000191a00001b
:1071c0001b1c00001d1e00001f200000001f0000ef
:1071d0001c1f00001e1f00001e1f00001f1e0000bd
:1071e0001f1e00001f0000001f1d00001f1e0000ca
:1071f0001f1e00001f1f00001e1f00001e1f00009a
:10720000005e0000bce20000613f0000dd83000082
:10721000c29c00007e200000a3fd00001f41000072
:107220009dc30000217f0000fca20000401e000062
:107230005f010000e3bd00003e60000082dc000052
:10724000237d00009fc10000421c0000fea0000042
:10725000e1bf00005d03000080de00003c62000032
:10726000bee00000025c0000df810000633d000022
:107270007c220000c09e00001d430000a1ff000012
:1072800046180000faa40000277900009bc5000002
:1072900084da000038660000e5bb000059070000f2
:1072a000db85000067390000bae4000006580000e2
:1072b00019470000a5fb000078260000c49a0000d2
:1072c000653b0000d9870000045a0000b8e60000c2
:1072d000a7f900001b450000c69800007a240000b2
:1072e000f8a60000441a000099c70000257b0000a2
:1072f0003a64000086d800005b050000e7b9000092
:107300008cd20000306e0000edb30000510f000081
:107310004e100000f2ac00002f71000093cd000071
:10732000114f0000adf30000702e0000cc92000061
:10733000d38d00006f310000b2ec00000e50000051
:10734000aff10000134d0000ce900000722c000041
:107350006d330000d18f00000c520000b0ee000031
:10736000326c00008ed00000530d0000efb1000021
:10737000f0ae00004c12000091cf00002d73000011
:10738000ca94000076280000abf500001749000001
:1073900008560000b4ea000069370000d58b0000f1
:1073a00057090000ebb50000366800008ad40000e1
:1073b00095cb000029770000f4aa000048160000d1
:1073c000e9b70000550b000088d60000346a0000c1
:1073d0002b75000097c900004a140000f6a80000b1
:1073e000742a0000c8960000154b0000a9f70000a1
:1073f000b6e800000a540000d78900006b35000091
:107400000505000005050000050f00000f0f000036
:107410000f0f0000070300000b0f00000b0f000010
:10742000030b00000b0300000b0700000701000026
:1074300001010000010b00000b070000010b000020
:10744000030700000f010000010100000405000017
:107450000b020000070f0000070f000005050000e9
:10746000070700000000000000000000000000000e
:10747000000000000000000000000000000000000c
:1074800000000000000000000000000000000000fc
:1074900000000000000000000000000000000000ec
:1074a00000000000000000000000000000000000dc
:1074b00000000000000000000000000000000000cc
:1074c00000000000000000000000000000000000bc
:1074d00000000000000000000000000000000000ac
:1074e000000000000000000000000000000000009c
:1074f000000000000000000000000000000000008c
:10750000013900000203000001000000000000003b
:1075100014000000f0000000484500004154000045
:10752000202000002000000021390000020300009c
:10753000010000000000000014000000f000000046
:107540004f50000054490000434100004c0000002f
:10755000223a0000020300000100000000000000c9
:1075600028000000fd0000004f50000054200000e3
:107570004854000020000000243b0000021b0000d3
:1075800001000000000000002d00000002010000ca
:107590004f50000048540000434f000020000000fe
:1075a000400900000200000001000000000000008f
:1075b00032000000c20100004d43000050200000d6
:1075c0002020000020000000d07a0000030300000b
:1075d0000100000000000000280000009b030000e4
:1075e0004f4800005344000020200000200000000d
:1075f000d17a00000f0300000119000023410000b0
:1076000037000000460500004f4800005f530000af
:107610005641000044000000d2fa000003030000bd
:107620000100000000000000280000008f0500009d
:107630004f4800005f5400004b2000002000000075
:10764000d3fa00000f0300000119000023410000dd
:1076500037000000e20400004f4800005f540000c3
:107660005641000044000000d47b0000031b0000d2
:1076700001000000000000002d000000a003000039
:107680004f4800004353000020200000200000006d
:10769000d57b00000f1b00000119000023410000f2
:1076a00037000000460500004f480000435300002b
:1076b0005641000044000000d6fb00000f1b0000f4
:1076c0000119000023410000370000007e04000083
:1076d0004f480000435400005641000044000000a1
:1076e000d779000003030000010000000000000043
:1076f000280000009b030000485400005f53000076
:107700004420000020000000d87900000f03000092
:107710000119000023410000370000004605000069
:10772000485400005f530000564100004400000030
:10773000d9f900000f0300000119000023410000e7
:1077400037000000e2040000485400005f540000cd
:107750005641000044000000da79000003030000f5
:107760000100000000000000280000009b03000052
:107770004f5000005f530000442000002000000034
:10778000db7900000e030000011900002341000016
:1077900028000000f1020000485400005f42000091
:1077a0004541000043000000dc7a00000e030000a9
:1077b000011900002341000037000000bc02000056
:1077c0004f4800005f5600004144000020000000c8
:1077d000dd7b00000e1b00000119000023410000aa
:1077e00037000000bc0200004f480000435f00006b
:1077f00056410000440000008349000001000000e1
:10780000010000000000000041000000f401000041
:1078100053530000523200002020000020000000de
:10782000a14900000d000000012500002c640000ab
:1078300046000000e204000053530000525f0000c5
:10784000564100004400000048090000020000000a
:107850000100000000000000410000009001000055
:107860004d490000502000002020000020000000b2
:10787000814900000000000001000000000000003d
:107880003c000000d0070000434300004f200000f0
:1078900020200000200000008249000002000000bb
:1078a000010000000000000037000000dc000000c4
:1078b0004d490000434300004f200000200000001d
:1078c0004909000000000000010000000000000065
:1078d000ac0d0000a00f00004c430000442000004d
:1078e00052500000540000008549000001000000d3
:1078f000010000000000000057000000a802000086
:1079000053420000415300004532000020000000b7
:107910008749000001000000010000000000000095
:107920003a0000009600000053420000415300005e
:1079300045340000200000008849000001000000dc
:1079400001000000000000003c000000e80300000f
:1079500042450000414300003220000020000000aa
:107960008649000001000000010000000000000046
:107970003a0000009600000042450000414300002c
:1079800034200000200000009e4900000d0000008f
:10799000011900002341000050000000f401000024
:1079a000435f00005641000044200000200000001a
:1079b000a44900000d000000012500002c58000023
:1079c00050000000ee020000575f0000564100002a
:1079d0004420000020000000a5c900000d000000a8
:1079e000012500002c6400003c000000460500005a
:1079f000545700005f560000414400002000000082
:107a000020390000020c000001000000000000000e
:107a1000340000005e010000494f00004e200000cd
:107a200020200000200000004109000002000000aa
:107a3000010000000000000032000000c201000050
:107a400046520000492000002020000020000000d5
:107a50008449000001000000010000000000000057
:107a60002b000000f4010000415300004e440000d0
:107a70005220000020000000a0490000000000008b
:107a8000010000000000000032000000c8000000fb
:107a9000505600005234000020200000200000005a
:107aa0009f490000000000000100000000000000ed
:107ab00032000000941100005056000052320000c5
:107ac00020200000200000009d490000010000006f
:107ad000010000000000000032000000c8000000ab
:107ae000535200005a50000056520000340000006b
:107af0009c4900000100000001000000000000009f
:107b0000320000004c1d0000535200005a5000008b
:107b100056520000320000009b49000001000000a6
:107b2000010000000000000032000000c80000005a
:107b3000535200005a3400002020000020000000b2
:107b40009a49000001000000010000000000000050
:107b500032000000d0070000535200005a320000eb
:107b60002020000020000000c349000003000000a6
:107b70000100000000000000c800000090010000ab
:107b8000415000005a410000492000002000000040
:107b9000c4490000020000000100000000000000d5
:107ba000bc020000bc02000031360000574100005a
:107bb0005920000020000000233a0000021b0000b2
:107bc000010000000000000023000000060100008a
:107bd000434f0000484500004154000020000000d1
:107be000c549000002000000010000000000000084
:107bf000bc020000bc02000031360000465200000a
:107c00004920000020000000894900000000000019
:107c100001000000000000003c000000a40600007d
:107c2000545f000042410000534500002000000066
:107c3000c749000000000000010000000000000033
:107c4000e8030000e80300004c4900005520000054
:107c50002020000020000000c649000002000000b3
:107c60000100000000000000bc020000bc02000097
:107c70003136000050410000492000002000000083
:107c80004549000002000000010000000000000063
:107c900000000000000000005350000052490000a6
:107ca0004e4b0000200000004609000000000000cc
:107cb00001000000000000000000000000000000c3
:107cc00052450000504500004154000020000000d3
:107cd000470a000002000000010000000000000050
:107ce0008a0200008a02000045560000414300005d
:107cf0002020000020000000c14a00000200000017
:107d000001000000000000006400000064000000aa
:107d1000435f0000434100004c4c00002000000085
:107d20009049000002000000010000000000000077
:107d300082000000f401000052530000545f000074
:107d40004d490000430000008a4a00000200000084
:107d50000100000000000000fa0000009001000097
:107d6000444100004d50000045520000200000003a
:107d7000300b0000020000000100000000000000c5
:107d80006400000064000000432000005052000026
:107d90004f20000020000000430a00000200000005
:107da00001000000000000008a0200008a020000ba
:107db00045560000414300005f4d000020000000d8
:107dc000cd090000020000000100000000000000da
:107dd000f4010000f4010000505200004f5f000069
:107de000504e000054000000a249000001000000b5
:107df000010000000000000032000000d007000079
:107e0000535300004e4400005220000020000000a8
:107e1000a3c90000010000000100000000000000f4
:107e20002d000000a2050000545f00005353000025
:107e30005232000020000000f509000000000000a0
:107e40000100000000000000be0000000000000073
:107e50004c46000046520000202000002000000098
:107e6000f64a0000000000000100000000000000d1
:107e7000be00000000000000535400004154000008
:107e80005f43000054000000f74b000000000000ba
:107e90000100000000000000be0000000000000023
:107ea00053540000415400005f4c0000500000009b
:107eb000f84b00000000000001000000000000007e
:107ec000be00000000000000504600004c4f0000c3
:107ed0004f44000020000000f909000000000000ed
:107ee0000100000000000000be00000000000000d3
:107ef000454c0000454300002042000020000000e7
:107f0000fa0900000000000001000000000000006d
:107f1000be000000000000004c440000525f000062
:107f20005320000020000000fb09000000000000ba
:107f30000100000000000000be0000000000000082
:107f4000434d0000204900004e5400002000000076
:107f5000fd0b000000000000010000000000000018
:107f6000be00000000000000535f0000434f00000f
:107f70004e54000020000000fe0b00000000000036
:107f80000100000000000000be0000000000000032
:107f9000434f00004e56000020200000200000004b
:107fa000c8490000020000000100000000000000bd
:107fb000460000002c1a00004c4f0000435f0000f8
:107fc000434e000054000000f44b0000000000008d
:107fd0000100000000000000be00000000000000e2
:107fe0004c450000445f0000424100004c0000008e
:107ff000bc090000020000000100000000000000b9
:108000000000000000000000524600005f52000027
:10801000505400002000000002390000020300005c
:10802000010000000000000000000000000000004f
:10803000524600005f48000054200000200000006d
:108040009149000002000000010000000000000053
:108050005a00000084030000344d00004943000032
:10806000434f000020000000c24900000300000050
:108070000100000000000000ae010000841c0000b0
:108080004c5000005a410000492000002000000030
:10809000ca490000030000000100000000000000c9
:1080a000120200002e220000344c0000505a000042
:1080b0004120000020000000c9490000030000002a
:1080c00001000000000000001e0000001e00000073
:1080d00034410000505a0000412000002000000000
:1080e000c049000002000000010000000000000084
:1080f0005a00000084030000344d00004950000085
:10810000434300004f000000330b0000020000005a
:1081100001000000000000004600000046000000d2
:10812000485900004252000049440000200000006d
:10813000ce0b000002000000010000000000000063
:108140004600000046000000505200004f50000062
:108150004e5400002b000000310b00000200000014
:10816000010000000000000000000000000000000e
:10817000524600005f4f0000502000002000000029
:10818000320b0000020000000100000000000000af
:108190000000000000000000524600005f4f000099
:1081a0005048000054000000ba4b000001000000dd
:1081b0000100000000000000ac0d0000ac0d00004c
:1081c000524600005f540000524100004e00000083
:1081d000b74b00000200000001000000000000009a
:1081e0000000000000000000524600005f43000055
:1081f0005048000054000000b34b00000100000094
:10820000010000000000000000000000000000006d
:10821000524600005f5300004e4400004200000040
:10822000500b0000020000000100000000000000f0
:108230000000000000000000524600005f4d0000fa
:108240004350000020000000bb0b000002000000b3
:10825000010000000000000000000000000000001d
:10826000524600005f4d0000495000002000000011
:10827000b04b000001000000010000000000000001
:108280000000000000000000524600005f420000b5
:108290004f50000020000000de49000001000000f7
:1082a0000100000000000000280000009b03000007
:1082b000364b0000505f00005320000020000000fb
:1082c000df4900000d0000000119000023410000fb
:1082d0002d00000046050000364b0000505f0000f6
:1082e0005356000020000000e0c90000010000001b
:1082f0000100000000000000280000008f050000c1
:10830000364b0000505f0000545300002000000076
:10831000e1c900000d000000011900002341000028
:108320002d000000e2040000364b0000505f00000a
:1083300054530000560000008b490000020000006a
:1083400001000000000000004c040000780500005f
:10835000464100004e200000435400004c00000045
:108360008e4900000a00000001000000000000002b
:1083700046000000900100004c500000344900000d
:108380004f20000020000000340b0000020000001d
:108390000100000000000000460000004600000050
:1083a0004343000044200000202000002000000083
:1083b000ff010000000000000000000000000000bd
:1083c0000000000000000000494e0000564100007f
:1083d0004c49000044000000000000007d00000047
:1083e000000000003c0000003800000038000000e1
:1083f0003900000000000000000000000000000044
:1084000000000000cefa0000fcf90000fcf90000ba
:10841000fcf90000fcf90000c2f80000ccf80000f4
:10842000eaf80000fcf80000e8d0000000000000be
:1084300000000000190000003800000038000000b3
:1084400038000000380000000000000000000000bc
:108450000000000000000000fafa00000afb000023
:1084600030fb000056fb000086fb0000c2f8000055
:10847000ccf80000eaf80000fcf80000b0fb0000b7
:1084800000000000000000000200000038000000b2
:108490003f00000040000000380000000000000025
:1084a000000000000000000000000000e8d0000014
:1084b000fcf90000fcf90000fcf90000fcf90000e8
:1084c000c2f80000e8d00000eaf80000fcf8000064
:1084d000e8d00000000000000000000005000000df
:1084e00041000000380000003f0000004200000092
:1084f000000000000000000000000000000000007c
:10850000e8d00000fcf90000fcf90000fcf90000d4
:10851000fcf90000c2f80000e8d00000eaf8000012
:10852000fcf80000e8d0000000000000000000009f
:1085300005000000410000003f0000004200000074
:1085400043000000000000000000000000000000e8
:1085500000000000e8d00000fcf90000fcf9000079
:10856000fcf90000fcf90000c2f80000ccf80000a3
:10857000e8d00000fcf80000e8d000000000000097
:108580000000000005000000380000003f0000006f
:10859000440000003800000000000000000000005f
:1085a0000000000000000000e8d00000fcf900001e
:1085b000fcf90000fcf90000fcf90000c2f8000022
:1085c000ccf80000eaf80000e8d00000e8d0000095
:1085d00000000000000000000a000000e1000000b0
:1085e000e200000038000000380000000000000039
:1085f000000000000000000000000000e8d00000c3
:10860000fcf90000fcf90000fcf90000fcf9000096
:10861000e8d00000e8d00000e8d00000e8d000007a
:10862000c2fb000000000000000000003c00000051
:10863000450000003800000046000000380000003f
:10864000000000000000000000000000000000002a
:10865000dcfb0000e8d00000e8d00000e8d000001b
:10866000e8d0000062f800007af8000092f80000fc
:10867000aaf80000e8d000001e0000000000000082
:108680003c000000470000003800000048000000e7
:1086900038000000000000000000000000000000a2
:1086a00000000000ecfb0000e8d00000e8d0000073
:1086b000b4f900006af9000062f800007af80000de
:1086c00092f80000aaf80000e8d000001e000000a8
:1086d000000000003c0000004700000038000000df
:1086e0004900000038000000000000000000000009
:1086f000000000000000000010fc0000e8d00000b6
:10870000e8d00000b4f900006af9000062f8000047
:108710007af8000092f80000aaf80000e8d0000003
:108720001e000000000000003c00000047000000a8
:10873000380000004b00000038000000000000007e
:1087400000000000000000000000000034fc0000f9
:10875000e8d00000e8d00000b4f900006af9000099
:1087600062f800007af8000092f80000aaf8000011
:10877000e8d000001e000000000000003c000000e7
:1087800047000000380000004c00000038000000e6
:1087900000000000000000000000000000000000d9
:1087a00048fc0000e8d00000e8d00000b4f9000068
:1087b0006af9000062f800007af8000092f8000000
:1087c000aaf80000e8d000001e0000000000000031
:1087d0003c00000047000000380000005a00000084
:1087e0003800000000000000000000000000000051
:1087f000000000005efc0000e8d00000e8d00000af
:10880000b4f900006af9000062f800007af800008c
:1088100092f80000aaf80000e8d000001e00000056
:10882000000000003c00000047000000380000008d
:10883000610000003800000000000000000000009f
:1088400000000000000000006efc0000e8d0000006
:10885000e8d00000b4f900006af9000062f80000f6
:108860007af8000092f80000aaf80000e8d00000b2
:108870001e000000000000003c0000004700000057
:108880003800000068000000380000000000000010
:108890000000000000000000000000007efc00005e
:1088a000e8d00000e8d00000b4f900006af9000048
:1088b00062f800007af8000092f80000aaf80000c0
:1088c000e8d000001e000000000000003c00000096
:1088d0004700000038000000690000003800000078
:1088e0000000000000000000000000000000000088
:1088f0008efc0000e8d00000e8d00000b4f90000d1
:108900006af9000062f800007af8000092f80000ae
:10891000aaf80000e8d000001e00000000000000df
:108920003c000000470000003800000090000000fc
:1089300092000000000000000000000000000000a5
:10894000000000009efc0000e8d00000e8d000001d
:10895000b4f900006af9000062f800007af800003b
:1089600092f80000aaf80000e8d000001e00000005
:10897000000000003c00000047000000380000003c
:1089800091000000920000000000000000000000c4
:108990000000000000000000c6fc0000e8d000005d
:1089a000e8d00000b4f900006af9000062f80000a5
:1089b0007af8000092f80000aaf80000e8d0000061
:1089c00018000000000000003c000000470000000c
:1089d000380000006a0000003800000000000000bd
:1089e000000000000000000000000000eefc00009d
:1089f000e8d00000e8d00000b4f900006af90000f7
:108a000062f800007af8000092f80000aaf800006e
:108a1000e8d0000018000000000000003c0000004a
:108a2000470000003800000074000000380000001b
:108a30000000000000000000000000000000000036
:108a40001efd0000e8d00000e8d00000b4f90000ee
:108a50006af9000062f800007af8000092f800005d
:108a6000aaf80000e8d000001c0000000000000090
:108a70003c000000470000003800000051000000ea
:108a800038000000000000000000000000000000ae
:108a90000000000056fd0000e8d00000e8d0000013
:108aa000b4f900006af9000062f800007af80000ea
:108ab00092f80000aaf8000068fd0000180000000d
:108ac000000000003c0000004700000038000000eb
:108ad000ea00000038000000000000000000000074
:108ae000000000000000000070fd0000e8d0000061
:108af000e8d00000b4f900006af9000062f8000054
:108b00007af8000092f80000aaf80000e8d000000f
:108b1000180000000000000058020000470000009c
:108b2000380000008a00000038000000000000004b
:108b300000000000000000000000000080fd0000b8
:108b4000e8d00000e8d00000b4f900006af90000a5
:108b500062f800007af8000092f80000aaf800001d
:108b6000e8d0000018000000000000003c000000f9
:108b700047000000380000006600000038000000d8
:108b800000000000000000000000000000000000e5
:108b900090fd0000e8d00000e8d00000b4f900002b
:108ba0006af9000062f800007af8000092f800000c
:108bb000aaf80000e8d00000180000000000000043
:108bc0003c00000047000000380000006700000083
:108bd000380000000000000000000000000000005d
:108be00000000000bcfd0000e8d00000e8d000005c
:108bf000b4f900006af9000062f800007af8000099
:108c000092f80000aaf80000e8d000001800000068
:108c1000000000003c000000470000003800000099
:108c2000950000009200000000000000000000001d
:108c30000000000000000000e8fd0000e8d0000097
:108c4000e8d00000b4f900006af9000062f8000002
:108c50007af8000092f80000aaf80000e8d00000be
:108c600018000000000000003c0000004700000069
:108c70003800000096000000920000000000000094
:108c8000000000000000000000000000f8fd0000ef
:108c9000e8d00000e8d00000b4f900006af9000054
:108ca00062f800007af8000092f80000aaf80000cc
:108cb000e8d0000018000000000000003c000000a8
:108cc00047000000380000009b0000009c000000ee
:108cd0000000000000000000000000000000000094
:108ce00008fe0000e8d00000e8d00000b4f9000061
:108cf0006af9000062f800007af8000092f80000bb
:108d0000aaf80000e8d000001800000000000000f1
:108d10003c0000004700000038000000b2000000e6
:108d2000b300000000000000000000000000000090
:108d30000000000018fe0000e8d00000e8d00000ad
:108d4000b4f900006af9000062f800007af8000047
:108d500092f80000aaf80000e8d000001800000017
:108d6000000000003c000000470000003800000048
:108d7000be000000bf000000000000000000000076
:108d8000000000000000000028fe0000e8d0000005
:108d9000e8d00000b4f900006af9000062f80000b1
:108da0007af8000092f80000aaf80000e8d000006d
:108db00018000000000000003c0000004700000018
:108dc00038000000c3000000c400000000000000e4
:108dd00000000000000000000000000038fe00005d
:108de000e8d00000e8d00000b4f900006af9000003
:108df00062f800007af8000092f80000aaf800007b
:108e0000e8d0000018000000000000003c00000056
:108e10004700000038000000c800000038000000d3
:108e20000000000000000000000000000000000042
:108e300054fe0000e8d00000e8d00000b4f90000c3
:108e40006af9000062f800007af8000092f8000069
:108e5000aaf80000e8d000001000000000000000a8
:108e60000a0000004700000038000000c9000000b0
:108e700038000000000000000000000000000000ba
:108e8000000000005efe0000e8d00000e8d0000016
:108e9000b4f900006af9000062f800007af80000f6
:108ea00092f80000aaf80000e8d000001e000000c0
:108eb000000000003c0000004700000038000000f7
:108ec000cf0000003800000000000000000000009b
:108ed00000000000000000006efe0000e8d000006e
:108ee000e8d00000b4f900006af9000062f8000060
:108ef0007af8000092f80000aaf80000e8d000001c
:108f000000080000000000003c00000038000000e5
:108f100038000000380000003800000000000000a9
:108f20000000000000000000000000008cfe0000b7
:108f30009cfe000032ff0000c8ff0000f8ff0000a8
:108f400062f800007af8000092f80000aaf8000029
:108f50008852000000090000000000003c000000f2
:108f60003800000038000000380000003800000021
:108f700000000000000000000000000000000000f1
:108f80008c52000090520000945200009852000051
:108f90009c52000062f800007af8000092f800008d
:108fa000aaf80000a0520000000800000000000025
:108fb0000200000048000000380000004a000000e5
:108fc0003800000000000000000000000000000069
:108fd00000000000a4520000e8d00000e8d000002b
:108fe000a8520000a852000062f800007af80000c1
:108ff00092f80000aaf80000e8d000000009000084
:1090000000000000020000004900000038000000dd
:109010004a000000380000000000000000000000ce
:109020000000000000000000ac520000e8d000008a
:10903000e8d00000b0520000b052000062f800001a
:109040007af8000092f80000aaf80000e8d00000ca
:10905000000c0000000000003c0000005a0000006e
:10906000380000003800000038000000491d0000f2
:109070005d0000000000000001000000b45200008c
:10908000b8520000bc520000c0520000c4520000a0
:1090900062f800007af8000092f80000aaf80000d8
:1090a000c85200000026000000000000140000006c
:1090b000c50000005e0000005f00000060000000ce
:1090c00000000000000000000000000000000000a0
:1090d000cc520000e8d00000e8d00000e8d000004a
:1090e000e8d0000062f800007af8000092f8000072
:1090f000aaf80000e8d00000000d00000000000009
:109100003c00000061000000380000003800000052
:10911000380000004c20000060000000000000004b
:1091200001000000d0520000d4520000d8520000cc
:10913000dc520000dc52000062f800007af8000007
:1091400092f80000aaf80000e052000000170000aa
:10915000000000003c000000380000003800000063
:10916000380000003800000000000000000000008f
:109170000000000000000000e4520000e85200007f
:10918000e8520000ec520000f052000062f80000cb
:109190007af8000092f80000aaf80000e8d0000079
:1091a00000170000000000003c0000003800000034
:1091b0003800000038000000380000000000000007
:1091c000000000000000000000000000f452000059
:1091d000f8520000fc52000000530000045300004d
:1091e00062f800007af8000092f80000aaf8000087
:1091f0000853000000180000000000003c000000c0
:10920000380000003800000038000000380000007e
:10921000000000000000000000000000000000004e
:109220000c530000105300001053000014530000b2
:109230001853000062f800007af8000092f800006d
:10924000aaf80000e8d000000018000000000000ac
:109250003c0000003800000038000000380000002a
:1092600038000000000000000000000000000000c6
:10927000000000001c530000f8520000fc520000e7
:10928000005300000453000062f800007af8000068
:1092900092f80000aaf8000008530000000b00003c
:1092a00000000000040000004d0000004e0000001f
:1092b0004f0000005000000000000000000000000f
:1092c0000000000000000000e8d00000e8d000002e
:1092d000e8d00000e8d00000e8d00000e8d00000ae
:1092e000e8d00000e8d00000e8d00000e8d000009e
:1092f000000e0000960000003c0000006800000026
:10930000380000003800000038000000171a000084
:109310001d20000023000000010000002053000079
:1093200024530000285300002c5300003053000049
:1093300062f800007af8000092f80000aaf8000035
:109340003453000000000000000000003c0000005a
